:020000040800F2
:100000000080001011640008C1700008C57000086D
:10001000C9700008CD700008D17000080000000011
:10002000000000000000000000000000D570000883
:10003000D970000800000000DD700008D508000835
:10004000D3080008B3680008BB690008636A0008A9
:100050006F6B0008E36B0008DF6C0008F36C0008AE
:10006000E1700008476E0008F36E000809340008CC
:1000700015340008213400082D34000839340008F4
:1000800045340008513400088B6F0008CB6F00081E
:100090001F700008BF700008C3700008E9700008F6
:1000A000C7700008CB700008CF700008D37000083C
:1000B000D7700008DB700008DF700008E7700008E8
:1000C000EF70000873720008CB720008E772000836
:1000D000177300085D340008693400081B790008B4
:1000E00093790008737A00087B7A0008937A0008F5
:1000F000977A00089B7A00082B860008078700087B
:10010000778800083B8A0008678A00086B8B000824
:10011000DB8B0008278C0008CB8C00086F8F000851
:10012000BB8F0008E38F00089B9000080B9100082C
:100130008B910008279200085792000887920008C8
:10014000A792000807990008A39B00080000000080
:10015000000000000000000000000000000000009F
:10016000000000000000000000000000C79B000825
:10017000F39B00080B9C0008AB9D0008979E0008AD
:100180008FA000083BA10008E7A10008A7A2000873
:10019000D3A2000800000000E7A20008CFA30008D7
:1001A000E3A30008E7A90008DFAC00080BAD0008D6
:1001B00037AD0008BFAE00080FAF000837AF00082A
:1001C000B7B10008FBB10008D3B200080FB50008B2
:0801D000D3B5000883B6000856
:1001D80084B041F24870C1F20000006845F2ED5168
:1001E800CAF6CE41884200F0688303F0FFF903F0B5
:1001F80005F841F28070C1F2000000684DF6836195
:10020800C4F21B31A0FB01014BF61670890CC0F635
:1002180000000EF015F902F03FFE06F0CBFB02F0ED
:10022800EFFA02F053FB02F09FFB06F0EDFA06F03E
:100238003DFB02F0E5FD02F009FE06F095FC02F038
:10024800D7FE06F0BFFE03F02BF903F06DF903F0BB
:10025800B3F902F09BFD06F095FE02F07DFF4EF229
:100268009860C0F600000BF09EFA0DF03BF805F020
:10027800FBFF0BF0EDFE05F075FE032818D8DFE84C
:1002880000F00209100240F20000C1F200000BF079
:1002980051FF0DE040F20000C1F200000CF008F838
:1002A80006E040F20000C1F2000000210CF010F955
:1002B80041F2902040F2000AC1F20000C1F2000AA7
:1002C80004F014F94FF090404FF4806109F066FC97
:1002D800B0B9322003F0C8F94FF090404FF4806174
:1002E80009F05CFC60B94EF2A760C0F600000BF0A4
:1002F8005AFA40F20000C1F2000001210CF0E8F8BF
:1003080041F29026C1F20006304604F0EFF806F0FC
:1003180065FC40F20007DAF81010BAF81420BAF8B1
:10032800163040F68C25C2F20007C1F200053846A7
:1003380000950CF029FB304604F0D8F801F06CF970
:1003480040F664540025C1F20004C4F27F0520463B
:10035800294608F067F940F6F840C1F2000029463E
:1003680008F060F940F68C40C1F200007F2108F0E7
:1003780059F940F62040C1F20000294608F052F928
:1003880040F6B430C1F200007F2108F04BF9304646
:1003980004F0ACF840F23421C2F2000120464022B9
:1003A80008F0AEF9002840F0868240F68C4040F212
:1003B8003431C1F20000C2F20001032203F070F9E7
:1003C800002840F0788240F6204040F24031C1F2E7
:1003D8000000C2F20001012203F062F9002840F097
:1003E8006A8240F6B43040F24431C1F20000C2F2F1
:1003F8000001042203F054F9002840F05C8241F225
:100408009024C1F20004204604F070F805F07CFA4C
:10041800204604F06BF84DF62B10C0F600000BF0E8
:10042800C2F90CF023FCBAF8180020B341F290246A
:100438000025C1F2000400BF4FF0904020210122A6
:1004480003F0C4FD4FF4AF7003F00EF9204604F03A
:100458004DF84FF090402021002203F0B7FD4FF4F3
:10046800AF7003F001F9204604F040F8BAF818001C
:1004780001358542E0D341F2C0259FEDDB8B9FED2E
:10048800DC9B9FEDDDABC1F20005002000264FF09C
:10049800000B039008E000BF40F62030C1F20000D6
:1004A8002221C0F88C10464641F29020C1F200008B
:1004B80004F01CF82868012834D140F23424C2F230
:1004C8000004B4F8FE0001F01FF8B4F8FC0001F0D5
:1004D80093FB01F079FADAF8D800DAF8E4104FF46F
:1004E8007A7281FB000100230DF088FACAF808012E
:1004F800DAF8D800DAF890114FF47A7281FB00012B
:1005080000230DF07BFACAF884010020286040F629
:100518006450C1F200002146402208F0F1F800289A
:1005280040F0C98141F2BC20C1F2000000680128F6
:1005380006D140F23430C2F20000006801F0D8FC65
:1005480041F2B820C1F200000068012806D140F24B
:100558004030C2F20000006801F01EFD41F2B420F4
:10056800C1F200000068012845D140F24439C2F2C6
:100578000009D9F8000001F09FF8D9F8040001F04B
:100588008BFBD9F8080006F079F858EC187B3A4646
:10059800434605F051FF55EC194B22462B4605F012
:1005A8004BFFCDF808B0D346019656EC1AAB52462D
:1005B800334605F041FF0DF0BBF9ABF85001D9F80F
:1005C8000C0006F05BF83A46434605F035FF224634
:1005D8002B4605F031FF5246DA46DDF808B040F206
:1005E80000073346019EC2F2000705F025FF0DF013
:1005F8009FF9AAF8520141F2B020C1F20000006848
:1006080001280BD105F03EFC01F01EF9AAF898016B
:1006180041F2B020C1F200000021016003F01EF891
:10062800841B804618BF0124BAF85401BBF1000F9F
:100638004FF00005C8BF012504281BD34DF68210D2
:10064800C0F600000BF0AFF840F20046C4F6000612
:100658004FF0070930464FF400610022AAF80691CE
:1006680003F0B4FC30464FF480510022AAF80691FA
:1006780003F0ACFC41F24420C1F2000000680168BC
:100688004068039801F00F0686422ED0DAF8280158
:100698000130CAF82801DAF824010130CAF8240127
:1006A800DAF820010130CAF8200141F2AC20C1F289
:1006B8000000006820B94FF09040102109F080FA3E
:1006C80000F0FEFB01F094FC0CF0E2FA0CF0A8FB41
:1006D8000CF0E6FD02F0D4FD01F072FBAAF89C01D3
:1006E80001F086F8AAF816010396BAF81A0000284D
:1006F80000F08D8097F82600002840F08880BAF82E
:100708001A0040F2F13188420DDC01380A2821D85C
:10071800DFE800F0063A3E3320D0534337475F0006
:10072800504600216EE0B0F57D7F1ADB58D040F2CC
:10073800D241884264D041F2525188420AD141F2F2
:10074800487045F2ED51C1F20000CAF6CE41016091
:1007580003F0F6F84EF61060C0F600000BF023F830
:1007680052E040F2F231884236D040F2F33188420A
:10077800F0D1012006F0BAFA46E050460BF098FD99
:1007880042E005F0A5F83FE050460BF0D3FC3BE013
:10079800504601210BF09CFE36E050460BF030FC31
:1007A80032E0504600F094F840F23420C2F20000E3
:1007B800B0F8FC0001F0D0F926E050460BF000FC40
:1007C80040F23420C2F20000B0F8FC000CF0A4F8AB
:1007D8001AE000F029F917E0002006F087FA13E084
:1007E80006F02EFB10E000BF000000000070A740DC
:1007F8000000000000003540000000000000F03E4E
:10080800504601210BF060FF0020AAF81A0004EA04
:100818000500ABEB000B4FF090404FF4806109F0FE
:10082800BDF998B941F2C025BBF1000FC1F200052E
:1008380024D10A2002F018FF4FF090404FF4806155
:1008480009F0ACF938B14FF0000B17E041F2C025C0
:10085800C1F2000512E041F2AC21C1F200010868C2
:1008680010B10020086007E0012008604FF09040B8
:100878001021012203F0AAFB4FF4FA7B384605F059
:1008880071FC002846463FF40FAE38460CF006F9D6
:1008980002287FF401AE41F2AC20C1F200000068EA
:1008A800464600287FF400AE38460CF043F9464629
:1008B800FAE500BFFEE706F00FFA41F248710020A2
:0A08C800C1F20001086002F05FFCBD
:0208D200FEE73F
:0408D40006F0FABC74
:1008D8002DE9F04704464CF67630C0F600000DF0DE
:1008E800AFFDD4F89C00002800F08780D4F89C0065
:1008F8000DF058F89FED460B5AEC105B2A4653460C
:100908000CF018FF40F2E042C1F2000292ED000B39
:1009180056EC107B3A4633460CF00CFF9FED3E0B2D
:1009280058EC109B4A46434605F086FD05F094FEB8
:10093800C4F89400B4F8CE003A46A4F89800B4F885
:10094800CC003346A4F89A004EF6D530C0F6000025
:100958000DF076FDD4F89C000DF024F82A46534695
:100968000CF0E8FE02464EF65C00C0F600000B46AE
:100978000DF066FDB4F998000DF014F89FED280B02
:1009880055EC106B32462B460CF0D4FE02464EF660
:100998006B00C0F600000B460DF052FDB4F99A004A
:1009A8000DF000F832462B460CF0C4FE02464CF619
:1009B800BA30C0F600000B460DF042FDD4F89400A2
:1009C80005F05CFE4A46434605F036FD02464EF603
:1009D8001470C0F600000B460DF032FD4CF65E4078
:1009E800C0F600000DF02CFD40F20000C1F200003E
:1009F8000021BDE8F0470BF067BE4EF6F230C0F6B6
:100A08000000BDE8F0470AF0CEBE00BF00BF00BF3F
:100A18000000000000408F400000000080842E414C
:080A280000000000000059402D
:100A30002DE9F04F81B04EF67600C0F600000DF0C3
:100A400003FD40F2000AC1F2000ABAF8CE00AAF88B
:100A5000A000BAF9A0000CF0A9FF9FED490B54ECDF
:100A6000109B4A46234600940CF068FE02464EF660
:100A70008D00C0F600000B460DF0E6FCBAF9CE0082
:100A8000BAF99810401A0CF091FF4A4623460746DF
:100A90008B460CF053FE02464CF68A40C0F600002E
:100AA0000B460DF0D1FC40F2D040C1F2000090EDB9
:100AB000000B4EF69C0056EC104BC0F60000224690
:100AC00033460DF0C1FCDAF89C000CF06FFF9FED8F
:100AD0002E0B55EC108B42462B460CF02FFE024697
:100AE0004CF61E60C0F600000B460DF0ADFCDAF8C7
:100AF0009C000CF05BFF42462B460CF01FFE22468A
:100B000033460CF01BFE9FED220B53EC102B0CF028
:100B1000F5FC3A465B460CF011FE9FED1F0B54ECC2
:100B2000105B2A46234605F08BFC0CF005FFCAF843
:100B3000A400DAF8A4000CF039FF2A4623460CF092
:100B4000FDFD009B4A4605F07BFC9FED150B53EC29
:100B5000102B0CF0D3FC02464EF6CF00C0F600007E
:100B60000B460DF071FC4EF62870C0F600000DF03B
:100B70006BFC5046002101B0BDE8F04F0BF0A8BD62
:100B800000000000000059400000000000408F40BD
:100B9000000000000000F0BF0000000065CDCD4166
:080BA000000000000000F03F1E
:100BA8002DE9F04F87B04EF61240049041F26C20C8
:100BB80004AD0024C1F2000029460222CDE9054413
:100BC80008F008F88DF812008DF80C40CDE90144C2
:100BD80040F6D05001AC4FF47A77C1F200002946B4
:100BE80022460923009704F03FF89DF8040040F2DC
:100BF800000AFF28C1F2000A34D19DF805009DF8CB
:100C0800101088422ED19DF806009DF811108842D8
:100C180028D19DF807009DF81210884222D141F290
:100C28006C209DF80C50211DC1F20000042207F031
:100C3800D1FFA84216D19DF8080000F0CC00842806
:100C480010D19DF909109DF80B209DF80A00CBB230
:100C580042EA034242EA002000F17F42002948BFED
:100C6800501C07E0BAF882010130AAF8820104F0AA
:100C78004BFE002041F2143BC1F2000BDBF80010E0
:100C88006FF0004291421CBF0131CBF8001041F2D5
:100C98001831C1F200010A6802EBD2731044A0EBCC
:100CA8006300086000EBD0704110CAF88811DAF8C8
:100CB8007810C1EB600441F2DC20C1F2000004604E
:100CC800DAF8D400DAF88010DAF88820401A5043AD
:100CD8000CF068FE9FED680B58EC109B4A464346A3
:100CE8000CF028FD0CF024FECAF88C01251A41F2FC
:100CF800E420C1F200000560BAF9CC00BAF97E1010
:100D0800401A0CF04FFE0446DAF890000E460CF03C
:100D180049FE2246334605F08FFB4A4643460CF00F
:100D280009FD0CF005FE41F2E021281AC1F200018C
:100D380008600CF037FE9FED520B53EC102B05F0BA
:100D48007BFB9FED510B53EC102B05F075FB9FEDD2
:100D5800500B53EC102B05F06FFB064641EC100BC3
:100D680040F2E040C1F2000080ED000BDAF8940098
:100D78000F4605F083FC9FED480B53EC102B0CF04D
:100D8800D9FC32463B4605F057FB064641EC100BB2
:100D980040F2D040C1F2000080ED000B0F46BAF9D6
:100DA800CE00BAF99810401A0CF0FCFD0446DAF8A7
:100DB800A4000D460CF0F6FD9FED390B53EC102BFB
:100DC8000CF0B8FC22462B4605F036FB9FED360B9F
:100DD80053EC102B0CF08EFB02460B46304639467E
:100DE80005F02AFB044641EC100B40F2D8409FED79
:100DF800301BC1F200000E4680ED000B51EC110BC8
:100E08009FED2D0BC80F314660F3DF7153EC102BAB
:100E1800204605F0A9FB10B1DAF8900107E020465A
:100E280031464A46434605F007FB0CF081FDCAF8F7
:100E3800E400DBF80000152813DBDAF8E400DAF840
:100E4800E8108842C4BFDAF8E400CAF8E800DAF823
:100E5800E400DAF8EC108842BCBFDAF8E400CAF81B
:100E6800EC0041F2B020C1F200000121016007B09E
:100E7800BDE8F08F00BF00BF0000000000408F40B9
:100E88000000000000000840000000000000494089
:100E9800000000000000803E0000000080842E4119
:100EA8000000000065CDCD41000000000000F03FCB
:100EB8000000000000000000000000000020614069
:100EC8002DE9F04F81B02DED028B86B040F2000580
:100ED80040F2F84BC1F20005C1F2000BD5F85CA056
:100EE800DBE900014EF680620843C0F2360205D104
:100EF800D5F82C0100215043CBE9000140F20056FF
:100F0800C1F20006D6E90001084305D1D5F8300141
:100F180000215043C6E90001D5F8E400B5F9701086
:100F2800B0EB010829D4B5F8520005F0A7FB9FEDF6
:100F3800C80B59EC106B32464B460CF0FBFB0746CE
:100F480040460C4605F09AFB02460B4638462146B9
:100F580005F072FA0446B5F9D6010F460CF022FDE9
:100F6800324640F200564B46C1F200060CF0E2FB56
:100F780002460B462046394642E0E86DB5F868104F
:100F8800B0FBF1F77842804580F2668240460CF06B
:100F980009FD044641EC180B3846D1468A460CF048
:100FA80001FD8DED048B9DF81730024683F080001B
:100FB8008DF81700DDE904030F4619463B460CF08F
:100FC800B9FB41EC180BB5F8500005F057FB9FED45
:100FD800A20B53EC102B0CF0ADFB9FEDA10B53ECC7
:100FE800102B0CF087FA41EC110BB0EE480AF0EE2A
:100FF800680A0DF085F951EC100B22465346CA4693
:1010080005F01AFA0CF094FCC5F8F000D5F8E400E5
:10101800B0F1FF3F11DDD6E900014EF6806210EB1A
:10102800080041EBE871C0F236020023C6E900016E
:101038000CF01AFDC5F830011BE0DBE90001C8F12E
:101048000002801841EBE2714EF68062C0F236026F
:101058000023CBE900010CF007FDC5F82C01D5F8F9
:101068002C014FF47A71EA6D4843B0FBF2F0A5F811
:101078003C01D5F8F000D5E93E120023091842EBEF
:10108800E070C5E93E10D5F8F000D5E958124FF4E4
:101098006164091842EBE070C5E95810D5E95801B8
:1010A8004FF461620CF0AAFCC5F84001D5F80001C4
:1010B80041F2A4290028C1F2000902DCD9F8000095
:1010C80080B1D5E970014FF4616210EB080041EB83
:1010D800E871C5E97001D5E9700100230CF08EFCB8
:1010E800C5F8C801D5F8E400D5E978120023091835
:1010F80042EBE070C5E97810D5E978014FF46162F8
:10110800AAFB04470CF07AFCC5F8D801D5F8D80139
:1011180000284FF47A7006D0D5F84011D5F8D821B8
:10112800484390FBF2F0A5F8D601D5E93E01201A14
:1011380077EB0100B8BFC5E93E47D5E9580101384A
:1011480071F1000008DB0020C5E95800C5F840012E
:10115800C5E97800C5F8D801E86DB5F85410D5F898
:10116800D820B5F8583041F234369A42C1F2000618
:101178001CDD484305F082FA9FEDE10B53EC102B80
:101188000CF0D8FA05F028FAD5F8E420D317101A8D
:1011980073EB01000ADA308801303080B5F8561058
:1011A80000B2884204DDB5F8560000E00020308027
:1011B800B6F90000B5F8561088425CDB0020C5E996
:1011C8003E47C5E95800C5F840010CF005F9D9F8C3
:1011D8000000002804BF0120C9F8000041F2A8203F
:1011E800C1F20000016801293ED100210160D5F853
:1011F800E8014EF68064D5E97023C0F23604A0FBFE
:1012080004010CF0FBFBA5F84401D5F8EC01D5E985
:101218006E23A0FB04010CF0F1FBA5F84601D5F8FC
:101228002811D5F8C821D5F82431B5F94401B5F904
:101238004671D5F8D860D5F8E440CDE900074EF6F8
:101248006870C0F60000029603940DF0F9F812E0F9
:101258000000000000408F400000000000005940DE
:10126800000000000000F0BF0020C5E97000C5F8CC
:10127800C801C5E96E00D5E93E014FF4616200235B
:101288000CF0BCFBC5F8F400B5F8B800002859D03C
:10129800B5F85001B0F57A7F40F2BD80B5F852013B
:1012A800C0087C2800F2B78041F23230C1F2000059
:1012B800018801318AB20A2A0180C0F0B280D9F8C7
:1012C80000100A220129028040F09380D5F82001FD
:1012D800B0F5616FC0F08D80D5F8200142F600713D
:1012E800C0F20D01884200F2848004F0CDFD0CF0BC
:1012F8005DF84FF2F014D5E97001CFF6FF7422467D
:101308004FF0FF330CF07AFBC5F8E801D5E96E0120
:1013180022464FF0FF330CF071FBC5F8EC01D5F80D
:101328002811D5F80C21D5F8E831D5F82001D5F8E1
:10133800D870D5F8E460CDE900074EF66B10C0F61A
:10134800000053E0D5F8D800B5F88011884262DA79
:10135800D5F8D800B0F57A7F5DDD41F23230C1F2C0
:101368000000018801318AB20A2A018059D3D9F8CC
:1013780000100A22012902803BD1D5F82001B0F5DE
:10138800966F36D3D5F820014FF68041C0F20A0196
:1013980088422ED804F078FD0CF008F84FF2F014CB
:1013A800D5E97001CFF6FF7422464FF0FF330CF0F9
:1013B80025FBC5F8E801D5E96E0122464FF0FF3359
:1013C8000CF01CFBC5F8EC01D5F82811D5F80C2158
:1013D800D5F8E831D5F82001D5F8D870D5F8E4600B
:1013E800CDE900074EF62810C0F6000002960DF071
:1013F80027F841F2A8210020C1F200010122C5F816
:101408002401C9F800000A60C5E97000C5F8C801E0
:10141800C5E96E0005E041F23230C1F2000000215A
:101428000180B5F8640048F2A0640428C0F2010401
:1014380020D8DFE800F0031C16191300EA6DD5E97F
:101448003E014FF46167A0FB040301FB0431A2FBDA
:1014580007230CF0D3FA0EE04046D5E504F082FFEE
:1014680009E004F031FF06E004F048FF03E004F06F
:1014780019FD00E00020C5F80001EA6DD5E93E013C
:101488004FF46167A0FB040301FB0431A2FB0723AF
:101498000CF0B4FA48F21F54C5F2EB1450FB04F0F8
:1014A800410901EBD070A5F8CC0104F0FBFC50FB1E
:1014B80004F0410901EBD070A5F8CE0104F004FF57
:1014C80050FB04F0410901EBD070A5F8D00104F0FD
:1014D80015FF50FB04F0410901EBD070A5F8D201CB
:1014E80004F040FF50FB04F0410901EBD070A5F86F
:1014F800D40106B0BDEC028B01B0BDE8F08F00BF8F
:08150800000000000000594042
:101510002DE9F04F81B041F20C33C1F2000319689C
:101520006FF00042914280461CBF481C186041F297
:101530001030C1F200000168A1EB5111414401607B
:1015400048F20000CFF6FF7000EB51100CF02EFABD
:101550009FED2B0B59EC10AB52464B4604F070FF3D
:101560009FED290B5BEC104B22465B4604F068FFB5
:101570009FED270B55EC106B32462B4604F060FFB5
:101580000CF0DAF940F20007C1F20007C7F8D80002
:1015900041F20C30C1F200000068B0F5A07F13DD0D
:1015A000D7F8D800D7F8DC108842C4BFD7F8D800E5
:1015B000C7F8DC00D7F8D800D7F8E0108842BCBFE5
:1015C000D7F8D800C7F8E00040460CF0EFF99FEDDF
:1015D000120B53EC102B0BF091FF52464B4604F0CC
:1015E0002FFF22465B4604F02BFF32462B4604F0C9
:1015F00027FF0CF0A1F9C7F8940101B0BDE8F08F06
:10160000000000000070A74000000000000026401D
:10161000000000000000003F000000000000E0C0EB
:1016200080B547F2A850C1F6FF7001889FED221ADD
:1016300000EE101AB8EE400A9FED202A20EE010AB3
:1016400020EE020A41F2D421408CBCEEC00AC1F265
:10165000000181ED000A10EE101A00EE100AB8EE3B
:10166000400A20EE010A20EE020A41F2D820BCEE28
:10167000C00AC1F2000080ED000A10EE100A401A04
:1016800041F2D021C1F20001086004F0FBFF9FEDA0
:10169000080B53EC102B0CF051F841EC100B40F2FE
:1016A000C840C1F2000080ED000B80BD00BF00BF4C
:1016B000000000000000544000803B4500008039DD
:1016C000B0B540F6B8314843000C04F0DBFF0446E7
:1016D00041F2D420C1F2000000680D4604F0D2FFB0
:1016E00002460B462046294604F0A6FE40F2C842B8
:1016F000C1F2000292ED000B53EC102B0CF01EF81F
:101700009FED0B0B53EC102B0BF0F8FE9FED0A0B2B
:1017100053EC102B04F094FE0CF00EF940F2000193
:10172000C1F20001A1F8CC00BDE8B04004F0F2BB6A
:101730000000000000003E40000000000000594092
:10174000004B00000000010001000000000000004C
:101750000000000000000000000000000000000089
:101760000000000000000000000000000000000079
:1017700090D0030000000000000000000000000006
:1017800040420F000000000040420F000000000037
:101790000000000000000000FFFFFFFFFFFFFFFF51
:1017A00000D68AEAFFFFFFFF007884C9FDFFFFFF34
:1017B000DE0369000071020000401F000A00020001
:1017C000606DE06001000200C05DA861A073606D03
:1017D00083FF7D0070177C153CF630F870177C1580
:1017E00054F248F4320038FF204E07008403010011
:0817F0000100406A64000000E2
:1017F800B0B540F20005C1F20005B5F83C01C8B12A
:10180800D5F8340104F03AFF0446D5F838010D46FE
:1018180004F034FF02460B46204629460BF08AFFA7
:101828009FED070B53EC102B04F006FE0CF080F82C
:1018380000B2B0BD4FF6FF7000B2B0BD00BF00BF30
:081848000000000000005940FF
:101850002DE9F04740F2000941F20838C1F20009D1
:10186000C1F20008D9F82801D8F8001040F6E40ABF
:10187000401AC1F2000AA9F89A010AF1040051467F
:10188000FC220CF0A3FC40F2E475C1F20005281D17
:101890002946FC220CF09AFCD9F8E4000022CAF890
:1018A0000000D9F8D800002128606FF00040002324
:1018B0006FF000465AF82240002C48BF6442B44200
:1018C00038BF264655F822709C4288BF2346002F19
:1018D00048BF7F42874238BF38468F4202F101023B
:1018E00088BF3946402AE5D19D1B48BF6D42081A82
:1018F00048BF4042D9F85C10B9F86820B1FBF2F15A
:1019000046F26762C6F2666251FB02F1CA1002EB50
:10191000D1718D4205DA6FF00100013000B2BDE8EF
:10192000F087192804D24FF6FE7000B2BDE8F087A8
:1019300000234FF0FF314FF0FF3200BF0AEB830767
:101940007F685AF82360BF1B48BF7F429742C8BFD9
:10195000194603F10103C8BF3A463F2BEED12029B7
:101960002ED104F08FFE044628460E4604F08AFE6F
:1019700002460B46204631460BF0E0FE9FED120B6F
:1019800053EC102B04F05CFD0BF0D6FFA9F81C0102
:10199000D9F8280140F23422C8F8000009F2F220F8
:1019A0000021C2F2000200BF32F8213002EB8107B1
:1019B00020F8803C7B880131402920F80239F3D19E
:1019C000002000B2BDE8F087000000000088C3409E
:1019D0002DE9F04140F234276FF000404FF0FF3125
:1019E0000023C2F200074FF0FF36002237F82350E1
:1019F000A84228BF284688BF1E46AA429CBF2A4646
:101A000019460133402BF1D107EB810107EB860327
:101A100049885B88101AA1EB03080BF0C7FF9FED04
:101A2000440B53EC102B04F00BFD0BF085FF0BF077
:101A3000BDFF40F20005C1F200050446D5F8940050
:101A40000E4604F01FFE9FED3C0B53EC102B0BF0E9
:101A500075FE2246334604F0F3FC0BF06DFF04469E
:101A600040460BF0A3FF9FED360B53EC102B04F018
:101A7000E7FC9FED350B53EC102B04F0E1FC9FEDE0
:101A8000340B53EC102B04F0DBFC0BF055FFE96D2D
:101A9000B5F86820B1FBF2F146F26762C6F2666201
:101AA00051FB02F18A1002EBD171220048BF624261
:101AB0008A4205DA6FF00100411C08B2BDE8F081EE
:101AC00002004FF6FE7148BF42420A2A2CD30BF0A7
:101AD0006DFF804620460E460BF068FF02460B461F
:101AE000404631460BF02AFE9FED1B0B53EC102BAA
:101AF00004F0A6FC0BF020FFA5F81E01D5F8280184
:101B0000B81C002130F8022C05EB410382F400429E
:101B1000A3F8F42230F8042B013182F4004240296A
:101B2000A3F87423EED1002108B2BDE8F08100BF14
:101B300000000000804F12400000000080842E4111
:101B4000000000000070A7400000000000002640D8
:101B5000000000000000003F000000000088C340BB
:101B600070B540F20006C1F20006D6F8B010401A77
:101B7000A0F500400BF01AFF9FED170B53EC102B54
:101B800004F05EFC9FED160B53EC102B04F058FC98
:101B90009FED150B53EC102B0BF0D0FD9FED140BAC
:101BA00053EC102B0BF0CAFD0446D6F89C000D46F2
:101BB0000BF0FCFE22462B460BF0C0FD9FED0E0BFA
:101BC00053EC102B04F03CFC04F04AFDC6F8B400C2
:101BD00070BD00BF00BF00BF000000000070A74044
:101BE000000000000000003F000000000000444032
:101BF000FCA9F1D24D62403F0000000080842E41DC
:101C000070B540F20006C1F20006D6F8B010401AD6
:101C1000A0F500400BF0CAFE9FED170B53EC102B04
:101C200004F00EFC9FED160B53EC102B04F008FC97
:101C30009FED150B53EC102B0BF080FD9FED140B5B
:101C400053EC102B0BF07AFD0446D6F8B4000D4689
:101C500004F018FD9FED100B53EC102B0BF06EFDF4
:101C600022462B4604F0ECFB0BF066FEC6F8900112
:101C700070BD00BF00BF00BF000000000070A740A3
:101C8000000000000000003F000000000000444091
:101C9000FCA9F1D24D62403F0000000080842E413B
:101CA00010B540F20004C1F2000440F6B831A4F8C7
:101CB000C81004F0E7FC9FED0C0B53EC102B04F064
:101CC000BFFB9FED0B0B53EC102B04F0B9FB9FED0A
:101CD0000A0B53EC102B04F0B3FB0BF02DFEA4F811
:101CE000CA0010BD00BF00BF000000000070A74088
:101CF0000000000000000840000000000000F03E6E
:101D000070B50446049816460D4621604A6033B10A
:101D1000012B09D14FF480524FF4C06106E04FF41B
:101D200080524FF4806101E000210022013818BF89
:101D300001204003C5E902202846296109F05EFA26
:101D400038B14EF6C440C0F6000009F030FD04F092
:101D5000C7FF284603F080FCB6F5964F0CD80598CF
:101D600004F090FC9FED160B53EC102B04F068FB75
:101D700004F076FC01460BE040F2D6604DF683613C
:101D80007043C4F21B31A0FB0101012000EB914123
:101D9000284609F071FF28684FF48072016841F00D
:101DA0008061016054F8270B214603F0B3FB30B18A
:101DB0004DF23610C0F600000CF046FBFEE770BD99
:081DC0000000000000000C40CF
:101DC800F0B581B040F20004C1F20004B4F8580044
:101DD80004F054FC9FED420B53EC102B04F02CFB49
:101DE8000BF0A6FD41F2F425C1F20005B4F8581035
:101DF8002E68A4F89E61D4F8D87087420CDC084697
:101E080004F03CFC9FED380B53EC102B04F014FB52
:101E18000BF08EFD87420CDA41F2EC20C1F2000093
:101E2800002101606FF001002960013000B201B0AB
:101E3800F0BD41F2EC21C1F200010868002808BF9A
:101E48000F60086800F10A02974202DC0A388742EC
:101E580005DA00224FF6FE700A602A60E6E7D4F839
:101E6800E400B4F97020904206DA00200860286087
:101E78006FF001000138D9E7701C42F63121884221
:101E8800286006D3D4F8E400B4F87010401AA4F817
:101E98001801B4F9180101281EDBD4F8280144F20E
:101EA8000751CCF22E21A0FB010141F2F020C1F232
:101EB80000000268090C8A420ED0016041F2F82045
:101EC800C1F200000168B4F91821A1EB9111114485
:101ED80001608809A4F81A010020A7E700BF00BF25
:101EE8007B14AE47E17AF03F0AD7A3703D0AEF3F73
:101EF80080B50BF057FD9FED1E0B53EC102B04F033
:101F08009BFA9FED1D0B53EC102B04F095FA9FEDF7
:101F18001C0B53EC102B0BF0EDFA9FED1B0B53EC45
:101F2800102B0BF007FC9FED1A0B53EC102B04F051
:101F380083FA0BF0FDFC40F20001C1F20001A1F8A8
:101F4800CE00B1F9CE20B1F9D030B1F9CE009A4225
:101F580002DDA1F8D00080BDB1F9D2209042BCBF0B
:101F6800B1F8CE00A1F8D20080BD00BF00BF00BF0D
:101F7800000000000070A740000000000000F03ED4
:101F88000000000000C082C00000000000002440E3
:081F98000000000000005940A8
:101FA00080B5A0F500400BF001FD9FED0D0B53EC4B
:101FB000102B04F045FA9FED0C0B53EC102B04F0A2
:101FC0003FFA9FED0B0B53EC102B04F039FA04F0A1
:101FD00047FB40F20001C1F20001C1F8D40080BD0E
:101FE000000000000070A740000000000000264034
:081FF000000000000000003FAA
:101FF8002DE9F04F81B040F2E84AC1F2000ADAE96F
:10200800000140F2000408434EF68060C1F200046B
:10201800C0F2360005D1D4F8341100224143CAE990
:10202800001240F2F04BC1F2000BDBE90012114341
:1020380005D1D4F8381148430021CBE90001B4F8A0
:102048007250D4F8E400B4F97010B0EB010826D44B
:1020580040460BF0A7FC07462846894604F00EFBCD
:102068009FED510B55EC106B32462B460BF062FB83
:102078003A464B4604F0E0F98146B4F9D6010F46DA
:102088000BF090FC32462B460BF054FB02460B46F5
:102098004846394604F0D0F90BF04AFC01E0D4F880
:1020A800F000C4F87C01D4F87C01D4F8D8104FF4BF
:1020B8007A7281FB000100230BF0A0FC226ED4E9A8
:1020C8005C371B184F41C4E95C37D4E95A37C0184C
:1020D8007941C4E95A01D4F800014FF4616101283B
:1020E800A2FB01560EDBD4F8D8004FF47A7280FBBD
:1020F800080100230BF082FCD4E96E2380185941B3
:10210800C4E96E01D4E95C014FF46162281A76EBE8
:102118000100B8BFC4E95C56D4E95A01002301386C
:1021280071F10000A4BF0020C4E95A00D4E95A01A3
:102138000BF064FCC4F84801D4E95C014FF4616217
:1021480000230BF05BFCC4F87801D4F80801D4F83C
:102158000811B0F1FF3F12DDDBE90002002340184F
:1021680042EBE1714EF68062C0F23602CBE9000123
:102178000BF07AFCC4F8380101B0BDE8F08FDAE959
:1021880000024942401842EBE1714EF68062C0F20B
:1021980036020023CAE900010BF066FCC4F83401DA
:1021A80001B0BDE8F08F00BF0000000000408F4084
:1021B80050EC101B4FF0FF3202EB105240F2FE734E
:1021C8009A4280F09A802DE9F84F2DED028B82B06B
:1021D80001A809F0CAFC019F554B54EC105B284636
:1021E800214600220BF086F981468A46514B284643
:1021F800214600220BF07EF943F6CE32C6F27F620A
:10220800AA1A4AF29E02C3F6E67274EB0202BCBF37
:1022180054464D46804644EC105B0E46BEBF5646BB
:10222800C846013F4FF0FF300CF04AF851EC100B54
:10223800414B00220BF05EF902460B464046314600
:102248000BF078FA05460E4602460B4604F0F4F801
:1022580083468A4641EC180B42F2E079C0F6000941
:1022680048460221B0EE480AF0EE680A09F095FCEB
:1022780051EC100B314A324B0BF03CF904468846BE
:1022880009F110000321B0EE480AF0EE680A09F0DF
:10229800BEFC53EC102B204641460BF04BFA5A4635
:1022A800534604F0C9F82A46334604F0C5F82A46CE
:1022B80033460BF01FF90646884638460BF072FB8A
:1022C80004460D461F4A204B04F0B6F832464346F2
:1022D8000BF010F9064688461C4B2046294600227A
:1022E80004F0AAF8324643460BF004F941EC100B0F
:1022F80002B0BDEC028BBDE8F88F20F000434A42E3
:1023080040F20002C7F6F07272EB030308D31042E2
:1023180007D00028BCBF002102F5002040EC101BAC
:1023280070479FED010B7047000000000000F0FFB0
:102338000000E0BF0000F0BF0000E03F9AB5B31214
:10234800FF0750C0A80C615C10D02BBF0030E63FDF
:102358002DE9F04F83B056EC107BC6F30A500138D4
:1023680040F2FE71884280F0A98043F6EF10CFF664
:10237800FA60C01B42F64260C4F28600B041C0F267
:10238800B2804BF6D240CDF67A50C01B42F22B30C9
:10239800CCF28600B041C0F0898044F22320C0F618
:1023A800924026F00041381A49F6A140C3F6C730DA
:1023B80071EB00007DD3544D0195F00F2C4660F36E
:1023C800DF74524A524B3846314604F035F8002241
:1023D80023460BF08FF80BF0ABFA02900BF0E2FA01
:1023E800044688464B4B002204F026F83A4633460A
:1023F8000BF080F806460F46474A484B20464146B0
:1024080004F01AF832463B460BF074F880460C4646
:1024180002460B4604F010F806460F46404A414B68
:1024280004F00AF8404A414B0BF064F832463B4648
:1024380004F002F8A5F5801300220BF05BF8424681
:10244800234603F0F9FF82468B46394A394B30461A
:10245800394603F0F1FF384A384B0BF04BF8044685
:1024680088460020294652465B4603F0E1FF0546B0
:102478008946304639462246434603F0DDFF2A4660
:102488004B460BF037F802460B46504659460BF0C0
:1024980051F90022019B0BF02DF841EC100B02982A
:1024A800013003B0BDE8F04F0BF00ABF9FED100BF1
:1024B80001E09FED130B03B0BDE8F08F26F000405C
:1024C800794240F20001C7F6F07171EB0002F2D3D5
:1024D800484038437FF46FAF002EBCBF064607461E
:1024E80046EC107BE7E79FED040BE4E700BF00BF75
:1024F8000000000000000000000000000000F07F65
:10250800000000000000F03F0000E03F3CF92F9E73
:102518002C15F73F0030E6BFA80C615C10D02B3FAC
:102528001CDC586FA452F13EE0F6B36FE4707C3FB8
:102538000938DE6F993F403FB35142718E71AC3F0D
:102548002DE9F8432DED068BB0EE408AF0EE608A57
:1025580058EC104B0020C3F6F07088EA00012143C4
:1025680000F0A98055EC116B00F18042154200F093
:10257800A780C8F30A51013940F2FD73994279D80E
:10258800C5F30A51A1F2FF714FF60203CFF6FF73AC
:1025980099426FD3304629460BF0CAF907460BF02B
:1025A80001FAB7F1004F40D07040694008433CD170
:1025B8009FED799B002FB0EE49AAF0EE69AA25D0CD
:1025C8003E4648BF7E429FED74AB59EC1A4B55EC22
:1025D800188B4046294622464B4603F02DFFF2074A
:1025E80004BF4946204641EC1A0B4FEA56094046BB
:1025F800294642462B4603F01FFF012E04BF2946F9
:10260800404641EC180B5FEA0906DED151EC190B84
:1026180055EC1A8B42462B460BF08CF8002F5CBF0A
:102628002946404641EC110B08E02046414600226D
:10263800002303F0B5FF48B19FED651BB0EE410ADA
:10264800F0EE610ABDEC068BBDE8F8836FF3DF7826
:1026580048EC104BFFF7ACFD53EC102B30462946E5
:1026680003F0EAFE41EC100BBDEC068BBDE8F84325
:10267800FFF76EBE28F00041634272EB01031AD3E4
:1026880025F00043D6F1000972EB0303D6D318EA0C
:10269800020F18D088F0704383F07F63234331D052
:1026A80082EA080222434FD13DA0002DA8BF08307E
:1026B80090ED001BC2E7B0EE481AF0EE681ABDE7CD
:1026C8009FED351BBAE7304629460BF031F907462E
:1026D8000BF068F985EA010286EA00031A437FF4E1
:1026E80060AF37A0002DA8BF08304FEAD872D0E9F4
:1026F8000010034662F3DF73FA0708BF034643EC92
:10270800111B9BE726A0002DA8BF0830294690ED95
:10271800008B30460BF00CF904460BF043F959ECEA
:10272800183B70404FEAD8764A46694066F3DF7234
:10273800084318461CBF4A461846E10704BF4A46E4
:10274800184642EC110B79E700F1004202F1804390
:102758006B40334311D188EA020020439FED0E1BE2
:102768003FF46CAF4FF6FF70C3F6EF7014A28142CE
:1027780088BF083292ED001B60E7814208D388EADF
:1027880002000BA1204308BF083191ED001B55E75B
:102798009FED031B52E700BF000000000000F03F60
:1027A8000000000000000000000000000000F07FB2
:1027B800000000000000F07F000000000000F03F73
:1027C800000000000000F07F000000000000000092
:0827D800000000000000F87F82
:1027E000EDAF16204A62304029BD56B31544E9BF0B
:1027F00077900D9CFE0B88C07E2615FA838073406F
:082800000FCE674B80D541C0EB
:10280800B0B58CB040F664500024C1F200004FF01F
:10281800A0410422C0E9001482614FF480714FF492
:10282800805281830121C2631C2200F1440C0B9465
:10283800CDE90944CDE90744CDE90544CDE9034490
:10284800CDE90144C0E90244C0E90444016280F8CA
:102858002440C0E90B4480F8384080F840108023B9
:102868008CE81C00016504F053FD002818BF04F033
:1028780033FA4FF40040CDE90A0440F664500625C7
:10288800C1F2000009A9099505F0F2FF002818BF58
:1028980004F022FA0220C0F23040CDE901050120FF
:1028A80003900020C4F27F000490042005900020CB
:1028B800069040F66450C1F2000001A905F0EAF85C
:0C28C800002818BF04F008FA0CB0B0BDE6
:1028D40070B588B040F6F84040F200110024C1F20F
:1028E4000000C5F20001C0E900144FF48071818337
:1028F4004FF4805104250126C1631C2100F14403D7
:10290400CDE90644CDE90444CDE90244CDE90044CF
:10291400C0E90244C0E904448561066280F82440A9
:1029240080F8384080F84060802256C304F0F2FCFE
:10293400002818BF04F0D2F90820C0F69040009097
:102944000620CDE901060020C4F27F00CDE903058D
:1029540040F6F840C1F200006946059405F09CF881
:0C296400002818BF04F0BAF908B070BDDC
:1029700010B58CB040F68C4040F200410024C1F20A
:102980000000C5F20001C0E900144FF4807181839A
:10299000032101624FF4805101220823C1631C21ED
:1029A00000F1440C0B94CDE90944CDE90744CDE98D
:1029B0000544CDE90344CDE90144C0E90244C0E93E
:1029C0000442836180F82440C0E90B4480F8382039
:1029D00080F8402080238CE81A00026504F09CFCFB
:1029E000002818BF04F07CF940F68C40C1F20000CA
:1029F00009A9099405F040FF002818BF04F070F9F8
:102A00000220C0F23040019006200290072003907F
:102A10007F200490042005900020069040F68C4012
:102A2000C1F2000001A905F039F8002818BF04F030
:102A300057F941F20000C3F2602001900C2002908F
:102A400040F68C40C1F2000001A905F027F80028EB
:102A500018BF04F045F92020C1F2F0400190122087
:102A6000029040F68C40C1F2000001A905F016F872
:0C2A7000002818BF04F034F90CB010BDB1
:102A7C0070B59CB0044600201B90CDE91900CDE93F
:102A8C00170002A8542103F037FE206800F13040F3
:102A9C004FEA3020062800F27581DFE810F00700BD
:102AAC008800730173014500D60019014FF40040F2
:102ABC0002904FF08050139002A801F0B9FD00284D
:102ACC0018BF04F007F941F20431C1F200010A68A1
:102ADC0041F24C00C4F20200531C0B6042B9016875
:102AEC0041F400510160016801F400510191019918
:102AFC000168002641F001010160006817A900F08F
:102B0C000100019001980320CDE917004FF090408F
:102B1C00199606F0F3FE41F23C150820C1F20005AF
:102B2C00C4F20200052181E04FF4803002904FF096
:102B3C008040149002A801F07BFD002818BF04F01F
:102B4C00C9F841F20031C1F200010A6841F24C00AF
:102B5C00C4F20200531C0B6042B9016841F480417D
:102B6C000160016801F4804101910199016800261E
:102B7C0041F002010160006817A900F00200019009
:102B8C00019842F2030017900320189040F2004085
:102B9C00C4F60000199606F0B1FE0820C4F202003B
:102BAC0041F27C052830C1F200052521D0E04FF41C
:102BBC00004002904FF08050139002A801F038FDB5
:102BCC00002818BF04F086F841F20431C1F200016C
:102BDC000A6841F24C00C4F20200531C0B6042B96B
:102BEC00016841F400510160016801F40051019148
:102BFC0001990168002641F001010160006817A9E4
:102C0C0000F0010001900198C0201790032018904B
:102C1C004FF09040199606F071FE0820C4F20200A5
:102C2C0041F2DC051430C1F20005242180224FF45E
:102C3C0000734FF4006C28606960AE60EE602A612E
:102C4C006B61C5F818C0EE6193E04FF480300290D0
:102C5C004FF08040149002A801F0EAFC002818BF45
:102C6C0004F038F841F20031C1F200010A6841F277
:102C7C004C00C4F20200531C0B6042B9016841F4D1
:102C8C0080410160016801F4804101910199016862
:102C9C00002641F002010160006817A900F0020053
:102CAC00019001984FF4404017900320189040F287
:102CBC000040C4F60000199606F020FE0820C4F26D
:102CCC00020041F21C053C30C1F2000526213FE018
:102CDC004FF4803002904FF08040149002A801F025
:102CEC00A7FC002818BF03F0F5FF41F20031C1F238
:102CFC0000010A6841F24C00C4F20200531C0B6044
:102D0C0042B9016841F480410160016801F48041DD
:102D1C00019101990168002641F0010101600068F0
:102D2C0017A900F00100019001984FF44070179022
:102D3C00032018904FF09040199606F0DFFD082004
:102D4C00C4F2020040F6BC755030C1F200052721D8
:102D5C0080224FF480734FF4006C4FF0200E2860EB
:102D6C006960AE60EE602A616B61C5F818C0C5F889
:102D7C001CE028462E6205F0A3FF08B103F0AAFF61
:082D8C006565AC621CB070BD6E
:102D940080B541F26C2043F20001C1F20000C4F29C
:102DA4000201016040F201118180FF2300214FF0F4
:102DB400070C1022C0E9043181610121C0E902C27B
:102DC400016205F04FFE002814BFBDE8804080BDBD
:042DD40003F084BFC5
:102DD800006843F20001C4F20201884200D0704743
:102DE80081B041F24800C4F20200016841F4805108
:102DF8000160006800F480500090009801B07047AE
:102E080080B540F6986046F60001C1F20000C4F2B1
:102E180000010022C0E9001210210123C0E90222AA
:102E2800C0F80F20C0E90513C0E90733C0E909332A
:102E3800C0E90B33C0E90D22C26300F0D5FD0028BC
:0C2E480014BFBDE8804080BD03F046BF11
:102E540080B540F6346046F60041C1F20000C4F289
:102E640000010022C0E9001210210123C0E902225E
:102E7400C0F80F20C0E90513C0E90733C0E90933DE
:102E8400C0E90B33C0E90D22C26300F0AFFD002896
:0C2E940014BFBDE8804080BD03F020BFEB
:102EA0002DE9F04786B0002741F24C000597CDE9A7
:102EB0000377CDE90177C4F20200016840F20048CF
:102EC00041F0040101600168C4F6000801F004014A
:102ED00000910099016808F5806641F020010160C9
:102EE0000168002201F0200100910099016842F27E
:102EF000030441F001010160016801F0010100914A
:102F00000099016841F002010160016801F00201CD
:102F100000910099016841F008010160006842F2E7
:102F2000030100F0080000900098304601F052F8CC
:102F30004FF09040302100224FF0300901F04AF864
:102F400040464FF4E05100224FF4E05A01F042F8BD
:102F500001AD0194012430462946CDE9024704978A
:102F600006F0D2FC4FF090402946CDE90194CDE91E
:102F7000037706F0C9FC40462946CDE901A4CDE916
:102F8000037706F0C1FC4FF48060CDE901074FF0F4
:102F900090402946039406F0B7FC042001904FF4BA
:102FA000041608F500602946CDE9026406F0ACFC81
:102FB0008020CDE9010640462946039406F0A4FC92
:102FC0004FF40070CDE9010740462946039706F00B
:102FD0009BFC08200021002200F05EFC082000F08D
:102FE0009BFC17200021002200F056FC172000F067
:082FF00093FC06B0BDE8F08778
:102FF80080B541F29C1048F20041C1F20000C4F2D1
:10300800000148F2BE220023C2F2B1024FF0010CC7
:1030180080E80E10C0E90433C0E90633036206F005
:10302800F1FD002818BF03F057FE41F29C10C1F2D1
:103038000000002107F028F8002818BF03F04CFE14
:1030480041F29C10C1F20000002107F073F800283B
:0C30580014BFBDE8804080BD03F03EBE08
:10306400B0B59CB00446002502A854211B95CDE9B7
:103074001955CDE9175503F043FB206848F2004188
:10308400C4F20001884236D047F60001C4F20001C0
:10309400884261D14FF480700290002402A80B94FE
:1030A40001F0CAFA002818BF03F018FE41F24C05DB
:1030B400C4F20205286817A940F0040028602868B3
:1030C40000F00400019001984FF440701790122012
:1030D400CDE9180408201B9040F60000C4F6000057
:1030E4001A9406F00FFCE86840F08040E860E86855
:1030F40000F080402EE04FF40030029002A80C95BE
:1031040001F09AFA002818BF03F0E8FD41F24C04DC
:10311400C4F20204206817A940F00400206020686B
:1031240000F0040001900198C0201790122018901C
:103134000020CDE9190008201B9040F60000C4F6D9
:10314400000006F0DFFB206940F0020020612069E6
:0C31540000F00200019001981CB0B0BD1A
:1031600080B541F2902043F20001C1F20000C4F2A8
:1031700000014FF47A73032280E80E00C36007F069
:1031800033F8002814BFBDE8804080BD03F0A8BD1F
:1031900082B04EF28010CEF2000072B600214FF0E5
:1031A000FF3200BF00EB810340F8212001310829E4
:1031B000C3F80021F6D10020C1F6FF70D0E900016C
:1031C00080F3088841F26000C4F202000268012323
:1031D00042F001020260006800F0010001900198D5
:1031E0000020C4F20100026863F30202026062B6CA
:1031F00088474DF69B14C0F6000400BF204608F037
:04320000D6FAFBE718
:1032040070B594B006AC2046382103F079FA002555
:103214004FF400700595CDE90355CDE9015507F04C
:1032240061F807F055F841F29000C4F20200016819
:10323400032621F0180101602D2006904FF4803000
:103244000790012010210890CDE90B000220109175
:1032540008210D90CDE90E60CDE9111013902046A0
:1032640007F0BEF860B90F20CDE9010601A80321DB
:10327400CDE90355059507F0B5FB08B914B070BD49
:0432840003F02CFD2A
:10328800B0B540F2000541F2E821C1F20005C1F2F3
:103298000001D5F828010A68904200D1B0BD086045
:1032A80007F014F841F24424C1F200042046012139
:1032B8004BF6BE6201F0C4FCD5F82C212046022151
:1032C80001F0BEFCD5F830212046032101F0B8FCFE
:1032D800D5F834212046042101F0B2FCD5F8382174
:1032E8002046052101F0ACFCD5F82821204606210E
:1032F80001F0A6FCD5F80C212046072101F0A0FC1E
:10330800D5F810212046082101F09AFCD5F8402173
:103318002046092101F094FCD5F8482120460A21CD
:1033280001F08EFCD5F8F42020460B2101F088FC32
:10333800D5F8782120460C2101F082FCD5F8D82157
:0C33480020460D21BDE8B04001F07ABC29
:103354000A4601464DF6FE00C0F600000BF072B8B6
:1033640010B596B0044601A8542103F0C9F92068A9
:1033740042F60001C4F20001884201D016B010BD2B
:103384004FF4002001904FF48070159001A801F0D3
:1033940053F9002818BF03F0A1FC41F25800C4F20D
:1033A4000200816B41F400418163016841F4806152
:1033B4000160006800F480600090009816B010BDB1
:1033C40080B582B041F25800C4F20200816841F035
:1033D40001018160816801F0010101910199016895
:1033E40041F080510160006800F080500090009826
:1033F400022003F077FF00F04DF902B0BDE88040F1
:0434040006F0E4BF2B
:0C34080041F23C10C1F2000005F0BCBE17
:0C34140041F2DC00C1F2000005F0B6BE81
:0C34200041F27C00C1F2000005F0B0BEDB
:0C342C0041F21C00C1F2000005F0AABE35
:0C34380040F6BC70C1F2000005F0A4BE1C
:0C34440040F65C70C1F2000005F09EBE76
:0C34500040F6FC60C1F2000005F098BEE0
:0C345C0040F62030C1F2000008F0BAB9C0
:0C34680040F68C20C1F2000008F0B4B95E
:10347400802808D0042814D141F2B020C1F2000001
:1034840001210160704740F20000C1F20000B0F871
:1034940054110131A0F85411B0F856110131A0F8BB
:0434A4005611704706
:1034A80080B540F6203043F60001C1F20000C4F2B6
:1034B80001014FF49642002380E80E0000F10C0150
:1034C8004FF4806C4FF00C0E81E80850C0E90633C9
:1034D800C0E90833836207F08DFE002818BF03F0A7
:1034E800FBFB40F62030C1F20000002102F00EF98B
:1034F800002818BF03F0F0FB40F62030C1F20000AE
:10350800002102F075F9002818BF03F0E5FB40F62A
:103518002030C1F2000008F093FC002814BFBDE879
:08352800804080BD03F0D8BB18
:1035300010B540F68C20C1F2000044F2004C4FF46C
:1035400080530021C4F2000C4FF496424FF4806E79
:103550000C24C0E90231C0E90611C0E908118162FA
:103560004FF40041C0E900C2C0E904E4816307F000
:1035700045FE002818BF03F0B3FB40F68C20C1F2D3
:103580000000002102F0C6F8002818BF03F0A8FBD5
:1035900040F68C20C1F20000002102F02DF9002835
:1035A00018BF03F09DFB40F68C20C1F2000008F02C
:1035B0004BFC002814BFBDE8104010BD03F090BBC9
:1035C00080B540F2085045F60041C1F20000C4F257
:1035D000000101604FF4027181800221C17100215C
:1035E000816000F08DFF002814BFBDE8804080BDE1
:0435F00003F076BBB3
:1035F40080B5032000F032F90F2000F007F808B17D
:0C360400012080BDFFF7DCFE002080BD2F
:1036100041F27071C1F20001096809B310B50446A6
:1036200041F28070C1F200004FF47A720068B2FB80
:10363000F1F1B0FBF1F005F001FA01460F2C4FF06B
:1036400001000CD859B94FF0FF302146002200F09C
:1036500023F941F26C710020C1F200010C6010BD31
:04366000012070478E
:0C36640041F2A020C1F200000068704795
:10367000B0B50446FFF7F6FF054641F27070C1F29F
:1036800000000068611C18BF044400BFFFF7EAFF98
:08369000401BA042FAD3B0BDBB
:103698003020C4F20100016821F001010160704787
:1036A8002DE9F041036840F20016C5F20006B34266
:1036B8004FF4C16708BF4FF40277B3F1A04F03F18D
:1036C800304308BF4FF40277BC594FEA3323062B27
:1036D80026D8012707FA03F313F0730F20D00368E5
:1036E8009F687F0703D490F85870012F02D10220F9
:1036F800BDE8F08104F01F0706F5A0640125A34288
:1037080080F8585018BF002F1AD10D46904604462D
:1037180004F03CF9F0B1002184F85810BDE8F081BC
:103728004CF28A13C0F60003804618460F4640F252
:10373800DB711546FFF70AFE39462A464046CEE7B2
:10374800052FE2D0092FE0D0002180F85810012081
:10375800BDE8F0812168E06D40F601739843224688
:1037680000F58070B142E06509D040F20050C5F222
:1037780000008142084608BF06F5407001E04FF09E
:10378800A040884211BF002FD06D20F48010D06572
:10379800D06D43F60507C0044FF0000044BF106E1B
:1037A80020F006001066506D47F67526C0F6000733
:1037B800C0F6000647F67D240023C0F60004C0E9E1
:1037C8000B761C2744630F6082F858304B68144608
:1037D80043F010034B60CB682A4643F00103CB60EB
:1037E8004031434605F0FAFB21688A6822F000421E
:0C37F80022F03F0204328A60BDE8F0813C
:103804000146806AC36DC26D13F0500F05D0D20615
:103814000FD4406D426B0846104742F40071C165F5
:1038240001680B68CA681B0705D4910709D503F022
:103834005FBB04F02DB912F4406FF8D1C968890454
:10384400F5D4C16D21F48071C165C16DC9045EBF39
:0C385400C16D41F00101C16503F04ABBE9
:1038600010B504460338052806D34EF20A10C0F6F8
:103870000000A621FFF76EFD4EF60C50CEF20000C0
:1038800001684FF6FF02114064F30A2141F08061A4
:0838900041F0FD71016010BD63
:1038980070B515460E46102A044606D34EF20A1095
:1038A800C0F60000BE21FFF751FD102E06D34EF2E0
:1038B8000A10C0F60000BF21FFF748FD4EF60C5075
:1038C800CEF2000001684FF0FF33C1F3022181F00E
:1038D8000702042A28BF0422033903FA02F238BF78
:1038E800002126EA02028A4003FA01F125EA0101D1
:1038F8001143002C4FEA011105D44EF20040CEF2DC
:103908000000215470BD04F00F021044017270BD14
:10391800B0F1FF3F0DDD00F01F01012202FA01F1B5
:103928001C2202EAD0004EF20012CEF200028150B0
:1039380070474EF20A10C0F60000D221FFF706BD0C
:0439480000F000F893
:10394C004EF60C50BFF34F8FCEF2000001680422EC
:10395C0001F4E061C0F2FA5211430160BFF34F8FE2
:04396C0000BFFDE7B4
:10397000B0B55FEA520C10D0D0F800E0002300BFD1
:10398000CC18CD5A6488BCF1010C44EA054403F11B
:103990000403CEF80040F3D100E00023D2071EBF9D
:0C39A0000268C95A118000680068B0BDC0
:1039AC0070B5D0E913C4D0F854E0CCF80440BEF1A3
:1039BC00000F1CBFD0E9164CC4F804C0D0E910CEDF
:1039CC00046886680EF01F00012505FA00F0CCF89B
:1039DC00040008466360102E04BF10460A46A0601F
:0439EC00E26070BD68
:1039F000002800F005812DE9F0410446006846F2F8
:103A00000048C4F20008404513D046F60001C4F255
:103A1000000188420DD046F60041C4F20001884200
:103A200007D04EF6A460C0F600004FF49871FFF77F
:103A300091FC206840450AD16068102807D34EF6F3
:103A4000A460C0F6000040F23311FFF783FCA068C9
:103A5000002818BFB0F5807F40F0EF80E0680528AF
:103A600007D34EF6A460C0F600004FF49B71FFF739
:103A700071FC207C022807D34EF6A460C0F600003B
:103A800040F23711FFF766FC607C022807D34EF640
:103A9000A460C0F600004FF49C71FFF75BFCA07CB3
:103AA000022807D34EF6A460C0F6000040F2391198
:103AB000FFF750FC60690138B0F5007F07D34EF680
:103AC000A460C0F600004FF49D71FFF743FCA069AD
:103AD0000138802807D34EF6A460C0F6000040F2FB
:103AE0003B11FFF737FCE0690138B0F5807F07D361
:103AF0004EF6A460C0F600004FF49E71FFF72AFC5A
:103B0000206A0138802807D34EF6A460C0F6000072
:103B100040F23D11FFF71EFCA068B0F5407F2FD1A9
:103B2000606A0138202807D34EF6A460C0F6000072
:103B30004FF4A071FFF70EFCA06A0138102807D3DC
:103B40004EF6A460C0F6000040F24111FFF702FCFF
:103B5000E06A0138202807D34EF6A460C0F60000C2
:103B60004FF4A171FFF7F6FB206B0138102807D343
:103B70004EF6A460C0F6000040F24311FFF7EAFBE6
:103B8000606B1D2807D34EF6A460C0F6000040F21B
:103B90004511FFF7DFFBA06B092807D34EF6A460A1
:103BA000C0F600004FF4A371FFF7D4FBE06B40F0C8
:103BB0008070B0F1807F07D04EF6A460C0F60000A0
:103BC00040F24711FFF7C6FB94F85C0028B90020CB
:103BD00084F85D00204602F045FF2068816921F0ED
:103BE00010018161FFF73EFD054600BF2068816935
:103BF000090707D5FFF736FD401B0B28F6D312E067
:103C000001207047816941F001018161FFF72AFDC0
:103C1000054600BF20688169C9071BD1FFF722FD57
:103C2000401B0B28F6D3206E032140F001002066D4
:103C3000012084F85C10BDE8F081B0F5407F3FF4CE
:103C40000DAF4EF6A460C0F6000040F23511FFF74C
:103C500081FB03E78169404541F00201816104BFB6
:103C60006168C8F80011217C8269012922F04002B4
:103C700018BF40328261617C8269012922F480424E
:103C800008BF02F580428261A17C8269012922F489
:103C9000805218BF02F5805282618369D4E9021212
:103CA00023F440730B438361836923F0A40383618E
:103CB000036923F0100303619AB1012A0DD0022A8F
:103CC00009D08369032A43F080038361036943F0C9
:103CD0001003036105D1202200E0042283691A4306
:103CE0008261D4E90552D4E90736571E6FF0FF020E
:103CF00002EB032343EA4763771E1F430023CFF6FB
:103D0000FF7303EB05463743B1F5407FC76110D120
:103D1000D4E90917D4E90B65013F02EB06223A43C7
:103D20006FF00F0707EB05173A4303EB014111430F
:103D3000C160D4E90D23E16BD0F8C0704AF250762F
:103D40003943C0F8C01008F5806708F58041B842D3
:103D500004BF4AF25071C4F2000108F50067C4F2D2
:103D60000006B84208BF06F554712164D0F880708F
:103D700027F4F81747EA0242C0F8802001F17002E8
:103D80006264D0F8802022F0706242EA0362C0F8D8
:103D9000802001F1B000A06401F5C470E06401F579
:103DA0001870206501F51E70606501F554700022E1
:103DB00041F8042B8142FBD300200121A06520663D
:083DC00084F85C10BDE8F081FD
:103DC80070B542F210060446C4F20206FFF746FC3C
:103DD800054600BF3068C00306D5FFF73FFC401B0F
:103DE800A042F7D9032070BD30684CF2FA31014087
:103DF80008D041F24C70C1F2000042680A434260A8
:103E0800012005E03068C0074FF0000001D0012113
:043E1800316070BDE8
:103E1C0042F21400C4F20200016841F0004101605A
:083E2C000068C043C00F70479D
:103E3400416842F2200CC4F2020C062204290260FA
:103E440020D803291ED00722042902601AD8DFE8EB
:103E540001F0030B07190F00614651F80C2F0AE01B
:103E6400614651F82C2F06E0614651F8102F02E00C
:103E7400614651F8302F02F07F0282600968C1F375
:103E84000641C160B0B5DCF80010C9B20A46AA29DF
:103E940018BFBB22CC2908BF0A460261DCF8001017
:103EA400C26921F0FF01531E012B816173D801689F
:103EB40047F2E05541F0080101600021C4F201011C
:103EC4000B68C1F6FF75DB05298840F20003C0F6D4
:103ED40004034FF6FF7409D4A1424FF0006E10D0D2
:103EE40029684FF0006361F358230AE0A14205D02A
:103EF40029684FF0006E61F3582E00E09E464FF0A3
:103F04000063DCF8001049020DD4022A1FD0012AF4
:103F14003BD1DCF804104FF0006361F31213036229
:103F2400DCF808301CE0022A1FD0012A2DD1DCF86D
:103F340004104FF6F873C0F2030303EAC10171449D
:103F44000162DCF8081003EAC10171441CE0DCF8EA
:103F540024104FF0006361F312130362DCF828307D
:103F64004FF0006163F312110EE0DCF824104FF6F9
:103F7400F875C0F2030505EAC10119440162DCF8D1
:103F8400281005EAC10119444162DCF8081001F067
:103F940000411143C1610268C16A42F01003036029
:103FA400DCF850304D1E012D03F4803383620ED8AB
:103FB40042F030020129026004D0022907D10CF139
:103FC400540101E00CF150010968C9B20163B0BDAC
:103FD40070B516460C46054679B1022E07D34EF24B
:103FE4003F70C0F6000040F29B11FFF7B1F91820B2
:103FF400002E08BF28202C5070BD4EF23F70C0F632
:1040040000004FF4CD71FFF7A3F9022EE7D2EEE7DB
:104014002DE9F04381B00446006880690840401AE5
:10402400B0FA80F0400982422CD1DDF82080154698
:104034000E461F4603F1010912E000BF20688069A3
:104044003040801BB0FA80F0400985421ED02068C1
:1040540080693040801BB0FA80F04009854211D15C
:1040640020463946424600F089F9D8B9B9F1000F23
:10407400EDD0FFF7F5FA002FE0D0A0EB0800B8422E
:10408400E5D9DBE7002001B0BDE8F083606C40F0C7
:1040940020006064202084F84100002084F842005D
:0C40A40084F84000012001B0BDE8F0836A
:1040B000F0B581B004460068806980071CD41546BD
:1040C0000E464F1C08E000BF20688069800716D5A7
:1040D0002068806980070FD4204631462A4600F0C8
:1040E0004FF9C0B9002FF3D0FFF7BCFA002EEBD088
:1040F000401BB042ECD9E7E7002001B0F0BD606C96
:1041000040F020006064202084F84100002084F802
:0C411000420084F84000012001B0F0BD26
:10411C0070B5044600688069800619D415460E46B1
:10412C0008E000BF20688069800615D5206880698A
:10413C0080060DD4204631462A4600F01BF948B9BA
:10414C00FFF78AFA002EEDD0401BB042EED9E9E71A
:10415C00002070BD012070BD606C40F020006064D8
:10416C00202084F84100002084F8420084F84000AC
:04417C00012070BDF1
:1041800000688169890744BF002181628169C9078C
:0C41900002BF816941F0010181617047AC
:10419C002DE9F04F81B08B46591E89B21E46174649
:1041AC000229044607D34CF27260C0F6000040F6B8
:1041BC00E111FFF7C9F894F8410020280AD10A9DB3
:1041CC0065B1DDF82C80B8F1000F07D094F84000F1
:1041DC0001280AD1022001B0BDE8F08F4FF4007025
:1041EC006064012001B0BDE8F08F012084F840002C
:1041FC00FFF732FA814620464FF400410122192381
:10420C00CDF80090FFF700FF0146012011B101B07D
:10421C00BDE8F08F212084F8410040204FF0000AC7
:10422C00DDF830C084F84200C4F844A0656242F264
:10423C000005C8F20005F2B2204659464FF08073D3
:10424C00A4F82A80C4F834A00095654605F0A8FDB2
:10425C00204629464A46FFF725FFB0B92068012EB3
:10426C0008D0390A8162204629464A46FFF71AFFD0
:10427C0058B92068F9B281622046802100222B4671
:10428C00CDF80090FFF7C0FE10B184F840A0A8E76D
:10429C00608DB0F5807F08D3FF2020850027204655
:1042AC005946FF224FF0807307E0608D0027208570
:1042BC00C2B2204659464FF00073009705F070FDCE
:1042CC000026FF270BE0608D59462085C2B22046A0
:1042DC004FF00073009605F063FD608D70B32046BF
:1042EC0029464A46FFF7DEFE00287FF47AAF606A63
:1042FC00216810F8012B8A626062608D013860853C
:10430C00208D01382085618D0029E6D00004E4D190
:10431C002046802100222B46CDF80090FFF774FE3A
:10432C0000287FF45EAF608DB0F5807FCBD32785FE
:10433C0020465946FF224FF08073CBE72046294692
:10434C004A46FFF7E5FE00287FF44BAF206820219A
:10435C00C16142684EF60003CFF600631A4042601A
:10436C00002084F8411084F8420084F8400001B029
:04437C00BDE8F08F19
:104380002DE9F04381B00446006816468369DA06D9
:1043900002D40026002548E00D461021C1612068A6
:1043A0008169890634D4002705F101094FF000081E
:1043B00008E048F0200801272068816901F0200109
:1043C000394328D1B9F1000FF6D0FFF74BF915B1F9
:1043D000801BA842F0D92068426894F84210836993
:1043E0001B040BD512F4804208D1202906D0416865
:1043F00041F480414160FFF735F906462068806945
:104400008006D9D4FFF72EF9801B1A28F6D3D0E7FF
:104410000121042604E0B7FA87F1490948F00406AF
:10442000012500291CBF2021C16120688169CA05BE
:104430001ED44A0524D489052AD4ADB12046FFF7FD
:104440009FFE20684EF600024168CFF600621140E0
:104450004160606C30436064202084F8410000209B
:1044600084F8420084F84000284601B0BDE8F0839B
:1044700046F001064FF480720125C2614A05DAD583
:1044800046F008064FF480620125C2618905D4D543
:1044900046F002064FF400710125C161CED1E3E779
:1044A00010B582B004460020CAF6AA2004EA000132
:1044B000814218BF14F47F0007D14EF2EE10C0F60F
:1044C000000040F23D11FEF745FF41F26000C4F2EA
:1044D0000200016841F001010160006800F0010084
:1044E000019001980420C4F2010001682143016099
:0444F00002B010BD49
:0C44F40001684AF6AA2200200A60704706
:10450000002859D070B50646006845F60041C4F24F
:104510000001884206D04CF6C200C0F60000872198
:10452000FEF718FF96F8910228B9002086F890024D
:10453000304602F09FFE032086F89102306801F0B9
:10454000C1F93079A8B100EB8001C90000224FF019
:10455000010C0023002400BFF51828332C74994265
:1045600004F1010485F811C0EA74C5E90822AA62C1
:10457000F2D180B106F5B4710022002301F8183C95
:10458000013301F8172C01F8152C41E9022241F8FA
:10459000282B9842F2D196E8070007F0AFFC0020E4
:1045A0000121307386F89112B17A012903D1304686
:0C45B00005F07AFE002070BD012070476D
:1045BC0041F20C01C4F2020151F8040C42F2004227
:1045CC00C0F2F40200F00C00042810462DD051F873
:1045DC00040C00F00C00082847F64000C0F27D10D7
:1045EC0023D051F8043C03F00C030C2B1ED180B5E6
:1045FC00D1F800C00B680CF0030CC3F3031E0B685E
:10460C000EF1010EBCF1030F08BF02460968B2FBA4
:10461C00FEF0C3F30623C1F341610222584302EBBF
:10462C004101B0FBF1F0BDE88040704700207047BD
:10463C002DE9F04381B004460068000306D14EF624
:10464C001330C0F600008321FEF77EFEA07841F205
:10465C0088090007C4F2020901D4002575E0206D19
:10466C004FEA3020042806D34EF61330C0F6000073
:10467C008B21FEF769FE59F8300C5FEAC0080BD4A9
:10468C0059F8300C40F0805049F8300C59F8300C87
:10469C0000F080500090009847F20007C4F2000729
:1046AC00386840F480703860FEF7D6FF054600BFCE
:1046BC003868C60508D4FEF7CFFF401B0328F7D394
:1046CC000325002E03D437E00025002E34D5D9F86D
:1046DC00080010F4407025D0216D884222D0D9F802
:1046EC000800D9F8081020F4407241F48031C9F860
:1046FC000810D9F80810C00721F48031C9F8081047
:10470C00C9F808200ED0FEF7A7FF064641F28937FC
:10471C00D9F80800800705D4FEF79EFF801BB8422D
:10472C00F6D3032545B9D9F80800216D20F4407063
:10473C0008430025C9F80800B8F1000F5EBF59F80E
:10474C00300C20F0805049F8300C2078C00711D084
:10475C006068042806D34EF61330C0F60000E02142
:10476C00FEF7F2FDD9F80000616820F00300084361
:10477C00C9F800002078800713D5A0684FEAB00074
:10478C00042806D34EF61330C0F60000EA21FEF7DB
:10479C00DBFDD9F80000A16820F00C000843C9F833
:1047AC0000002078400713D5E0684FEA3010042849
:1047BC0006D34EF61330C0F60000F621FEF7C4FD0A
:1047CC00D9F80000E16820F030000843C9F8000077
:1047DC002078000714D520694FEAB010042807D3BD
:1047EC004EF61330C0F6000040F20311FEF7ACFD9C
:1047FC00D9F80000216920F0C0000843C9F8000076
:10480C002078C00614D560694FEA3020042807D3FD
:10481C004EF61330C0F600004FF48871FEF794FD8D
:10482C00D9F80000616920F440700843C9F8000011
:10483C002078800614D5A0694FEAB020042807D34D
:10484C004EF61330C0F600004FF48E71FEF77CFD6F
:10485C00D9F80000A16920F440600843C9F80000B1
:10486C00207840060ED5E069002818BFB0F5805FAF
:10487C0040F04D81D9F80000E16920F44050084324
:10488C00C9F80000207800060ED5206A002818BF51
:10489C00B0F5804F40F04881D9F80000216A20F42F
:1048AC0040400843C9F800006078C0070ED0606A29
:1048BC00002818BFB0F5803F40F04381D9F80000C4
:1048CC00616A20F440300843C9F80000A0788007E2
:1048DC0012D5A06A032807D34EF61330C0F6000099
:1048EC004FF4A471FEF730FDD9F81400A16A20F042
:1048FC0003000843C9F814006078800714D5E06AF7
:10490C004FEAB040042807D34EF61330C0F600002F
:10491C004FF4AA71FEF718FDD9F80000E16A20F4F3
:10492C0040200843C9F80000607840071DD5206B73
:10493C004FEA3050042807D34EF61330C0F600006F
:10494C0040F25F11FEF700FDD9F80000216B20F456
:10495C0040100843C9F80000B1F5801F02BF59F898
:10496C007C0C40F4801049F87C0C607800071DD555
:10497C00606B4FEAB050042807D34EF61330C0F6E4
:10498C0000004FF4B971FEF7DFFCD9F80000616B41
:10499C0020F440000843C9F80000B1F5800F02BFB5
:1049AC0059F87C0C40F4801049F87C0C6078C006F7
:1049BC0017D5A06B002818BFB0F1807F40F0CE80D7
:1049CC00D9F80000A16B20F040700843C9F8000032
:1049DC00B1F1807F02BF59F87C0C40F4801049F88B
:1049EC007C0C607880061ED5E06B40F00060B0F166
:1049FC00006F07D04EF61330C0F6000040F297114E
:104A0C00FEF7A2FCD9F80000E16B20F040600843EF
:104A1C00C9F80000B1F1006F02BF59F87C0C40F4EA
:104A2C00801049F87C0C607840061ED5206C40F054
:104A3C000060B0F1006F07D04EF61330C0F60000E6
:104A4C004FF4D371FEF780FCD9F80000216C20F0F4
:104A5C0040600843C9F80000B1F1006F02BF59F87B
:104A6C007C0C40F4801049F87C0C6078000616D55C
:104A7C00606C002818BFB0F1805F7CD1D9F80000C1
:104A8C00616C20F040500843C9F80000B1F1805F20
:104A9C0002BF59F87C0C40F4803049F87C0CA078AB
:104AAC00C00716D0A06CB0F1004F18BF00286FD112
:104ABC00D9F80000A16C20F040400843C9F8000070
:104ACC00B1F1804F02BF59F87C0C40F4803049F8AA
:104ADC007C0CA078400716D5E06C002818BFB0F508
:104AEC00801F61D1D9F81400E16C20F44010084308
:104AFC00C9F81400B1F5001F02BF59F87C0C40F442
:104B0C00801049F87C0C284601B0BDE8F083B0F564
:104B1C00005F3FF4AFAE4EF61330C0F600004FF41A
:104B2C009371FEF711FCA5E6B0F5004F3FF4B4AE5F
:104B3C004EF61330C0F600004FF49871FEF704FCEB
:104B4C00AAE6B0F5003F3FF4B9AE4EF61330C0F60E
:104B5C00000040F23B11FEF7F7FBAFE6B0F1007F2F
:104B6C003FF42EAF4EF61330C0F6000040F2851124
:104B7C00FEF7EAFB24E7B0F1005F3FF47FAF4EF69F
:104B8C001330C0F600004FF4DA71FEF7DDFB75E769
:104B9C00B0F1804F8CD04EF61330C0F6000040F2CE
:104BAC00C511FEF7D1FB83E7B0F5001F9AD04EF686
:104BBC001330C0F600004FF4EC71FEF7C5FB91E723
:104BCC0070B504460068C16849061CD4C16841F040
:104BDC008001C160FEF740FD2168C968490612D406
:104BEC0005460026FEF738FD401BB0F57A7F84BFE2
:104BFC00032684F825602068C068400601D4032E83
:0C4C0C00F0D1F0B270BD0026F0B270BD17
:104C1800B0B5044600685F21C0F20101C160FEF72B
:104C28001DFD05462068C068800607D4FEF716FDFE
:104C3800401BB0F57A7FF5D90320B0BD0020B0BD88
:104C4800B0B50C462029154607D34EF67430C0F689
:104C5800000040F2E471FEF779FB42F20050C4F222
:084C6800000040F82450B0BD2B
:104C70002DE9F04381B0044680681E4615460F4674
:104C800038B14CF64620C0F600004FF49F61FEF7A5
:104C900061FBFEF7E7FC94F85D108146012908D11D
:104CA000002F4FF0010018BF002D0ED101B0BDE85C
:104CB000F0836068B0F5827F0DD104294FF00200C7
:104CC000F4D1A1680029EBD0F0E7002EEED094F8E3
:104CD0005C00012803D1022001B0BDE8F08301206F
:104CE00084F85C0094F85D00DDF8208004281CBF87
:104CF000052084F85D00002020662564A4F8466045
:104D0000A4F84460A763E687C4E913002068A68777
:104D1000E1684268B1F5E06F22F48052134698BF13
:104D200003F58053012E88BF134643600268731E4B
:104D300052065EBF026842F0400202606268B3FA47
:104D400083F3B2FA82F252095B09B1F5E06F43EAEC
:104D500002013DD931B137F8021BC160A763E08F72
:104D60000138E087012608F1010500BFE08F20B976
:104D7000B4F84600002800F0A38020688168890705
:104D80000CD5E18F51B1012E08D1A16B002631F86D
:104D9000022BC260A163E18F0139E1878168C907F5
:104DA0000DD0B4F8461051B1C068216C012621F82D
:104DB000020B2164B4F846000138A4F84600FEF75F
:104DC00051FC002DD2D0A0EB09004045CED36DE0C0
:104DD00000294FF6FE7111D0E28F022A05D337F871
:104DE000022BC2604FF6FE7004E03A780273A06BAB
:104DF000471C481CA763E28F1044E087012708F195
:104E000001054E1CE08F18B9B4F84600002857D0B1
:104E100020688168890717D5E18FA9B1012F13D1C7
:104E2000E28FA16B022A05D331F8022BC2604FF644
:104E3000FE7004E009780173A06B411C3046A16349
:104E4000E18F00270844E08720688168C90725D0E2
:104E5000B4F8461011B3B4F84610022912D3C16851
:104E6000226C22F8021B2264B4F846100239A4F81E
:104E70004610B4F8461001290FD8416841F480511A
:104E800041600AE0007B216C0870206C01302064D6
:104E9000B4F846000138A4F846000127FEF7E2FB0B
:104EA000002DAFD0A0EB09004045ABD3012084F822
:104EB0005D00002084F85C00032001B0BDE8F083B1
:104EC000204641464A4606F077F940B12020206648
:104ED000002084F85C00012001B0BDE8F0830120CF
:104EE00084F85D00002084F85C00206E002818BF64
:084EF000012001B0BDE8F083D0
:104EF8002DE9F04F83B04FF000091E4690460D464D
:104F080083468DF80790FEF7A9FB301A00EB0807D7
:104F1800FEF7A4FB41F28071C1F200010968232267
:104F28005143090DDBF800A079430291DAF8081023
:104F380029424DD0064608F1010404E0DBF80000E0
:104F48008068284217D0B5F5C06F02BF9AF80C00E8
:104F58008DF807009DF80700002CEFD0FEF77EFBC8
:104F6800801BB8420AD202980299002808BF074657
:104F7800481E0290E2E74FF0000929E0DBE9000152
:104F88004268B1F5827F22F0E00242600BD1DBF883
:104F98000810B1F5004F02D0B1F5806F03D1016858
:104FA80021F040010160DBF82810B1F5005F07D15E
:104FB800016821F400510160016841F40051016069
:104FC80001208BF85D0000208BF85C004FF003098E
:084FD800484603B0BDE8F08F6C
:104FE000F0B581B015460E460446FEF73BFB281A85
:104FF0008719FEF737FB41F28071C1F200010968A1
:10500000C1F3CB317943009121688968090602D444
:10501000002001B0F0BD0546013603E0206880683D
:105020000006F5D5002EF9D0FEF71CFB401BB84258
:1050300007D200980099002808BF0746481E009034
:10504000ECE7D4E900014268B1F5827F22F0E0028A
:1050500042600AD1A168B1F5004F02D0B1F5806F6E
:1050600003D1016821F040010160A16AB1F5005F40
:1050700007D1016821F400510160016841F4005139
:105080000160012084F85D00002084F85C000320AA
:0450900001B0F0BDBE
:10509400F0B581B00446406841F63121C0F21E11DA
:1050A400884207D34EF2FD70C0F6000040F6DD31B1
:1050B400FEF74EF9A068002818BFB0F5805F40F0F5
:1050C400C68048F200072168C4F20007E068B942CC
:1050D40014D04FEA3030042807D34EF2FD70C0F6E6
:1050E400000040F6E531FEF733F9206A40F4006031
:1050F400B0F5006F0FD040F6E63106E040F4005002
:10510400B0F5005F07D040F6E1314EF2FD70C0F615
:105114000000FEF71DF92069002818BFB0F5806F64
:1051240040F0A280606910B130F00C0007D04EF25C
:10513400FD70C0F6000040F6EA31FEF709F9A069F7
:105144004FEA3020042807D34EF2FD70C0F6000069
:1051540040F6EB31FEF7FCF8E06940F40040B0F5AE
:10516400004F07D04EF2FD70C0F6000040F6EC315F
:10517400FEF7EEF8606A0C2807D34EF2FD70C0F615
:10518400000040F6ED31FEF7E3F804F108014EC9E2
:105194002068194341EA0603E169066846F6F315F7
:1051A400CCF6FF752E4033430B4303604368B8428B
:1051B40023F4405342EA03024260A2691CBF236AFB
:1051C4001A43836823F06E4323F430631A438260E6
:1051D400C26A636A22F00F021A43C26244F6FF7283
:1051E400C4F2000290424FF0100218DC44F2004373
:1051F400C4F20003984244D044F60003C4F200030E
:1052040098424CD044F60043C4F2000398425BD168
:1052140041F28802C4F20202126892094CE045F29B
:105224000003C4F20003984232D0B8423ED043F6A1
:105234000003C4F20103984246D141F28802C4F249
:105244000202126845F29C63C0F6000338E0B0F134
:10525400805F3FF436AF4EF2FD70C0F6000040F6BA
:10526400DE31FEF775F82CE7B0F5C06F3FF45AAFA6
:105274004EF2FD70C0F6000040F6E931FEF768F822
:1052840050E741F28802C4F202021268920813E065
:1052940041F28802C4F202021268120A0CE041F2DE
:1052A4008802C4F202021268120905E041F288027F
:1052B400C4F202021268920A45F2AC63C0F600031B
:1052C40002F0030253F82220B84242F20040C0F236
:1052D400F40013D0B1F5004F1ED1082A00F2648007
:1052E4000026DFE802F00569736171616161B50050
:1052F40005F0F4FC002840F06A809DE0082A4ED8AE
:105304000026DFE802F0054C1E4C184C4C4C1C00E7
:1053140005F0E4FCB8B98FE0082A49D80026DFE894
:1053240002F0054F7447724747479C0005F0D6FCCE
:1053340000286BD180E0FFF73FF920B97CE04FF4FF
:105344000040002878D0616A4EF2B022C0F6000214
:1053540032F811206568B0FBF2F305EB45018B428E
:105364004FF001016BD32F03BB4268D80021002307
:1053740008F07CFB090241EA1061000210EB5500C1
:1053840041F100012A46002308F070FB4FF6005259
:10539400A0F54071C0F20F0291424BD34EE00020C1
:1053A40001260028CFD147E00020012678B943E048
:1053B4000020012650BB3FE005F0A6FC38B93BE0D5
:1053C40005F0A2FC10BB37E0FFF7F6F8A0B3616A62
:1053D4004EF2B022C0F6000232F811106268B0FB3F
:1053E400F1F0510801EB4000B0FBF2F04FF6EF7220
:1053F400A0F11001914221D84FF6F0710140C0F3A1
:105404004200084416E0FFF7D7F8A8B1616A4EF2EB
:10541400B022C0F6000232F811106268B0FBF1F05D
:1054240000EB5200B0FBF2F04FF6EF72A0F1100166
:10543400914203D82168C860314600E001214FF051
:1054440001100022A06662670846A26701B0F0BDA1
:105454004FF400400028BAD1EEE74FF40040002892
:04546400D4D1E9E7CF
:105468002DE9F04704460068C0690840401AB0FAC0
:1054780080F04009824237D1DDF82080A1F1400058
:1054880015460E46994630F0400A08F1010718BF44
:105498004FF0010A09E000BF2068C0693040801B56
:1054A800B0FA80F0400985421ED1002FF4D0FEF7F3
:1054B800D5F80146B8F1000F4FF0030015D0A1EB65
:1054C8000901414511D8206801680AEA91010129BA
:1054D800E2D1C16909070AD4C1690905DCD50325E8
:1054E80020264FF4006105E00020BDE8F087012583
:1054F800082108260162204606F026F90020C4F893
:0C550800906084F884002846BDE8F0871D
:10551400D0F88C30202B07D100294FF0010318BF9D
:10552400002A04D118467047022318467047002306
:10553400C366D0F800C048F20003C4F200039C45DF
:1055440012D080B5DCF804301B020BD5036853E895
:10555400003FD0F800C043F080634CE8003EBEF149
:0C556400000FF3D1BDE8804000F000B85B
:10557000B0B513460A46816500210446A0F85C30A8
:10558000C0F890102220C4F88C00D4F88000E8B154
:105590004BF2DD65C0F60005456325684BF6C54C4A
:1055A0004BF6555EC0F6000CC0F6000E816305F1A7
:1055B0002401C0E90BCE03F015FD38B11020C4F86A
:1055C00090002020C4F88C000120B0BD206948B1B3
:1055D000206850E8000F216840F4807041E8000224
:1055E000002AF5D12068083050E8000F216840F00B
:1055F0000100083141E80002002AF3D12068083098
:1056000050E8000F216840F04000083141E80002F6
:08561000002AF3D10020B0BD17
:10561800016851E8001F026821F0C00142E8001348
:10562800002BF5D10168083151E8001F026821F408
:105638000001083242E80013002BF3D12021C0F802
:04564800881070470F
:0C564C00806A0021A0F85E1000F0E8BCAD
:10565800016848F20002C4F20002914209D0D0F871
:105668008820202A03D190F88420012A03D102201F
:105678007047012070472422C0F888204A6842F405
:1056880000024A602021C0F88810002180F88410A8
:045698000020704737
:10569C0001000000040000000200000008000000EF
:1056AC0000000000040000000200000008000000E0
:1056BC00416E19B380B501684EF6047C8A6889681E
:1056CC00C0F6000C490F4EF60C7E1CF80130C0F6EB
:1056DC00000E1EF80110DB00B3FBF1F1C2F34262C5
:1056EC00A0F86A101CF802101EF80220C900B1FBC9
:1056FC00F2F1BDE88040A0F8681070470121A0F8D5
:08570C006A10A0F86810704754
:10571400B0B50446006844F6FF72C4F20002904239
:1057240012DC44F20042C4F20002904228D044F653
:105734000002C4F20002904222D044F60042C4F2B5
:10574400000290421CD011E045F20002C4F20002B3
:10575400904215D048F20002C4F2000290420FD0E9
:1057640043F60002C4F20102904209D04CF6DA205A
:10577400C0F600000D464FF41971FDF7E9FD294606
:1057840081F000404FEA7070072828D8012202FAFD
:1057940000F010F0F30F22D094F88400012801D116
:1057A4000220B0BD012084F884002420C4F88800BD
:1057B40020680568026822F001020260826822F013
:1057C4006042114381602046FFF776FF2068056040
:1057D4002020C4F88800002084F88400B0BD4CF672
:1057E400DA20C0F600000D4640F26521FDF7B0FD59
:0457F4002946D1E78A
:1057F80070B50446006844F6FF72C4F20002904295
:105808000D4612DC44F20041C4F20001884226D061
:1058180044F60001C4F20001884220D044F6004159
:10582800C4F2000188421AD011E045F20001C4F226
:105838000001884213D048F20001C4F200018842F6
:105848000DD043F60001C4F20101884207D04CF69E
:10585800DA20C0F6000040F29521FDF777FD4FEA07
:105868007560062807D34CF6DA20C0F6000040F22F
:105878009621FDF76BFD94F88400012801D10220E0
:1058880070BD012084F884002420C4F888002068B2
:105898000668016821F001010160816821F06061FA
:1058A800294381602046FFF705FF20680660202015
:0C58B800C4F88800002084F8840070BD53
:1058C4000146B0F8400044F27F0202400020A1F8F3
:0458D40040207047B9
:1058D80040F20000C1F20000B0F8CC104FF47A7327
:1058E800A0F88C10B0F98C10B0F97E20891A41F21A
:1058F800E422C1F2000212685A4392FBF1F200213D
:08590800C0F8902006F0E0BE9B
:105910002DE9F04F89B040F60004C4F6000420469B
:1059200001210122FEF756FB9620FDF7A1FE41F270
:105930009025C1F200052846FEF7DCFD2046022135
:105940000022FEF747FB9620FDF792FE2846FEF761
:10595000D1FD204602210122FEF73CFB9620FDF7F7
:1059600087FE2846FEF7C6FD204601210022FEF7ED
:1059700031FB40F6D05440F64620C1F2000406AD9B
:1059800006904FF47A76204629462A46022300964E
:10599000FFF76EF926208DF81800204629462A4682
:1059A00003230096FFF764F99DF81A000A2864D1D2
:1059B0009620FDF75DFE41F29020C1F20000FEF757
:1059C00099FD40F6D054C1F200042046202106F093
:1059D000AFFA06AD2327204629462A4603238DF831
:1059E00018700096FFF744F99DF81A004FF043082D
:1059F00000F0EF008DF81900204629462A460223C0
:105A00008DF818800096FFF733F9204629462A467C
:105A100003238DF818700096FFF72AF906AD20468B
:105A200029462A4603238DF818700096FFF720F9BF
:105A30009DF81A00294600F09F0020308DF81900CB
:105A400020462A4602238DF818800096FFF710F9A9
:105A5000204629462A4603238DF818700096FFF742
:105A600007F99DF81A0080060FD44EF60D10C0F607
:105A7000000005F09CFE00BFFEE74EF64470C0F645
:105A8000000005F094FE00BFFEE743F2514040F6EF
:105A9000D054ADF818000020C1F2000406AD8DF816
:105AA0001A004FF47A78204629462A460223CDF878
:105AB0000080FFF7DDF831208DF8180020462946D8
:105AC0002A460323CDF80080FFF7D2F89DF81A008C
:105AD000342805D04CF6BA70C0F6000005F067FE19
:105AE00040F6D059002704244EF6254AC1F2000999
:105AF00006AD04AE4FF0000B06E000BF002010BB67
:105B0000002CA4F101041ED0484629463246032346
:105B1000CDF818A08DF81270ADF81070CDF8008097
:105B2000FFF7A6F89DF81000FF28E7D19DF81100B7
:105B30009DF818108842E1D19DF812004FF0010B3A
:105B400003900120DCD0BBF1000F4DD0039840F64C
:105B5000D05540F060074FF0000804244FF045098D
:105B60004FF47A7AC1F2000506AE0DF1100B002059
:105B7000039000BF284631465A4602238DF81890FC
:105B80008DF81970ADF81080CDF800A0FFF770F80F
:105B90009DF81000FF2809D19DF811009DF81810FC
:105BA000884203D101210120039100E0002018B9AF
:105BB000002CA4F10104DDD10398F8B10BF104002D
:105BC00041F26C2A40F6D0590190002505264EF688
:105BD0002544C1F2000A06AF4FF47A78C1F20009F9
:105BE0000020039016E000BF4FF09040202103F00A
:105BF000EBFFC820FDF73CFDF6E700BF4FF09040FB
:105C0000202103F0E1FFFA20FDF732FDF6E700BFA7
:105C1000013E4AD0504639460222CDE9064502F0FF
:105C2000DDFF8DF81A00484639465A460623ADF87E
:105C300014500495CDF80080FFF71AF89DF8100075
:105C4000FF282DD19DF811009DF81810884227D10A
:105C50009DF812009DF81910884221D19DF813007B
:105C60009DF81A1088421BD19DF8150001990290E9
:105C70005046012202F0B2FF0299884210D19DF8ED
:105C8000140000F060006028039808BF0120039012
:105C90004FF0000008BF0C200E2804D1B8E700BF69
:105CA0000E200E28B4D00028B2D00398002863D06C
:105CB00041F29020C1F20000FEF71CFC41F26C2A78
:105CC00040F6D0574FF0000804244EF6F249C1F2D6
:105CD000000A06AE4FF47A75C1F200070DF1100B01
:105CE00000200390504631460222CDF8189002F071
:105CF00075FF8DF81A00384631465A460423CDF810
:105D000010800095FEF7B4FF9DF81000FF2815D114
:105D10009DF811009DF8181088420FD19DF81200CF
:105D20009DF81910884209D19DF813009DF81A10AA
:105D3000884203D101210120039100E0002018B91D
:105D4000002CA4F10104CDD10398F8B10BF10400AB
:105D500041F26C2A40F6D0590190002505264EF6F6
:105D60002144C1F2000A06AF4FF47A78C1F200096B
:105D70000020039016E000BF4FF09040202103F078
:105D800023FF4FF49670FDF773FCF5E74FF090405A
:105D9000202103F019FF4FF4AF70FDF769FCF5E720
:105DA000013E4AD0504639460222CDE9064502F06E
:105DB00015FF8DF81A00484639465A460623ADF8B5
:105DC00014500495CDF80080FEF752FF9DF81000A6
:105DD000FF282DD19DF811009DF81810884227D179
:105DE0009DF812009DF81910884221D19DF81300EA
:105DF0009DF81A1088421BD19DF815000199029058
:105E00005046012202F0EAFE0299884210D19DF923
:105E100014000121B0F1FF3F4FF00700C8BF002080
:105E2000039AD8BF0A460392092804D1B8E700BFF5
:105E300009200928B4D00028B2D00398A0B141F2BB
:105E40009024C1F200042046FEF754FB9620FDF793
:105E50000FFC2046FEF74EFB00F010F82046FEF740
:105E600049FB09B0BDE8F08F4FF09040202103F0CE
:0C5E7000ABFE4FF4C870FDF7FBFBF5E73C
:105E7C0040F60000C4F6000001210122FEF7A4B890
:045E8C00FAF78CBED7
:105E900040F20000C1F20000D0F84011D0F84021DB
:0C5EA000002948BF5242C0F80C21704796
:105EAC0040F20001C1F20001D1F84001B0F1FF3F16
:105EBC00DABFD1F8400140420020D1F80C21002A71
:105ECC0003DDD1F80C21D31701E0CA6D002310B506
:105EDC0048F29F64C0F20104611C80FB010107F0D1
:105EEC008BFD48F2A062C0F20102121A201A4FF088
:105EFC0000008841B8BF0022002944BF48F2A062CC
:085F0C00C0F20102104610BDB5
:105F140010B582B040F20004C1F20004B4F85A0093
:105F2400A4F88001B4F9CC00B4F96A10884219DAF3
:105F3400B4F8CCC0B4F9CC00B4F96C108842D8BF22
:105F4400B4F86CC0B4F96C00B4F96E10B4F96A20FA
:105F5400B4F95A300FFA8CFCCDF800C006F09CF866
:085F6400A4F8800102B010BD99
:105F6C0010B582B00DF1070200200021012300F0D2
:105F7C0019F89DF80700411CC8B202280ED846F249
:105F8C001C02C0F6000252F82000C900C9B24FF43E
:105F9C00813222FA01F405F004FC00E00324E0B2A3
:045FAC0002B010BD72
:105FB0002DE9F04F83B0924606465818012241F26F
:105FC000F0181D4602EB901700204FF47A79C1F2C9
:105FD000000800BF8BB213FA85F32C4641EA861203
:105FE000402B28BFC1F140041FFA80FB1AFA80F051
:105FF000A1B2CDE9000192B24046A0210223CDF822
:10600000089003F049FF01362D1B1BFA84F0013F75
:0C6010004FF00001DED103B0BDE8F08FBE
:0C601C008AD00008AEE900084BEC000838
:1060280010B5044640F20000C2F2000001210175DB
:10603800002180F83112D4F88010B4F85C20096887
:106048004968511AC0F82812D4F89000D4F8900082
:10605800042805D14EF6CC70C0F6000008F0F0F91F
:10606800D4F89000012805D14EF6DC70C0F6000087
:1060780008F0E6F9D4F89000022805D14EF6EC7045
:10608800C0F6000008F0DCF9D4F89000102805D11B
:106098004EF6A240C0F6000008F0D2F9D4F89000FD
:1060A800102805D14EF6A240C0F6000008F0C8F945
:1060B800D4F89000082805D14EF6B340C0F6000089
:1060C80008F0BEF9A16D20464FF48072FFF71EFA62
:1060D80038B14EF61420C0F60000BDE8104008F0B4
:0460E800AFB910BD7F
:1060EC0040F20000C2F20000002180F82610704738
:1060FC0003460068B3F82C224FF00C0C03F2271166
:08610C0083F826C005F060BA1B
:106114004FF6FF72C1B1B0B54FF0000C4AF2010E58
:1061240010F80C305A406FF0070300BF8EEA520497
:10613400D50708BF540801332246F7D30CF1010CEC
:0C6144008C45EDD1BDE8B04090B2704732
:1061500070B58E1E0C4631460546FFF7DBFFA95B86
:0C616000814218BF4FF0FF34204670BD94
:04616C00007D7047FB
:1061700070B540F2000CC1F2000C002BBCF81840C6
:1061800018BFA3420AD18B7891F803E04EEA0324AA
:10619000B4F5FE7F08D340F2862101E040F6863157
:1061A00081520220104470BD0D790CEB44067570CD
:1061B0004D7986180CF8145006258554737086F8AE
:1061C00002E00879F070487930710520104470BD04
:1061D0002DE9F04140F20006C1F20006002B378B9A
:1061E00018BFBB420CD10F7991F8058048EA072708
:1061F000A7F17C0515F17C0F05D84FF4647110E010
:1062000040F686310DE091F802C091F803E04EEAC5
:106210000C243D19A5F2FD1313F5FE7F06D24FF4B1
:106220002471815202201044BDE8F0818FB14FEA01
:106230004C2343EA4E03334408315E1C11F8013C01
:10624000013406F8023B11F8023BAC4206F8033C6D
:10625000F4D31023811883540020C8700520104403
:1062600081F801C081F802E081F80480BDE8F08186
:1062700040F20000C1F20000016E4FF2F012CFF6C2
:0C628000FF725143CA17C0E95A12704760
:10628C0010B540F20004C1F20004D4F80C0100284F
:10629C004FF6FF700ED4D4F80C11E26D91420CD273
:1062AC00E26D3AB14FF47A70E26DA1FB000100236C
:1062BC0007F0D8FBA4F8140110BD4FF47A70A4F8C1
:0462CC00140110BDEC
:1062D00040F20000C1F20000026E8AB180B5D0E940
:1062E0005C0148F2A06CC0F2010CA0FB0C034FF45F
:1062F000616E01FB0C31A2FB0E2307F083FB80BD16
:0463000000207047C2
:1063040040F20001C1F20001D1F84801B0F1FF3FB1
:10631400DABFD1F8480140420020D1F81021002A08
:1063240003DDD1F81021D31701E00A6E002310B564
:1063340048F29F64C0F20104611C80FB010107F074
:106344005FFB48F2A062C0F20102121A201A4FF059
:1063540000008841B8BF0022002944BF48F2A0626F
:08636400C0F20102104610BD59
:10636C0040F20000C1F20000D0F81011002907DD46
:10637C00D0F80C11D0F8402111444FEAE17C05E033
:10638C00C16DD0F840214FF0000C114470B5D0F81D
:10639C00D830B0F88061D0F81051012D03DBD0F863
:1063AC001041E51701E0046E0025981900EBD0733D
:1063BC005E10A1FB0602DB1701FB03214FF47A727E
:1063CC000CFB0611002307F017FB48F2A066C0F285
:1063DC000106A0FB060201FB062122462B4607F014
:1063EC000BFB20EAE070B042B8BF0646304670BDE9
:1063FC00034C206804348047FBE7F9F7E7FEFEE71F
:04640C0048F100084B
:1064100007F004F84EF60850CEF20000054901607E
:106420004EF68850CEF20000016851F47001016010
:08643000FFF7E4FF0000000883
:0864380083F0004307F05EB899
:10644000F0B540F2FF7681EA030C16EA115E1EBF3A
:10645000B64516EA1355B54252D021EA465141F4E9
:106460008011A1FB024723EA465343F48013AE4454
:10647000A0FB03650CF0004C36197D41A1FB0347DE
:1064800047F10003A0FB0217F619654153F1000321
:10649000094218BF46F0010640F2FE74B3F5007FD2
:1064A00013D2AEF5806EA64523D24CEA0331280301
:1064B00041EA155140EA16503203450872F1004294
:1064C00050F1000051EB0E51F0BDAEF2FF3EA6457B
:1064D0000FD24CEAC321E80241EA555140EA565036
:1064E000F202450872F1004250F1000051EB0E51EA
:1064F000F0BD1EEA0E0F2DD50CF000410020F0BDBE
:1065000016EA115F04BF01F000410020004218BFED
:1065100041F0010116EA135F04BF03F000430022BB
:10652000124218BF43F0010306EA1354B44218BFE5
:10653000B64503D00CF000410020F0BD21F0004131
:1065400023F00043B1EB065F0CD8B3EB065F09D82C
:1065500041B13BB10CF0004141F0FE4141F470010A
:106560000020F0BD40F20001C7F6F8710020F0BD38
:106570004FF4001C1CEB410F98BF1CEB430F11D8CC
:1065800051EA030C50EA4C0C5CEA020C0AD004D22B
:1065900082428B4180414042704790429941804104
:0865A0004042704700207047E3
:1065A8004FF4001C1CEB410F98BF1CEB430F11D894
:1065B80051EA030C50EA4C0C5CEA020C0AD004D2F3
:1065C8009042994180414042704782428B418041CC
:0865D8004042704700207047AB
:1065E000C1F30A5240F21E439A1A15DA203225DD11
:1065F000CB17C90241EA5051C00241F00041D141DC
:10660000D04048409140D14048405B1C18BF704783
:10661000404263EB01017047CB17C90241EA505178
:10662000C00241F00041202A28BF202231FA02F0A6
:10663000190008BF70474042894170474B00004233
:1066400018BF43F0010313F5001F88BF21F000417C
:10665000002011F000415CBF6FF00041C043704763
:106660000B0D40F21E42D21A09DBCB0243EA505016
:1066700040F00040202A28BF2022D0407047490027
:04668000804170479E
:1066840050B140F21D42B0FA80F1521A8840C30A58
:0C669400400503EB025170470100704705
:0866A000004870477C17001050
:1066A8005AB3844690EA01039B071FD1830707D09A
:1066B80011F8013B00F8013B521EF7D11CE084465B
:1066C800203A09D32DE9F007B1E8F807A0E8F80760
:1066D800203AF9D2BDE8F0071C3205D451F8043B42
:1066E80040F8043B121FF9D2043205D011F8013BDF
:0C66F80000F8013B521EF9D160467047CB
:1067040000220B0011001A0084465AB3830704D0F8
:1067140000F8011B521EF9D124E0C9B241EA01215B
:1067240041EA0141202A11D3203A2DE9F0030B4616
:106734000C460D460E460F4688468946A0E8FA03E5
:10674400203AFBD2BDE8F00320320BD0042A05D353
:1067540040F8041B121F05D0042AF9D200F8011BCB
:08676400521EFBD16046704794
:10676C0000B50549FFF796FF4158044A002908BFB8
:10677C008118084600BD00BF080000000C00000096
:0C678C00C6B60008B8670008986700084F
:1067980029E6000849E6000855E6000861E6000811
:1067A80081E600088DE60008EFBE000817BE000865
:1067B800FAD400083AD700083AD700083AD70008B0
:1067C8003AD700083AD700083AD700083AD700085D
:1067D8003AD700083AD70008FFFFFFFFFFFFFFFF87
:1067E800FFFFFFFFFFFF00002ED400089AED00080E
:1067F800A6EA0008B7ED0008FDEA000888ED0008E1
:0868080091ED000804EB00080B
:10681000B0B588B040F6204040F200510024C1F2EB
:106820000000C5F20001C0E900144FF48071042596
:10683000818301211C2200F1440CCDE90644CDE9FD
:106840000444CDE90244CDE90044C0E90244C0E972
:1068500004448561016280F82440C0E90B4480F85B
:106860003810C46380F8401080238CE81C00016558
:1068700000F052FD002818BF00F032FA1020C1F2DB
:10688000C000009006200190072002900020C4F272
:106890007F00CDE9030540F62040C1F200006946C3
:1068A000059401F0FBF8002818BF00F019FA08B0B1
:0268B000B0BD79
:0268B200FEE7FF
:1068B400B0B588B040F6B43040F200610024C1F2B3
:1068C4000000C5F20001C0E900144FF480710122F8
:1068D4000823818304251C2100F1440CCDE90644DE
:1068E400CDE90444CDE90244CDE90044C0E90244C1
:1068F400C0E904428361056280F82440C0E90B4486
:1069040080F83820C46380F8402080238CE81A0083
:10691400026500F0FFFC002818BF00F0DFF910202A
:10692400C9F2C000009006200190072002907F2049
:10693400CDE9030540F6B430C1F200006946059480
:1069440001F0AAF8002818BF00F0C8F90020CCF222
:10695400527000900C20019040F6B430C1F2000057
:10696400694601F099F8002818BF00F0B7F904202F
:10697400C0F6600000901220019040F6B430C1F2DD
:106984000000694601F088F8002818BF00F0A6F955
:106994000220C0F2304000901820019040F6B4303C
:1069A400C1F20000694601F077F8002818BF00F032
:0669B40095F908B0B0BD2A
:0269BA00FEE7F6
:1069BC0080B582B041F24800C4F2020001680022A6
:1069CC0041F004010160016801F004010191019999
:1069DC00016841F0010101600068002100F0010034
:1069EC00009000980B20FCF751FF0B20FCF78EFF5A
:1069FC000C2000210022FCF749FF0C20FCF786FF3D
:106A0C000D2000210022FCF741FF0D20FCF77EFF3A
:106A1C000E2000210022FCF739FF0E20FCF776FF38
:106A2C000F2000210022FCF731FF0F20FCF76EFF36
:106A3C00102000210022FCF729FF1020FCF766FF34
:106A4C00112000210022FCF721FF112002B0BDE82B
:066A5C008040FCF75BBF67
:026A6200FEE74D
:106A640010B59CB0044600201B90CDE91900CDE977
:106A7400170002A85421FFF743FE206846F60041A0
:106A8400C4F20001884233D046F60001C4F200018A
:106A9400884268D14FF4805002904FF000701090FB
:106AA40002A8FDF7C9FD002818BF00F017F941F24C
:106AB400FC21C1F200010A6841F24C00C4F2020058
:106AC400531C0B6042B9C16841F00071C160C168D8
:106AD40001F0007101910199016841F00201016026
:106AE4000068602100F002000190019809202CE068
:106AF4004FF4805002904FF00070109002A8FDF700
:106B04009BFD002818BF00F0E9F841F2FC21C1F216
:106B140000010A6841F24C00C4F20200531C0B60ED
:106B240042B9C16841F00071C160C16801F00071EF
:106B340001910199016841F0020101600068182186
:106B440000F00200019001980B2017910221189186
:106B540000211B9040F20040CDE91911C4F6000059
:0A6B640017A902F0CFFE1CB010BD0F
:026B6E00FEE740
:106B700080B541F2F01047F60001C1F20000C4F206
:106B8000000141F22E220023C0F2E2024FF0010C7C
:106B900080E80E10C0E90433C0E90633036203F055
:106BA00035F8002818BF00F09BF841F2F010C1F250
:106BB0000000002103F06CFA002818BF00F090F8E4
:106BC00041F2F010C1F20000002103F0B7FA0028F2
:106BD00018BF00F085F84FF48000BDE88040FDF755
:026BE0005FBC98
:026BE200FEE7CC
:106BE400B0B541F24420C1F20000012104F08EF955
:106BF4004BF6BE6188426FD14BF6AA70C0F6000016
:106C040004F0D3FD41F24424C1F2000420460221E1
:106C140004F07CF940F20005C1F20005C5F82C012E
:106C24002046032104F072F9C5F8300120460421FE
:106C340004F06CF9C5F834012046052104F066F926
:106C4400C5F838012046062104F060F9C5F828018A
:106C54002046072104F05AF9C5F80C012046082102
:106C640004F054F9C5F810012046092104F04EF946
:106C7400C5F8400120460A2104F048F9C5F8480146
:106C840020460B2104F042F9C5F8F40020460C21FB
:106C940004F03CF9C5F8780120460D2104F036F9DA
:106CA400C5F8D801D5F840014FF4616180FB0102B9
:106CB400C5E95802D5F8D80180FB0102C5E978027C
:106CC400D5F8480180FB0102C5E95A02D5F8F40061
:0A6CD40080FB0101C5E93E01B0BDDF
:026CDE00FEE7CF
:106CE0004EF2BA6072B6C0F6000004F060FD00BF5C
:026CF000FEE7BD
:026CF200FEE7BB
:106CF400B0B58EB001AD044628463421FFF700FD3F
:106D04002846FDF795F88CB34EF63C60C0F60000BB
:106D140004F04BFD0598AA2837D102200190BB202E
:106D2400059002F07FFA28B14EF2C960C0F6000067
:106D340004F03BFD02F08EFA28B14CF24200C0F69A
:106D4400000004F032FD4EF65C60C0F6000004F072
:106D54002CFD01A802F0A6FAE0B14DF69E30C0F673
:106D6400000004F022FD02F08DFA4CE00598BB28E7
:106D740026D102200190AA20059002F053FA10B304
:106D84004EF2C960C0F600003BE04DF65320C0F659
:106D9400000013E002F076FA4EF66C60C0F60000D4
:106DA40004F003FDFDF738F84CF28E00C0F6000045
:106DB40004F0FBFC4EF68460C0F6000004F0F5FC21
:106DC40001200EB0B0BD4BF6F670C0F6000004F022
:106DD400ECFC02F03FFA20B14CF24200C0F6000095
:106DE4000FE04DF6CE10C0F6000004F0DEFC01A862
:106DF40002F058FA50B102F045FA4DF63220C0F6CE
:106E0400000004F0D2FC00200EB0B0BD4EF62060AD
:106E1400C0F6000004F0C9FC02F034FA4EF66C60CF
:106E2400C0F6000004F0C1FCFCF7F6FF4CF28E0043
:106E3400C0F6000004F0B9FC4DF6E310C0F6000003
:026E4400BCE7A9
:026E4600FEE765
:106E480010B58EB001AC20463421FFF757FC204620
:106E5800FCF7ECFF06200190BB2005904FF4C440DE
:106E680006904FF4C040079002F0DAF928B14EF2CC
:106E7800C960C0F6000004F096FC02F0E9F928B1F8
:106E88004CF24200C0F6000004F08DFC4EF65C6047
:106E9800C0F6000004F087FC01A802F001FA0446DD
:106EA80040B14DF69E30C0F6000004F07CFC02F0C4
:106EB800E7F915E002F0E4F94EF66C60C0F6000060
:106EC80004F071FCFCF7A6FF4CF28E00C0F600003F
:106ED80004F069FC4EF68460C0F6000004F063FC20
:0A6EE800B4FA84F040090EB010BDAA
:026EF200FEE7B9
:106EF400006800F130414FEA312106293BD8DFE830
:106F040001F0043A3A3A1C2E3B0040F2006341F28D
:106F1400C021C5F20003C1F20001012298420A60B7
:106F24002AD040F20051C5F20001884217D040F245
:106F34000041C5F2000188421DD140F2006341F2D4
:106F4400BC21C5F20003C1F20001012298420A608B
:106F540012D040F20051C5F2000188420BD140F238
:106F6400006341F2B821C5F20003C1F2000101221D
:106F740098420A6000D0704741F2B420C1F2000088
:066F8400012101607047CD
:026F8A00FEE720
:106F8C0080B541F2442042F60001C1F20000C4F287
:106F9C00000100224FF0804E7F234FF0FF0C80E861
:106FAC000E10C0E90422C0E9062E026203F0BEFEF8
:0E6FBC00002814BFBDE8804080BDFFF78BBEEB
:026FCA00FEE7E0
:106FCC00B0B540F6D05043F60041C1F20000C4F217
:106FDC0000014FF4827200234FF4E06C4FF0010E6D
:106FEC004FF48024102580E80E100721C0E9043EE0
:106FFC00C0E90645C0E90833C0E90A31C0E90C33E1
:10700C0003F094FF002814BFBDE8B040B0BDFFF7FB
:02701C0061BE53
:02701E00FEE78B
:10702000F0B587B0006843F60041C4F200010025C6
:107030008842CDE90555CDE90355029501D007B049
:10704000F0BD41F24C00C4F20200C16802AC41F450
:107050000041C160C168022601F40041019101991B
:107060000168062741F001010160016801F001019A
:1070700001910199016841F0040101600068214615
:1070800000F00400019001984FF4004002904FF08E
:107090009040CDE903650595069702F035FC4FF465
:1070A000E050CDE9020640F60000C4F6000021469B
:0E70B000CDE90455069702F027FC07B0F0BDAD
:0270BE00FEE7EB
:0270C000FEE7E9
:0270C200FEE7E7
:0270C400FEE7E5
:0270C600FEE7E3
:0270C800FEE7E1
:0270CA00FEE7DF
:0270CC00FEE7DD
:0270CE00FEE7DB
:0270D000FEE7D9
:0270D200FEE7D7
:0270D400704703
:0270D600FEE7D3
:0270D8007047FF
:0270DA00FEE7CF
:0270DC007047FB
:0270DE00FEE7CB
:0670E000042002F087BD50
:0270E600FEE7C3
:0670E800802002F083BDD0
:0270EE00FEE7BB
:1070F0002DE9F0419CB00446002602A854211B96BD
:10710000CDE91966CDE91766FFF7FCFA206844F26D
:107110000041C4F2000188423CD043F60001C4F2B1
:107120000101884240F0A28001200290002402A8C0
:107130000394FDF783FA002818BFFFF7D1FD41F251
:107140005800C4F20200816841F480418160806887
:1071500000F480400190019841F24C00C4F202001A
:10716000016841F004010160006817A900F0040003
:1071700001900198302017900220CDE918040720D3
:107180001B9040F60000C4F600001A9402F0BCFB0D
:10719000252463E0022502A802950496FDF74EFA25
:1071A000002818BFFFF79CFD41F25800C4F202000E
:1071B000016841F24C0641F4003101600068C4F2FC
:1071C000020600F40030019001983068002740F07A
:1071D00001003060306817A900F0010001900198AB
:1071E0000C20CDE9170507201B904FF09040CDE90A
:1071F000197702F089FB40F65C75A6F57E60C1F256
:1072000000051A214FF0800885E883002846C5E96B
:107210000378C5E90577C5E9077701F057FD002830
:1072200018BFFFF75DFDC4F88050AC6240F6FC6506
:10723000A6F6CC70C1F200051B21102285E887015B
:107240002846C5E90577C5E9077701F03FFD002825
:1072500018BFFFF745FDE567AC62262420460021F4
:107260000022FCF719FB2046FCF756FB1CB0BDE8DA
:02727000F081AB
:02727200FEE735
:1072740010B596B0044601A85421FFF741FA2068DE
:1072840045F60041C4F20001884201D016B010BD99
:107294004FF4005001900020109001A8FDF7CCF9A4
:1072A400002818BFFFF71AFD41F25800C4F202008B
:1072B400016841F400010160006800F400000090DE
:0672C400009816B010BD99
:0272CA00FEE7DD
:1072CC0041F2707041F2A021C1F20000C1F2000144
:0A72DC0000680A681044086070475B
:0272E600FEE7C1
:1072E80010B504466FF00200044207D04CF2E200E9
:1072F800C0F6000040F2A221FCF728F83020C4F2C2
:0E7308000100016821F002012143016010BD67
:02731600FEE790
:1073180070B582B0044600200190ECB1206800F1FD
:1073280030404FEA3020062838D8012101FA00F011
:1073380010F0730F32D06068B0F5801F0FDBB0F526
:10734800001F19DAB0F5C01F36DAB0F5801F44D037
:10735800B0F5A01F41D038E0012002B070BDB0F5F3
:10736800403F13DBB0F5002F21DAB0F5403F34D0B1
:10737800B0F5802F31D028E0B0F5201F21DAB0F524
:10738800001F2AD0B0F5101F27D01EE028B3B0F593
:10739800803F22D0B0F5003F1FD016E04CF28A1093
:1073A800C0F6000040F29B11FBF7D0FFC3E714D0F2
:1073B800B0F5402F11D008E00FD0B0F5E01F0CD089
:1073C80003E00AD0B0F5301F07D04CF28A10C0F69F
:1073D80000004FF4CE71FBF7B9FFA0684FEAF00048
:1073E800042807D34CF28A10C0F6000040F29D1121
:1073F800FBF7ACFFE06840F40040B0F5004F07D061
:107408004CF28A10C0F600004FF4CF71FBF79EFFD4
:10741800206944F20A01884207D34CF28A10C0F668
:10742800000040F29F11FBF791FF6069022807D323
:107438004CF28A10C0F600004FF4D071FBF786FFBB
:10744800607F022807D34CF28A10C0F6000040F291
:10745800A111FBF77BFF206B4FEAB020042807D36C
:107468004CF28A10C0F600004FF4D171FBF76EFFA2
:10747800E06AA0F588614FEA71111C2900F2D481F5
:10748800012202FA01F14DF6E572C1F6010211423C
:1074980000F0CA81606B002818BFB0F1806F40F01F
:1074A800DD8094F83800022807D34CF28A10C0F621
:1074B800000040F2A511FBF749FFA069042809D094
:1074C800082807D04CF28A10C0F600004FF4D37198
:1074D800FBF73CFFE06B40F48050B0F5805F07D0CD
:1074E8004CF28A10C0F6000040F2A711FBF72EFFFD
:1074F800207F022807D34CF28A10C0F600004FF410
:10750800D471FBF723FF94F84000022807D34CF20C
:107518008A10C0F6000040F2A911FBF717FF606956
:1075280038B3206A0138102807D34CF28A10C0F605
:10753800000040F2AD11FBF709FF94F8240002287F
:1075480007D34CF28A10C0F600004FF4D771FBF74E
:10755800FDFE94F8240001280BD1A06A0138082800
:1075680007D34CF28A10C0F600004FF4D971FBF72C
:10757800EDFE94F8240001280AD1607F012807D184
:107588004CF28A10C0F6000040F2B711FBF7DEFE9D
:10759800E06D30B92046FBF76DFA0020206684F8CC
:1075A80058002168886880004FF6C070C5F6FF70E3
:1075B80042BF8A6802408A608A68D2001CD48A68FE
:1075C80000F18050104040F08050886041F2807097
:1075D800C1F20000006842F663528009C0F23E52D0
:1075E800A0FB02029009022202EB400001900198E0
:1075F80010B101980138F9E78868C00009D4E06D36
:1076080040F01000E065206E40F001002066012087
:1076180000E000208A68E36D02F0040203F0100322
:10762800D218E26D16D122F481720232E2658A68BC
:10763800D20740D140F2001341F48072C5F2000332
:107648009A4240F20802C5F2000214D11368D2F837
:10765800005118E042F010010120E2E0B0F1006FA3
:107668003FF41FAF4CF28A10C0F600004FF4D271FD
:10767800FBF76CFE15E7D2F800C4D2F80055D2F833
:10768800003645EA0C052B43DB0714D102F1F80359
:1076980099424FF4E063D4F804C008BF4FF4407334
:1076A800B1F1A04F08BF4FF44073D55825F47C15AD
:1076B80045EA0C05D550627FE36BD4E902C543EA7D
:1076C80042322A4394F8243042EA0C02012B42EA5F
:1076D800034206D1A36A0025CFF6FE7505EB4343A6
:1076E8001A43E36A23B1256B03F478732B431A43D7
:1076F800CB6844F20705CFF6F0752B401A43CA60F1
:107708000A69636B22F040621A430A618A681207A9
:1077180078D494F83820237F520042EA8332CB6829
:1077280044F20205AB431A43CA6022690B694AB1A5
:1077380043F480330B61D1F8C03043F6FF75AB4397
:107748001A4307E023F480320A61D1F8C02043F6D7
:10775800FF739A43C1F8C02094F84020012A4DD104
:10776800616C05464FEAB101082908D34CF28A102A
:10777800C0F6000040F27621FBF7E8FD2846A16C30
:107788004FEA7111092908D34CF28A10C0F600009B
:1077980040F27721FBF7DAFD2846E16C41F40071ED
:1077A800B1F5007F08D04CF28A10C0F600004FF403
:1077B8001E71FBF7CBFD2846216D40F2014241F4D2
:1077C8008061914208D04CF28A10C0F6000040F265
:1077D8007921FBF7BBFD28462168D4E911E3D4E9F8
:1077E800135C0A6940F2FD76B24342EA0E021A437C
:1077F8002A4342EA0C0242F0010202E00A6922F03E
:1078080001020A61216862690B6B012A23F00F02E9
:1078180002BF236A013B1A430A63E16D012262F346
:107828000101E16502B070BD21686FF0030301F149
:10783800304203EB3223032B0ED2B0F58C6F1EDBE4
:10784800B0F5986F33DAB0F58C6F3FF423AEB0F52E
:10785800946F3FF41FAE53E04FEA3222012A4CD80E
:10786800B0F5986F17DAB0F58C6F27DAB0F5806F3E
:107878003FF410AEB0F5846F3FF40CAE2BE0002857
:107888003FF408AEB0F5806F3FF404AEB0F5846FF6
:107898003FF400AE34E0B0F5CC6F16DAB0F5986F6F
:1078A8003FF4F8ADB0F5BC6F3FF4F4AD13E03FF42E
:1078B800F1ADB0F5BC6F3FF4EDAD21E03FF4EAADBA
:1078C800B0F5946F3FF4E6AD05E03FF4E3ADB0F5F5
:1078D800D06F3FF4DFAD40F20042C5F200029142A2
:1078E800ABD040F20062C5F200029142A5D040F24E
:1078F8000052C5F2000291429FD000283FF4CAAD61
:107908004CF28A10C0F6000040F2A311FBF71EFDEE
:02791800C0E5C8
:02791A00FEE786
:10791C00B0B5016804468A688868C0074FF000005B
:10792C0030D012F002022DD1886800F00D00012831
:10793C001FD1886820F0004020F03F0002308860A2
:10794C0003200860FBF788FE21688968C90701D10C
:10795C000020B0BD054603E020688068C007F7D062
:10796C00FBF77AFE401B0328F6D320688068C0071B
:10797C00F2D0E06D40F01000E065206E40F00100A8
:06798C0020660120B0BDE1
:02799200FEE70E
:1079940070B582B004460020019021688A68D2073D
:1079A40011D14FF6C076C7F6FF76886806F17F02DC
:1079B40010420AD0E06D40F01000E065206E40F007
:1079C40001002066012002B070BD88684FF4C162D6
:1079D400304040F00100886040F20010C5F2000021
:1079E400814208BF4FF40272B1F1A04F08BF4FF4B7
:1079F40002721058000220D4FBF732FE21680A6894
:107A0400D20717D1054603E021680868C00711D1E1
:107A14008868C00704D18868304040F0010088605D
:107A2400FBF71EFE401B0328EED320680068C00746
:107A3400EAD1BFE7002002B070BD41F28070C1F20C
:107A44000000006842F663518009C0F23E51A0FB79
:107A54000101880900EB40000C2101EB800000BF0C
:0E7A6400019001980028C7D001980138F8E77A
:027A7200FEE72D
:067A7400806A00F00FB86B
:027A7A00FEE725
:107A7C00806AC16D41F04001C165016E41F00401A5
:067A8C00016600F001B8E4
:027A9200FEE70D
:027A9400704739
:027A9600FEE709
:027A9800704735
:027A9A00FEE705
:107A9C002DE9F04381B0814600200090D9F8000018
:107AAC000D4600F130404FEA3020062800F2EF80FE
:107ABC00012101FA00F010F0730F00F0E880686803
:107ACC00B0F5007F19DAA0F58071182908D80122C9
:107ADC0002FA01F141F24102C0F2041211421BD12F
:107AEC00182800F2E680012101FA00F041F2400171
:107AFC00C0F2041108420FD1DBE0A0F50071182987
:107B0C0000F2CE80012202FA01F141F24102C0F2F0
:107B1C000412114200F0C480A868062873D2E868E9
:107B2C0040F200087F28C4F27F0809D0404507D0F6
:107B3C004CF28A10C0F6000040F6D521FBF704FC8D
:107B4C002869052807D34CF28A10C0F6000040F6CD
:107B5C00D621FBF7F9FBD9F800006969C068062249
:107B6C0002EA900040F6FF7222FA00F0814207D937
:107B7C004CF28A10C0F6000040F6D721FBF7E4FB6C
:107B8C00286904280BD099F84000012807D14CF241
:107B9C008A10C0F6000040F6DB21FBF7D5FBE96844
:107BAC002868414540F2FF11C2F2B05114D188420D
:107BBC003BDC7F21C1F65051884200F383800221C7
:107BCC00C0F23041884200F0E0814021C1F6201122
:107BDC00884200F0DA81A5E088423BDC3F21C1F607
:107BEC00201188427CDC012800F0CF810221C0F2F8
:107BFC003041884200F0C9810421C0F660018842FE
:107C0C0000F0C381C6E0B0F1004F3FF488AF20F024
:107C1C00010006283FF483AF4CF28A10C0F6000036
:107C2C0040F6D421FBF790FB79E740F2FF71C2F6E6
:107C3C003061884268DC40F20021C2F2B0518842C7
:107C4C0000F0A38140F20041C2F60021884200F00E
:107C5C009C8167E040F6FF71C3F26021884200F31B
:107C6C00848040F20021C2F2B051884200F08D8134
:107C7C0040F20041C2F60021884200F0868140F6B5
:107C8C000001C2F63061884200F07F8182E04CF244
:107C9C008A10C0F6000040F6D221FBF755FB0EE728
:107CAC00B0F5407F3FF438AF40F2063188423FF4E4
:107CBC0033AF4CF28A10C0F6000040F6D321FBF72C
:107CCC0043FB29E78021C1F65051884200F05D81C9
:107CDC0040F20011C2F28011884200F0568121E07E
:107CEC004021C1F62011884200F04F818021C1F65D
:107CFC005051884200F0498140F20011C2F28011CB
:107D0C00884200F0428145E040F60001C2F6306145
:107D1C00884200F03A8144F20001C3F6C021884247
:107D2C0000F03381D9F8002002F130414FEA3123C1
:107D3C00062B40F6E42100F27683DFE813F007000F
:107D4C00750074037403B000DA0011010F21C1F245
:107D5C00C001884249DC0421C0F66001884200F071
:107D6C0014810821C0F6904148E041F20001C3F2B1
:107D7C006021884200F0098144F20001C3F6C02161
:107D8C00884200F0028148F20001C3F6F06188429B
:107D9C0000F0FB80D9F8002002F130414FEA31238A
:107DAC00062B4FF42E6100F23E83DFE813F0070040
:107DBC0043033C033C038803C50302044FF6FF71E5
:107DCC00CCF68331884240F302830F21C1F2C0010B
:107DDC00884200F30D830021CCF68431884200F0F8
:107DEC00D4800821C0F690410BE31021C1F2C001F0
:107DFC00884200F0CA802021C1F2F041884200F094
:107E0C00C480A2F1A041A1F580714FEA3123052B6A
:107E1C0040F6E42100F20783DFE813F006000503C7
:107E2C00050341006B00A2001F21C1F2F041884202
:107E3C000FDC0421C0F66001884200F0A680082106
:107E4C00C0F69041884200F0A0801021C1F2C00120
:107E5C0010E02021C1F2F041884200F0968041F2FE
:107E6C000001C3F26021884200F08F8042F20001D1
:107E7C00C3F29061884200F0888040F20061C5F244
:107E8C0000018A426CD040F20051C5F200018A42D6
:107E9C002FD040F20041C5F200018A4272D10F216D
:107EAC00C1F2C00188420EDD1021C1F2C00188422E
:107EBC006BD02021C1F2F041884266D048F200011B
:107ECC00C3F6F06107E00421C0F6600188425CD083
:107EDC000821C0F69041884257D040F20061C5F2AB
:107EEC0000018A423CD040F20051C5F200018A42A6
:107EFC0048D11F21C1F2F04188420FDD41F6FF71DC
:107F0C00C3F29061884217DC2021C1F2F041884213
:107F1C003BD041F20001C3F2602117E00421C0F60E
:107F2C006001884231D00821C0F6904188422CD0A3
:107F3C001021C1F2C00109E042F20001C3F29061CC
:107F4C00884222D048F20001C3F6F06188421CD06E
:107F5C0040F20831C5F2000101F53E718A4211D19F
:107F6C0041F20001C3F2602188420ED042F20001BE
:107F7C00C3F29061884208D048F20001C3F6F06168
:107F8C00884202D040F6E4214DE299F858000128CD
:107F9C0003D1022001B0BDE8F0830121D9F8000023
:107FAC0089F858108168490732D4D5E900121F2688
:107FBC00C2F3012300EB83031F6B02F01F029640F8
:107FCC00C1F38461B7439140394319638168826876
:107FDC0001F0040102F00802891840F0CC802F68EF
:107FEC0000F114010422C7F34066AB6802EAD752D1
:107FFC0051F82640C7F304560727B740B3F1004F9A
:10800C0024EA07070CD18F50096841F000410DE0BC
:10801C00D9F85C0040F02000C9F85C000120D0E1E8
:10802C00B3403B438B50096821F000414161D5E9D5
:10803C000412C36804290BD1016E006E2968C0F3C9
:10804C0084604A034AD091FAA1F1B1FA81F147E078
:10805C00062707EA93039A402B6800EB8100016E18
:10806C004FF20007C0F2FF3703F0F84339401A43D0
:10807C00114341F000410166A86940F08070B0F1F5
:10808C00807F07D04CF28A10C0F6000040F61C31FD
:10809C00FBF75AF9287F022807D34CF28A10C0F656
:1080AC00000040F61D31FBF74FF9D9F800002969A3
:1080BC006030AA6950F8213023F080731A4340F8DD
:1080CC00212029692A7F50F82130012A23F00073DE
:1080DC0008BF03F1007340F821304CE0C1F3846118
:1080EC0088424FF6FF70C0F2070005D1D9F8001096
:1080FC000A6E22F000420A66D9F800104A6E496EE8
:10810C002A68C1F38461024257D092FAA2F2B2FA01
:10811C0082F2914205D1D9F800104A6E22F0004249
:10812C004A66D9F800108A6E896E2A68C1F3846198
:10813C00024247D092FAA2F2B2FA82F2914205D1EF
:10814C00D9F800108A6E22F000428A66D9F8001025
:10815C00CA6ECA6E29680142C2F3846037D091FAA4
:10816C00A1F1B1FA81F1884205D1D9F80000C16EB4
:10817C0021F00041C166D9F800008168C90740F0C0
:10818C008E802A68EF684FF6FF71C0F20701D0F8B5
:10819C00B060134607F018046FF3DF4321FA04F4C0
:1081AC009E43144026434745C0F8B06077D19BB13D
:1081BC0092FAA2F2B2FA82F20FE0C2F38462914216
:1081CC00A9D0AEE7C2F384629142B9D0BEE7C1F345
:1081DC0084618842C9D0CEE7920E013202F01E03B0
:1081EC002A68092B02EA01030AD80BB192FAA2F20F
:1081FC002A680A420FD092FAA2F2B2FA82F20BE08B
:10820C000BB192FAA2F22A680A4213D092FAA2F2A5
:10821C00B2FA82F20FE0920E013202F01F032A68CA
:10822C0001270A4207FA03F113D092FAA2F2B2FA2A
:10823C0082F20FE0920E013202F01F032A6801272E
:10824C000A4207FA03F10DD092FAA2F2B2FA82F2C4
:10825C0009E0920E013202F01F0202EB420241EAE7
:10826C0002510DE0920E013202F01F02002302EBCC
:10827C004202CFF6206303EB0252114341F000712E
:10828C00C1F3406300EB8300AA684369C1F3045156
:10829C0007278F40BB4302FA01F1194341612B6858
:1082AC000020C8F20800034200F08A8040F2083C2B
:1082BC00C5F2000CD9F800600CF58062ACF50275C3
:1082CC001046AE4204BF40F20830C5F20000B6F1D1
:1082DC00A04F04BF40F20830C5F20000016800272F
:1082EC00CCF22137BB4201F0E07E04D01024C9F25D
:1082FC00C004A3422FD10C022DD440F20061C5F270
:10830C0000018E4202D0B6F1A04F59D1016821F084
:10831C00E07141EA0E0141F40001016041F280700C
:10832C00C1F20000006842F663518009C0F23E5170
:10833C00A0FB0101880900EB40000C2101EB80003F
:10834C0000900098E0B300BF0098013800900098AE
:10835C000028F9D134E00024CCF25274A34208BFB7
:10836C005FEA1E6417D00020CCF6843083424FF0B5
:10837C00000008BF11F4800123D1B6F1A04F13D037
:10838C0040F20010C5F20000864219D0701BB0FA02
:10839C0080F0400909E0016821F0E07141EA0E012A
:1083AC0041F0807101600BE00120002818BF62468B
:1083BC00106820F0E07040EA0E0040F4800010607D
:1083CC000020002189F8581001B0BDE8F08342F27A
:1083DC000001CBF2906188423FF4D7AD0021CCF282
:1083EC00213188423FF4D1AD0021CCF2527108E02A
:1083FC001021C1F2C00188423FF4C7AD2021C1F267
:10840C00F04188423FF4C1ADA2F1A041A1F58071C9
:10841C004FEA3123052B4FF42E6104D8DFE803F02B
:10842C000A03034F8CC94CF28A10C0F60000FAF70D
:10843C008BFFAAE50F21C1F2C00188420FDD41F686
:10844C00FF71C3F29061884219DC1021C1F2C001A6
:10845C0088423FF49AAD2021C1F2F04119E000218D
:10846C00CCF2293188423FF490AD0021CCF68C310E
:10847C0088423FF48AAD0821C0F6904109E042F2EF
:10848C000001C3F2906188423FF47FAD0021C4F239
:10849C00527188423FF479AD40F20061C5F200019F
:1084AC008A4200F0868040F20051C5F200018A42F7
:1084BC0042D040F20041C5F200018A4276D1072138
:1084CC00C0F6904188420EDD1F21C1F2F041884276
:1084DC001ADC0821C0F6904188423FF456AD1021B9
:1084EC00C1F2C00119E042F20001CBF2986188425E
:1084FC003FF44BAD0021CCF2527188423FF445ADB4
:10850C000021CCF6843108E02021C1F2F0418842F0
:10851C003FF43BAD0021C4F2213188423FF435AD2C
:10852C0040F20061C5F200018A4242D040F2005193
:10853C00C5F200018A4239D10F21C1F2C001884233
:10854C000FDD41F6FF71C3F29061884219DC1021F6
:10855C00C1F2C00188423FF418AD2021C1F2F041B4
:10856C0019E00021CCF25A7188423FF40EAD002183
:10857C00CCF6843188423FF408AD0821C0F6904116
:10858C0009E042F20001C3F2906188423FF4FDAC75
:10859C000021C4F2213188423FF4F7AC40F208319B
:1085AC00C5F2000101F53E718A4202D04FF42E61F2
:1085BC0039E74FF6FF71CCF2517188424FF42E61BE
:1085CC000FDD41F6FF72C3F29062904219DC00227B
:1085DC00CCF2527290423FF4D8AC0022CCF68432EA
:1085EC0019E00822C8F6904290423FF4CEAC10221B
:1085FC00C9F2C00290423FF4C8AC2022C9F2F0424A
:10860C0009E042F20002C3F2906290423FF4BDAC2A
:0E861C000022C4F2213290423FF4B7AC03E7D3
:02862A00FEE769
:10862C00B0B582B004460020019020680D4600F1E0
:10863C0030404FEA302006284BD8012101FA00F0D7
:10864C0010F0730F45D07F2D0BD00020C4F27F00AB
:10865C00854206D04DF6B330C0F600008521FAF7FE
:10866C0073FE94F85800012802D1022002B0B0BD6C
:10867C00012084F858002046FFF74AF9E16D10B14B
:10868C0041F0100133E041F2021291430231E165F5
:10869C00216805F080438A6822F0404222F03F02B4
:1086AC001A4402F100428A604DF60262C0F20402E2
:1086BC008B68B3F1FF3F16DC019B01330193019BE7
:1086CC009342F5D3E06D40F0100020F00201012040
:1086DC000DE04DF6B330C0F600008421FAF734FEFD
:1086EC007F2DB2D1BDE7E16D012262F30101E1659D
:0A86FC00002184F8581002B0B0BD50
:02870600FEE78C
:108708002DE9F0419CB00446006840F2004740F46F
:108718008060C5F200071546B8420E4607D04DF6F0
:10872800B330C0F6000040F26531FAF70FFE607F03
:10873800022807D34DF6B330C0F6000040F2663188
:10874800FAF704FE206B4FEAB020042807D34DF651
:10875800B330C0F6000040F26731FAF7F7FD94F83D
:108768003800022807D34DF6B330C0F600004FF4A6
:108778005A71FAF7EBFD20688168490703D494F829
:108788005810012903D102201CB0BDE8F08140F245
:1087980000180121C5F2000884F858100021B0F132
:1087A800A04F1891199104D0B8420FD108F58060F4
:1087B80000E0404601902046FFF7E8F890B1B0B1DC
:1087C800002184F858101CB0BDE8F0810020019009
:1087D800E16D41F02001E16584F8580001201CB0EA
:1087E800BDE8F08101A8FFF7D1F80028E8D1226898
:1087F800606DE16D40F60173994301F58071E165A3
:1088080043F6050147F675274FF0000CC0F6000146
:10881800C0F60007C4F860C047F67D23C0E90B170F
:1088280040F20C71C0F60003C5F200011C27436337
:1088380008F50373424508BF1946176084F858C005
:108848005768B2F1A04F08BF194647F010035360AC
:1088580032462B4600F0C2FB21688A6822F00042AB
:0E88680022F03F0204328A601CB0BDE8F081AD
:02887600FEE71B
:1088780070B582B00446006840F2004640F480605B
:10888800C5F20006B0420D4607D04DF6B330C0F62B
:10889800000040F64C01FAF759FD2868092800F253
:1088A8008480012101FA00F040F2EF2108427CD0D7
:1088B800286890B16868002818BFB0F5004F2BD120
:1088C800A8684FEA30200C2807D34DF6B330C0F61D
:1088D800000040F65101FAF739FD94F858000128D4
:1088E80002D1022002B070BD0120002384F8580094
:1088F80001930093226840F2080CC5F2000CB2F113
:10890800A04F0CF1F80013D0B2421ABF0021012386
:108918000CF59F6173B13EE0B0F5404FD0D04DF6F5
:10892800B330C0F600004FF40561FAF70FFDC7E752
:10893800014683BB89689368194349072BD44FF4D0
:10894800E061D5F800E0824208BF4FF44071B2F10F
:10895800A04F08BF4FF440715CF80100BEF1000F52
:1089680020F460402AD06E6894F8383042F480725F
:1089780046EA4333184340F20013C5F200039A4213
:108988004CF801002CD1DCF80000DCF80021104381
:10899800C0074CD12EE0E06D40F02000E0650120DA
:1089A800002184F8581002B070BD4DF6B330C0F6FF
:1089B800000040F64D01FAF7C9FC79E740F20013D0
:1089C80042F48072C5F200039A424CF801001BD1B0
:1089D800DCF80000DCF800211043C00727D11DE0B7
:1089E800DCF80004DCF80025DCF8003610431843F6
:1089F800C0071CD15CF8010040F61F72AB689043B9
:108A0800184340EA0E000EE0DCF80004DCF800250C
:108A1800DCF8003610431843C00708D15CF80100A1
:108A280040F61F7290434CF801000020B8E7002080
:028A3800B6E79F
:028A3A00FEE755
:108A3C000138010E01D0012070474EF21001CEF228
:108A4C00000148604EF62350CEF20000F022027076
:0A8A5C000020072288600A607047BE
:028A6600FEE729
:108A680060B310B50446006843F20001C4F2020185
:108A7800884206D04CF25A20C0F600007021FAF75E
:108A880065FC607F20B9002020772046FAF7A0F91E
:108A9800022060772079022806D34CF25A20C0F6CB
:108AA80000007E21FAF752FC207948B1D4E902127D
:108AB800204600F0B5F868B1012010BD01207047CC
:108AC800206841F6B751C0F2C1414161816821F087
:108AD800180181606079022806D34CF25A20C0F64A
:108AE80000009021FAF732FC6079002814BF206951
:108AF8004FF0FF30616922684FEA71110429106153
:108B080006D34CF25A20C0F600009C21FAF71EFC4E
:108B18002068D4E90512836842F0800223F06003DC
:108B28001943802A816006D04CF25A20C0F6000012
:108B3800A021FAF70BFC2068A169226A8368013A30
:108B480023F080031943032A816006D34CF25A208C
:108B5800C0F60000A521FAF7F9FB01206077002094
:028B680010BD3E
:028B6A00FEE724
:108B6C0010B593080ED0D0F800E04FF0000C00BF09
:108B7C0051F80C40013B24BA0CF1040CCEF8004027
:108B8C00F6D101E04FF0000C02F00302DFE802F036
:108B9C001C02071111F80C100268117014E001EBA3
:108BAC000C0211F80C105278036842EA012119806A
:108BBC000AE001EB0C0211F80C105378046843EA3C
:0E8BCC0001212180917821700068006810BDA1
:028BDA00FEE7B4
:108BDC00B0B505460220687728682B6A8468012B9B
:108BEC0044F00104846010D0022B0AD0032B10D166
:108BFC002AB100BF51F8043B013A0360FAD1006876
:108C0C0008E02846FAF7AEFE04E02846FFF7A8FF76
:0A8C1C0000E0002001216977B0BDDF
:028C2600FEE767
:108C2800F0B581B04FEAF20714460D46042F064608
:108C380006D34EF26B10C0F600005F21FAF786FBF0
:108C4800E8070BD10120002232B131684D618A68F2
:108C580022F0180222438A6001B0F0BD1F2100BF34
:108C680049B1013901F01F0025FA00F0C007F7D01B
:108C7800032F04D9E6E74FF0FF31032FE2D8002095
:108C88000122DFE807F002030C15DDE710294FF099
:108C9800000238BF01220F2988BF0120D4E7082924
:108CA8004FF0000238BF0122072988BF0120CBE717
:108CB80007294FF0000238BF0122062988BF01208A
:028CC800C2E701
:028CCA00FEE7C3
:108CCC00D0B12DE9F0410446006840F20741C4F2EE
:108CDC000201884212DC5721C4F20201884222DCD4
:108CEC002F21C4F20201884238DC0821C4F20201AF
:108CFC00884257D01C2150E00120704740F2574168
:108D0C00C4F2020188421ADC40F22F41C4F2020183
:108D1C0088422ADC40F20841C4F20201884241D068
:108D2C0040F21C4139E07F21C4F20201884225DC6B
:108D3C005821C4F20201884234D06C212DE040F25B
:108D4C007F41C4F2020188421FDC40F25841C4F258
:108D5C000201884226D040F26C411EE03021C4F260
:108D6C00020188421ED0442117E040F23041C4F287
:108D7C000201884216D040F244410EE08021C4F238
:108D8C00020188420ED0942107E040F28041C4F2E7
:108D9C000201884206D040F29441C4F2020188429A
:108DAC0040F0D780A068002818BF102840F0AD8094
:108DBC00E06840F04000402806D04CF27A40C0F603
:108DCC000000A521FAF7C0FA206940F08000802845
:108DDC0006D04CF27A40C0F60000A621FAF7B4FA9D
:108DEC006069002818BFB0F5807F40F09A80A069B8
:108DFC00002818BFB0F5806F40F09F80E06940F00C
:108E0C002000202806D04CF27A40C0F60000A921A0
:108E1C00FAF79AFA206A4FEA3030042806D34CF25B
:108E2C007A40C0F60000AA21FAF78EFA606874281E
:108E3C0006D34CF27A40C0F60000AC21FAF784FA63
:108E4C0040F2000CC4F2020C20684FF6F8330CF51B
:108E5C008162CBF6FD73904238BF03F5806303EB60
:108E6C0000024CF6CD43CCF6CC43A2FB03230CF50D
:108E7C0080616FF00302D4E90287D4F810E03CBFA4
:108E8C000021C4F2020102EA9302C4E91012022189
:108E9C0084F82510016847F6F072914304F114022E
:108EAC0041EA08016CCA394341EA0E0111431943E6
:108EBC00294331430160204600F054F8A06804F1C6
:108ECC004801B0F5804F04BF0020606060680EC997
:108EDC00C7B2013803280F60536009D8204600F050
:108EEC0067F804F1540007C8002303604A6003E0EC
:108EFC000020C4E91500E06500200121E06384F83E
:108F0C00251084F82400BDE8F081B0F5804F3FF4C3
:108F1C004FAF4CF27A40C0F60000A421FAF714FAD5
:108F2C0046E7B0F5007F3FF462AF4CF27A40C0F6F2
:108F3C000000A721FAF708FA59E7B0F5006F3FF4E3
:108F4C005DAF4CF27A40C0F60000A821FAF7FCF9AC
:108F5C0054E74CF27A40C0F60000A321FAF7F4F97A
:028F6C0020E7FC
:028F6E00FEE71C
:108F700080B501684CF6CD4301F0FC02083ACCF60E
:108F8000CC43A2FB032C40F20842C4F20202D0F808
:108F900044E002F58363914238BF02F57E732EF000
:108FA000030103EB010ECCF30413012102F58F62E0
:0A8FB0009940C0E912E2016580BD9E
:028FBA00FEE7D0
:108FBC00017940F600120139C4F2020202EB81037E
:108FCC0002F1400C01F01F01012202FA01F1C0E98B
:068FDC00153CC165704761
:028FE200FEE7A8
:108FE400F0B581B016464FF6FF720F46591EC0F217
:108FF40003021D469142044607D34CF27A40C0F660
:10900400000040F2AB11FAF7A3F994F82400012808
:1090140020D0012084F8240094F82500012816D1DA
:10902400022084F825000020E063206832460168AD
:109034002B4621F00101016020463946FAF7B4FCC1
:109044002068226B016842B141F00E010BE0002060
:1090540084F82400022001B0F0BD21F00401016075
:10906400016841F00A010160A06C0168C90342BFB4
:10907400016841F480710160606D00281EBF0168C1
:1090840041F4807101602068016841F001010160D0
:06909400002001B0F0BD58
:02909A00FEE7EF
:10909C00014690F82500022827D180B50868D1E94F
:1090AC0010CE8A6C036823F00E030360136823F45C
:1090BC0080731360026822F0010202600EF01F0040
:1090CC00012202FA00F0CCF80400D1E91320506020
:1090DC00486D30B1026822F480720260D1E9160248
:1090EC0042600020BDE8804002E00420C8630120FB
:0E90FC00012281F82520002281F824207047EF
:02910A00FEE77E
:10910C0090F82510022930D180B50168D0E910CE35
:10911C00826C0B6823F00E030B600B6823F00103C9
:10912C000B60116821F4807111600EF01F02012197
:10913C0001FA02F2CCF80420D0E913325A60426DE5
:10914C0032B1136823F480731360D0E91623536093
:10915C0080F82510826B002180F824100AB190470A
:10916C000021BDE88040084670470421C1630121FD
:0E917C00002280F8251080F824200846704755
:02918A00FEE7FE
:10918C00B0B5D0E910C30268DCF8001003F01F037F
:10919C000424D2F800E09C400C4218BF1EF00405D9
:1091AC001AD102249C400C4218BF1EF002051FD19C
:1091BC00D94009071BD51EF0080118D0116821F001
:1091CC000E011160012101FA03F2CCF80420C163F5
:1091DC0080F82510416B18E0116889065EBF116894
:1091EC0021F004011160CCF80440016B91B9B0BDC1
:1091FC001168890606D4116821F00A011160012159
:10920C0080F82510CCF80440C16A0022002980F8AF
:0A921C002420ECD0BDE8B040084764
:02922600FEE761
:1092280042F20800C4F20200C168B1F1FF3F01DD5B
:109238000020704740F22311C4F26751016048F6DC
:0E924800AB11CCF6EF510160C068C00F70474B
:02925600FEE731
:1092580042F20C00C4F202008168490001D40020E7
:10926800704742F63B21C0F61901016046F67F615E
:0E927800C4F65D4101608068C0F380707047ED
:02928600FEE701
:1092880042F21400C4F20200016841F0804101601A
:0E9298000068012100F0804081EA907070476C
:0292A600FEE7E1
:1092A8002DE9F04F85B004460068402807D34EF2F8
:1092B800DC60C0F6000040F23B11FAF747F841F2D3
:1092C8004C79C1F2000999F80000012803D1022065
:1092D80005B0BDE8F08F0120002589F80000C9F825
:1092E8000450207842F2140B47F2E058C4F2020B03
:1092F800C1F6FF78C0074FF6FF7A00F08080D4E906
:109308000175E668042F56D8032F54D0B8F800002A
:10931800504504D0B8F80000B0F5007F31D1802066
:10932800854207D34EF2DC60C0F600004FF42A7184
:10933800FAF70CF8B8F80000504504D0B8F8000067
:10934800B0F5007F2AD18020864207D34EF2DC6038
:10935800C0F6000040F2A921F9F7F8FF4FF47A703F
:10936800FAF72EFD08B1012549E0042F3AD8DFE8C5
:1093780007F003302B39350045EA0640CBF81800D2
:1093880030E0B8F8000050454FF02000C8D0B8F8D9
:109398000010B1F5807F08BF4020C1E7B8F8000091
:1093A80050454FF02000CFD0B8F80010B1F5807FBD
:1093B80008BF4020C8E74EF2DC60C0F6000040F26B
:1093C800A721F9F7C3FFA1E745EA0640CBF8380023
:1093D80008E045EA0640CBF81C0003E045EA0640F1
:1093E800CBF83C00DBF8000040F40030CBF800007C
:1093F8004FF47A70FAF7E4FC050018BF01252078CD
:10940800800701D42F461EE02669AA2E18BFBB2E5E
:109418003CD14FF47A70FAF7D3FC012798B9DBF8FE
:109428000C0020F0FF003043CBF80C00DBF8000004
:1094380040F40030CBF800004FF47A70FAF7C0FC23
:10944800002808BF2F462078400740F1E680D4E97D
:1094580005654FF6FF71701EC0F20101884207D3FF
:109468004EF2DC60C0F6000040F21931F9F76EFFE9
:109478004FF47A70FAF7A4FC08B10127CDE0F007A1
:1094880004970ED10020039000211AE0CC2EC0D002
:109498004EF2DC60C0F600004FF43A71F9F756FF5F
:1094A800B7E705F4E060B0F5A06F039007D34EF27C
:1094B800DC60C0F6000040F22F31F9F747FF4FF4A7
:1094C800E06106F0060341EAC32106F4805341EA4D
:1094D800830106F0780741EA473706F0800147EA3A
:1094E800413705EAC620029705F4000700F48050CA
:1094F80005F480120197770705F4005E009248BFD3
:109508007044002B05F4804B18BF5844370705F406
:10951800803848BF4044F70605F4003C48BF40EA9D
:109528000C00B70605F4802948BF40EA0900770611
:1095380005F4002A48BF40EA0A000029009B18BF2A
:109548001843B305019B48BF184305F080727305A3
:1095580048BF104305F0007E320548BF40EA0E00C0
:1095680005F0806705F00061B20448BF3843720413
:1095780048BF0843039940EA01074FF0607106F4B9
:10958800C04001EA863141EA40303104029901EBDA
:10959800000808D441F24C7942F2140BC1F20009D8
:1095A800C4F2020B16E041F24C7942F2140B15F0AA
:1095B800405AC1F20009C4F2020B07D14EF2DC6036
:1095C800C0F6000040F2BB31F9F7C0FE47EA0A07CF
:1095D80048F0405805F0804116F4803018BF0F431A
:1095E800DBF80C1048EA803021EA00003843CBF859
:1095F8000C00DBF8000040F40030CBF800004FF41A
:109608007A70FAF7DDFB47F2E058049FC1F6FF785D
:109618004FF6FF7A002818BF01272078000740F18D
:10962800E080D4E90865AE4200F0DB80E069049789
:10963800029000F00300039001384746022807D340
:109648004EF2DC60C0F600004FF47D71F9F77EFE43
:1096580040F2000AC0F6040AB6F1006F0AF5802845
:109668000CD338884FF6FF71884240461EBF3968D0
:109678004FF0006061F39920864207D34EF2DC6018
:10968800C0F6000040F2F631F9F760FEB5F1006F60
:109698000BD338884FF6FF7188421EBF38684FF0E9
:1096A800006860F39928454507D34EF2DC60C0F6A0
:1096B800000040F2F731F9F749FE4FF47A70FAF7F3
:1096C8007FFB10B1B846012789E00020C4F20100F1
:1096D80001683888C905039AB8464FF6FF710AD45D
:1096E80088424FF0006111D0D8F800004FF0006AAE
:1096F80060F3582A0AE0884251461EBFD8F8000095
:109708004FF0006160F358214FF0006ADBF80C005D
:109718004002029800F0004012D4012A21D1DBF85F
:10972800102047F6FF7306F178419A4342EA111177
:10973800CBF8101005F1784109090BF1140233E058
:10974800012A1FD1DBF8103047F6FF77721ABB43A6
:1097580043EAD202691ACBF81020C9080BF11402A7
:1097680022E0022A26D1DBF8302047F6FF7306F103
:1097780078419A4342EA1111CBF8301005F178414B
:1097880009090FE0022A15D1DBF8302047F6FF73EC
:10979800A6EB0A019A4342EAD101CBF83010A5EBB7
:1097A8000A01C9080BF13402136847F6FF77BB4377
:1097B80019431160DBF8141021F000410843CBF87D
:1097C8001400DBF8000040F40030CBF800004FF440
:1097D8007A70FAF7F5FA049F002818BF01274FF6A8
:1097E800FF7A2078800654D5D4E90B65701E0228CC
:1097F80007D34EF2DC60C0F6000040F26541F9F78D
:10980800A5FDB8F80000504504D0B8F80000B0F540
:10981800007F1DD18020854207D94EF2DC60C0F65A
:10982800000040F26641F9F791FD4FF47A70FAF7BB
:10983800C7FA08B101272CE0022E16D0012E1BD141
:10984800DBF85C0020F0FF002843CBF85C0013E055
:10985800B8F8000050454FF02000DCD0B8F80010F0
:10986800B1F5807F08BF4020D5E7DBF8600020F025
:10987800FF002843CBF86000DBF8000040F400301C
:10988800CBF800004FF47A70FAF79AFA002818BF5C
:1098980001272078C00601D438462AE0A46A6FF46C
:1098A8008030044207D04EF2DC60C0F6000040F27F
:1098B8009A41F9F74BFD4FF47A70FAF781FA0028CC
:1098C8004FF0010015D1DBF85C0020F48030204314
:1098D800CBF85C00DBF8000040F40030CBF8000067
:1098E8004FF47A70FAF76CFA01460120002908BF94
:0E98F8003846002189F8001005B0BDE8F08F59
:02990600FEE77A
:109908002DE9F04F85B0039000F138404FEAB020C0
:1099180007280D46019006D34EF23F70C0F60000AE
:10992800A921F9F713FD2868010C01D180B230B9DB
:109938004EF23F70C0F60000AA21F9F707FD6868EB
:10994800B0F5881F80F20781122800F21E810121DC
:1099580001FA00F00F21C0F20601084200F015815B
:109968002868002800F0F480039A4FF0000902F1FB
:109978002001009141F20041C4F600018A424FF0F3
:10998800060208BF052201994FF0030C4FF00008AA
:109998004FF0000B052938BF0A4602920BE000BFC2
:1099A80028680BF1010B30FA0BF108F1020809F1F4
:1099B800040900F0CD80012101FA0BFA10EA0A0728
:1099C800EED0686800F00300013801281FD8E86865
:1099D800042808D34EF23F70C0F60000BB21F9F707
:1099E800B5FC4FF0030C039B0CFA08F198686A6801
:1099F8008843E96801FA08F1084398605868C2F397
:109A0800001120EA0A0001FA0BF10843586068685F
:109A180000F00300032815D0A868032808D34EF2E5
:109A28003F70C0F60000CC21F9F790FC4FF0030C12
:109A3800039B0CFA08F1D868AA68884302FA08F16F
:109A48000843D860686800F00300022827D101980D
:109A5800072808D34EF23F70C0F60000D921F9F765
:109A680075FC4FF0030C2869102808D34EF23F709C
:109A7800C0F60000DA21F9F769FC4FF0030C6FF02B
:109A88000300009C00EA5B00215809F01C020F2328
:109A98002E699340994306FA02F211432150039B21
:109AA8000CFA08F118686A68884302F0030101FAA1
:109AB80008F1084312F4403F18603FF471AF41F2D7
:109AC8006001C4F20201086840F2004440F001005D
:109AD80008600868C4F2010400F0010004900498CA
:109AE8002BF003004FF608462044CFF6FF76815945
:109AF80009F00C020F2393409943029B03FA02F2E8
:109B080011438151A068696840EA070240F20C4697
:109B1800CB0258BF20EA0702A260C4F201063068EF
:109B28008B0240EA070258BF20EA070232606068E9
:109B38008B0340EA070258BF20EA070262602068E8
:109B4800C90340EA070258BF20EA0702226027E754
:109B580005B0BDE8F08FB0F5081F0CDAB0F5881F26
:109B68003FF4FEAEB0F5901F3FF4FAAEB0F5041F17
:109B78003FF4F6AE09E03FF4F3AEB0F5441F3FF40E
:109B8800EFAEB0F5481F3FF4EBAE4EF23F70C0F6B3
:0A9B98000000AB21F9F7DAFBE2E66A
:029BA200FEE7DC
:109BA400B0B50C46054639B94EF23F70C0F6000018
:109BB4004FF4BD71F9F7CCFB2869204018BF012090
:029BC400B0BD32
:029BC600FEE7B8
:109BC800B0B50C46054639B94EF23F70C0F60000F4
:109BD80040F2B311F9F7BAFB686900EA040124EA14
:0A9BE800000040EA0140A861B0BD92
:029BF200FEE78C
:109BF40040F21441C4F201010A68024214BF086031
:069C04007047F9F735BCC2
:029C0A00FEE773
:109C0C0088B110B50446006847F2FF71C4F2000138
:109C1C0088420ADC45F20041C4F20001884218D0A7
:109C2C0045F6000109E00120704747F60001C4F237
:109C3C00000188420DD048F20041C4F20001884274
:109C4C0007D04CF27260C0F600004FF40871F9F7BF
:109C5C007BFBA068B0F5806F07D34CF27260C0F646
:109C6C00000040F22121F9F76FFBE068013802286F
:109C7C0007D34CF27260C0F6000040F22221F9F7D3
:109C8C0063FB206940F40040B0F5004F07D04CF264
:109C9C007260C0F6000040F22321F9F755FB6069B1
:109CAC00B0F5807F07D34CF27260C0F600004FF421
:109CBC000971F9F749FBA069082807D34CF27260C7
:109CCC00C0F6000040F22521F9F73EFBE06940F4B4
:109CDC000020B0F5002F07D04CF27260C0F60000E7
:109CEC0040F22621F9F730FB206A40F40030B0F541
:109CFC00003F07D04CF27260C0F6000040F2272102
:109D0C00F9F722FB94F8410028B9002084F84000B0
:109D1C002046F9F7A1F9242084F8410094E80310B7
:109D2C00E368026821F0706122F0010202600161B7
:109D3C008168012B21F4004181604FF4044108BF7C
:109D4C004FF4004141EA0C0181604168022B21F47F
:109D5C00006108BF01F500614160416841F000718C
:109D6C0041F400414160C16821F40041C16004F13B
:109D7C0010010EC9114341EA0321C160D4E9071255
:109D8C0011430160016841F00101016000202021B4
:0E9D9C00606484F84110206384F8420010BD1A
:029DAA00FEE7D2
:109DAC002DE9F04190460446006847F2FF72C4F278
:109DBC0000021D4690420F4608DC45F20041C4F2F9
:109DCC000001884216D045F6000107E047F6000175
:109DDC00C4F2000188420DD048F20041C4F20001E7
:109DEC00884207D04CF27260C0F6000041F6714117
:109DFC00F9F7AAFA069E002D18BFB5F1807F38D16D
:109E0C0043F6FF70C8F2000086420CDC42F2000000
:109E1C00C8F20000864215D042F20040C8F20000A1
:109E2C0086420FD006E044F20000C8F200008642E1
:109E3C0008D03EB14CF27260C0F6000041F673419E
:109E4C00F9F782FA6FF39F2721684FF4806347EA92
:109E5C00084003EA565328434A6883F07C43304356
:109E6C0083F41C4320F000401A4010434860BDE8C6
:109E7C00F081B5F1007FC3D04CF27260C0F60000E7
:0A9E8C0041F67241F9F760FABAE7F7
:029E9600FEE7E5
:109E98002DE9F04F81B00D46591E89B21E4617466E
:109EA8000229044607D34CF27260C0F6000040F65F
:109EB8006A21F9F74BFA94F8410020280DD1DDF812
:109EC80028A0BAF1000F0CD0DDF82C80B8F1000FF3
:109ED80007D094F8400001280AD1022001B0BDE85B
:109EE800F08F4FF400706064012001B0BDE8F08F7E
:109EF800012084F84000F9F7B1FB814620464FF471
:109F0800004101221923CDF80090FAF77FF80146A5
:109F1800012011B101B0BDE8F08F0C9942F2004266
:109F28002220C8F2000284F8410040204FF0000BC4
:109F380084F84200C4F844B0C4F824A09246A4F8B7
:109F48002A808846A2F5806CF2B220462946002372
:109F5800C4F834B0CDF800C0FFF724FF20464146CE
:109F68004A46FAF7A1F8B0B92068012E08D0390A94
:109F78008162204641464A46FAF796F858B9206861
:109F8800F9B281622046402100224346CDF8009074
:109F9800FAF73CF810B184F840B0A5E7608DB0F549
:109FA800807F07D3FF20208520462946FF224FF0D7
:109FB800807306E0608D29462085C2B220464FF0A6
:109FC8000073CDF800A0FFF7EDFE0026FF270BE099
:109FD800608D29462085C2B220464FF00073009656
:109FE800FFF7E0FE608D90B320460421002243462F
:109FF800CDF80090FAF70AF800287FF475AF2068CA
:10A00800616A406A0870606A218D01306062481E8A
:10A018002085618D01396185618D0029E2D00004B8
:10A02800E0D12046802100224346CDF80090F9F780
:10A03800EDFF00287FF458AF608DB0F5807FC7D35F
:10A04800278520462946FF224FF08073C7E7204620
:10A0580041464A46FAF75EF800287FF445AF206883
:10A068002021C16142684EF60003CFF600631A4012
:10A078004260002084F8411084F8420084F84000CF
:06A0880001B0BDE8F08FFD
:02A08E00FEE7EB
:10A09000B0B50446006847F2FF72C4F20002904275
:10A0A0000D4608DC45F20041C4F20001884215D09B
:10A0B00045F6000107E047F60001C4F200018842BE
:10A0C0000CD048F20041C4F20001884206D04EF2A2
:10A0D000EE10C0F600006321F9F73CF96FF48050F0
:10A0E000054206D04EF2EE10C0F600006421F9F7EA
:10A0F00031F994F84100202803D194F84000012858
:10A1000001D10220B0BD242084F8410020680168FC
:10A1100021F001010160016821F4805101600168B2
:10A1200029430160016841F001010160202084F8A9
:0AA130004100002084F84000B0BD9B
:02A13A00FEE73E
:10A13C00B0B50446006847F2FF72C4F200029042C8
:10A14C000D4608DC45F20041C4F2000188420ED0F5
:10A15C0045F6000107E047F60001C4F20001884211
:10A16C0005D048F20041C4F2000188422BD1102DD9
:10A17C0006D34EF2EE10C0F600009221F9F7E4F887
:10A18C0094F84100202803D194F84000012801D113
:10A19C000220B0BD242084F841002068016821F021
:10A1AC0001010160016821F4706141EA052101603F
:10A1BC00016841F001010160202084F84100002079
:10A1CC0084F84000B0BD4EF2EE10C0F600009121B4
:0AA1DC00F9F7BAF8102DCCD2D2E743
:02A1E600FEE792
:10A1E80000285AD0B0B50446006843F20001C4F212
:10A1F8000001884206D04EF29E70C0F60000B521DC
:10A20800F9F7A4F86068072806D34EF29E70C0F6E6
:10A218000000B621F9F79AF8A068B0F5805F06D378
:10A228004EF29E70C0F60000B721F9F78FF8E0688B
:10A23800B0F5805F06D34EF29E70C0F60000B821DC
:10A24800F9F784F894E807004CF6CC43036045F22C
:10A258005553036041608260F9F700FA2168CA68C3
:10A26800520710D0054603E02168C86840070AD0A5
:10A27800F9F7F4F9401B3228F6D32068C068400784
:10A28800F2D00320B0BD0A69E068824206BF4AF6F0
:0EA29800AA20086008610020B0BD01207047B8
:02A2A600FEE7D1
:10A2A80001220168C0F8D022002280F8C822B1F843
:10A2B800540040F00100A1F85400B1F8540040F0F7
:0AA2C80002020020A1F854207047A4
:02A2D200FEE7A5
:10A2D40047F20000C4F20000016841F4807101609B
:02A2E4007047C1
:02A2E600FEE791
:10A2E80010B547F200040028C4F200043DD0B0F5D0
:10A2F800007F10D0B0F5806F06D04EF24F20C0F628
:10A3080000009D21F9F722F82068022161F34A2014
:10A318002060002010BD2068D4F8801000F4C060D0
:10A3280041F48071B0F5806FC4F88010F1D12068D5
:10A33800012161F34A20206041F28070C1F20000DF
:10A348000068322250434DF68362C4F21B32A0FBF0
:10A35800020201EB924000216369013841F10002D9
:10A368005B052BD5002AF7D128E02068D4F88010A7
:10A3780000F4C06021F48071B0F5806FC4F88010DB
:10A38800C7D12068012161F34A20206041F2807022
:10A39800C1F200000068322250434DF68362C4F2D5
:10A3A8001B32A0FB020201EB9240002163690138D5
:10A3B80041F100025B0501D5002AF7D1606940052B
:06A3C800A7D5032010BD23
:02A3CE00FEE7A8
:10A3D00047F20800C4F20000016841F480410160C6
:02A3E0007047C4
:02A3E200FEE794
:10A3E40000285CD02DE9F04182B00446006850B1E9
:10A3F40010F02F0007D14CF63210C0F6000040F2E6
:10A404004511F8F7A5FF207841F20006C007C4F211
:10A41400020646D12078800767D42078000700F12F
:10A42400A3802078400740F18D81A068052805D8D5
:10A43400012101FA00F010F0230F07D14CF632107D
:10A44400C0F600004FF4FA71F8F782FFB06D5FEACE
:10A45400C00808D4B06D40F08050B065B06D00F015
:10A4640080500190019847F20007C4F20007386851
:10A47400C00500F1CB80386840F480703860F9F78B
:10A48400EFF805463868C00500F1C080F9F7E8F830
:10A49400401B0228F6D9032002B0BDE8F081012058
:10A4A40070476068002818BFB0F5803F40F0A18075
:10A4B400B06800F00C01F068082978D0032281F01C
:10A4C4000C0122EA00000844B0FA80F040096ED181
:10A4D40065683068B5F5A02F00F0B580B5F5803F0C
:10A4E40040F0B88040F48030BAE0E06840F4807016
:10A4F400B0F5807F07D04CF63210C0F600004FF460
:10A50400C071F8F725FF2069802807D34CF6321074
:10A51400C0F6000040F28111F8F71AFFB068F16844
:10A5240000F00C0004284BD001F0030180F00C0073
:10A5340081F002010844B0FA80F0400940D1E1689A
:10A544003068002900F0A78040F480703060F9F78B
:10A5540087F805463068400500F1B280F9F780F8C5
:10A56400401B0228F6D9D6E06069022807D34CF6CE
:10A574003210C0F600004FF4E471F8F7E9FE6169A7
:10A58400D6F8940000294BD040F00100C6F894009E
:10A59400F9F766F8054600BFD6F8940080073FF542
:10A5A40040AFF9F75DF8401B0228F5D9B3E03068F5
:10A5B40080037FF52FAF606800287FF42BAF0DE197
:10A5C4003068400503D5E068002800F00781706812
:10A5D400216920F0FE4040EA0160706041F26C7035
:10A5E400C1F200000068F9F711F8002840F0F68085
:10A5F40013E7B0F5A02F3FF45BAF4CF63210C0F672
:10A60400000040F24B11F8F7A3FE51E7A568D6F815
:10A614009000052D5CD0012D63D140F0010068E06D
:10A6240020F00100C6F89400F9F71AF8054600BFB7
:10A63400D6F8940080077FF5F4AEF9F711F8401BC3
:10A644000228F5D967E040F480203060306840F497
:10A65400803005E020F480303060306820F48020C1
:10A664003060F8F7FDFF002D054610D030688003F8
:10A674003FF5D0AEF8F7F4FF401B6428F6D94AE062
:10A68400F8F7EEFF401B64284FF0030015D830683C
:10A694008003F5D4BEE620F480703060F8F7E0FF64
:10A6A400054600BF306840057FF5B7AEF8F7D8FF20
:10A6B400401B02284FF00300F4D902B0BDE8F0813A
:10A6C4007068216920F0FE4040EA01607060A4E6F1
:10A6D40040F00400C6F89000D6F8900040F0010065
:10A6E40007E020F00100C6F89000D6F8900020F0B2
:10A6F4000400C6F89000F8F7B3FF002D054641F2B8
:10A70400883714D0D6F89000800714D4F8F7A8FF3F
:10A71400401BB842F6D9032002B0BDE8F08100BF67
:10A72400F8F79EFF401BB8424FF00300C5D8D6F897
:10A7340090008007F4D4B8F1000F5EBFB06D20F034
:10A744008050B065207880064CD4E069032807D394
:10A754004CF63210C0F600004FF41971F8F7F8FD0A
:10A76400E069002800F02781B16801F00C010C2990
:10A774005CD1012832D0F068216A00F003028A42D9
:10A784002CD1626A6FF00F0300F0F00103EB0212A8
:10A79400914223D1A16A00F4FE4209028A421DD1EA
:10A7A400E16A00F07842C9068A4217D1226B00237D
:10A7B400CFF6E07303EA025200F4C001A2F50012DE
:10A7C40091420BD1616B4FF07E4202EA016100F0CD
:10A7D400C06001F17E41884200F0ED80012002B0AA
:10A7E400BDE8F081A069022807D34CF63210C0F608
:10A7F400000040F23B21F8F7ABFDA169D6F89800C0
:10A8040000296ED040F00100C6F89800F8F728FF40
:10A81400054600BFD6F89800800796D4F8F720FFC5
:10A82400401B02284FF00300F4D946E702286CD1FC
:10A83400206A032801D8012807D14CF63210C0F64B
:10A84400000040F26E21F8F783FD606A0138102899
:10A8540007D34CF63210C0F6000040F26F21F8F72F
:10A8640077FDA06A0838782807D34CF63210C0F672
:10A8740000004FF41C71F8F76BFDE06A02381E28E3
:10A8840007D34CF63210C0F6000040F27121F8F7FD
:10A894005FFD206B082800F29280012101FA00F08C
:10A8A40010F4AA7F00F08B80606B082800F290807F
:10A8B400012101FA00F010F4AA7F00F089803068C9
:10A8C40020F080703060F8F7CBFE054630688001D8
:10A8D4002DD5F8F7C5FE401B02284FF00300F5D92B
:10A8E400EBE620F00100C6F89800F8F7B9FE05463B
:10A8F400D6F8980080077FF528AFF8F7B1FE401B23
:10A9040002284FF00300F3D9D7E6306820F08070B6
:10A914003060F8F7A5FE04463068800144D5F8F7A6
:10A924009FFE001B02284FF00300F5D9C5E6F0682E
:10A9340048F20C01C0F29F1100EA010C04F120015D
:10A944008EC96FF00F00D4E90C5400EB0210002202
:10A95400CFF6E07241EA0C0102EA05520843A2F57F
:10A9640000124FF07E4540EA032005EA04651043D7
:10A9740005F17E4540EAC7602843F060306840F046
:10A9840080703060F06840F08070F060F8F768FE26
:10A994000446306880010ED4F8F762FE001B0228DA
:10A9A4004FF00300F5D988E6F0684FF6FC71CFF656
:10A9B400EE610840F060002002B0BDE8F0814CF682
:10A9C4003210C0F6000040F27221F8F7C1FC6BE7C8
:10A9D4004CF63210C0F6000040F27321F8F7B8FCD0
:02A9E4006DE71D
:02A9E600FEE78A
:10A9E8002DE9F047002800F03381044600680D4641
:10A9F8000F2802D810F00F0007D14CF63210C0F61D
:10AA0800000040F20B31F8F7A1FC102D07D34CF6EB
:10AA18003210C0F600004FF44371F8F797FC42F289
:10AA2800000AC4F2020ADAF8000000F00F008542BA
:10AA38000DD9DAF8000020F00F002843CAF800000A
:10AA4800DAF8000000F00F00A84240F001812078F9
:10AA580041F20808C007C4F202080CD14FF00009FF
:10AA68002068810759D4B9F1000F77D0D8F80000D1
:10AA780020F0F00070E060680138032807D34CF636
:10AA88003210C0F6000040F22331F8F75FFC61682D
:10AA980058F8080C022900F0D980032940F0DB801F
:10AAA800800140F1D580D8F80400D8F8041000F0EF
:10AAB8000300032842F20040C1F30311C0F2F4007E
:10AAC800D8F8042001F1010104BF47F64000C0F2A4
:10AAD8007D10B0FBF1F0D8F80410C2F30622504301
:10AAE800C1F34161022202EB4101B0FBF1F04BF2EC
:10AAF8000041C0F2C44188420CD9D8F8000010F0D7
:10AB0800F00F00F0B3802078800703D5A0680028F4
:10AB180000F0AC804FF00009B1E0410742BFD8F81F
:10AB2800001041F4E061C8F80010000706D5D8F815
:10AB38000000072161F30D20C8F80000A0686FF03D
:10AB4800070101EB3011082980F0B780D8F8000020
:10AB5800A16820F0F0000843C8F80000DAF8000007
:10AB680000F00F00854219D2DAF8000020F00F003B
:10AB78002843CAF80000F8F771FD064641F2883705
:10AB8800DAF8000000F00F00A84207D0F8F766FDD9
:10AB9800801BB842F4D90320BDE8F087207840072D
:10ABA80019D5E0686FF0030101EB302104290AD3BD
:10ABB8004FEA302038B14CF63210C0F600004FF49E
:10ABC8006771F8F7C3FBD8F80000E16820F4E0608B
:10ABD8000843C8F80000207800071AD520696FF0EC
:10ABE800030101EB302104290AD34FEA302038B1A0
:10ABF8004CF63210C0F6000040F2A331F8F7A6FB7D
:10AC0800D8F80000216920F4605040EAC100C8F873
:10AC18000000F9F7CFFCD8F800104FF26C02C1F32E
:10AC28000311C0F60002515C41F2807201F01F016D
:10AC380020FA01F141F26C70C1F200000068C1F223
:10AC480000021160BDE8F047F8F7DEBC800304D4C9
:10AC58000120BDE8F0874005FAD5F9F7ABFC4BF2C7
:10AC68000041C0F2C44188427FF654AFD8F80000D2
:10AC7800082161F307104FF00109C8F80000D8F85F
:10AC88000000616820F003000843C8F80000F8F7E6
:10AC9800E5FC064641F28837D8F80000616800F004
:10ACA8000C00890088423FF4DBAEF8F7D7FC801B24
:10ACB800B842F1D90320BDE8F0874FEA30100028E8
:10ACC8003FF444AF4CF63210C0F6000040F27A313F
:06ACD800F8F73CFB3AE72F
:02ACDE00FEE78F
:10ACE00041F2807041F20801C1F20000C4F2020199
:10ACF000006809684FF27C02C1F30221C0F600022D
:0AAD0000515C01F01F01C8407047CC
:02AD0A00FEE762
:10AD0C0041F2807041F20801C1F20000C4F202016C
:10AD1C00006809684FF27C02C1F3C221C0F6000240
:0AAD2C00515C01F01F01C8407047A0
:02AD3600FEE736
:10AD380088B310B50446406840F04000402807D06A
:10AD48004CF6D610C0F6000040F23511F8F7FEFABE
:10AD5800A068802807D34CF6D610C0F600004FF440
:10AD68009B71F8F7F3FAE068B0F5004F07D34CF69B
:10AD7800D610C0F6000040F23711F8F7E7FA20695C
:10AD8800B0F5800F09DB14D0B0F5C00F11D0B0F1C9
:10AD9800806F0ED005E00120704750B1B0F5001F5C
:10ADA80007D04CF6D610C0F600004FF49C71F8F7A7
:10ADB800CDFA606940F00040B0F1004F07D04CF682
:10ADC800D610C0F6000040F23911F8F7BFFAA069B2
:10ADD80040F48010B0F5801F07D04CF6D610C0F6AE
:10ADE80000004FF49D71F8F7B1FAE06940F0804037
:10ADF800B0F1804F07D04CF6D610C0F6000040F2F4
:10AE08003B11F8F7A3FA206A40F00050B0F1005F58
:10AE180007D04CF6D610C0F600004FF49E71F8F734
:10AE280095FA94F8250028B9002084F824002046D3
:10AE3800F8F794FA022084F825002068C168C9064A
:10AE48000CD4CA214162532141622046F9F7BAFE67
:10AE580058B108B32168FF224A6200E000200028A8
:10AE680004BF012184F8251010BD94E803508269BD
:10AE780022F08E6222F04002826122691143A269A7
:10AE880083691143194381614EEA0C4101612046EF
:10AE980000F012F80028DDD12168D4F814C0D4E9F4
:10AEA80007E28B6923F060431A4342EA0E0242EA42
:06AEB8000C028A61CEE7E6
:02AEBE00FEE7AD
:10AEC00010B504460068C16821F08001C160816945
:10AED000890609D42046F9F79FFE00280EBF0020FE
:10AEE000032084F8250010BD816921F020018161D3
:10AEF0002046F9F791FE00281ABF032084F82500A8
:0EAF0000002021688A6942F020028A6110BD9B
:02AF0E00FEE75C
:10AF100010B50C46202907D34EF67430C0F6000059
:10AF200040F2FC71F8F716FA42F20050C4F2000049
:06AF300050F8240010BDE2
:02AF3600FEE734
:10AF3800A8B1B0B50446006842F6FF71C4F2010139
:10AF480088420EDC43F60001C4F2000188421CD09E
:10AF580043F60041C4F20001884216D00DE00120FA
:10AF6800704743F20001C4F2010188420DD043F654
:10AF78000041C4F20101884207D04CF64620C0F6D1
:10AF8800000040F24711F8F7E1F9606850B1B0F5F8
:10AF9800827F07D04CF64620C0F600004FF4A4711B
:10AFA800F8F7D4F9A068002818BFB0F5806F40F012
:10AFB8008680E068A0F540704FEA30200D2807D35E
:10AFC8004CF64620C0F600004FF4A571F8F7BEF91C
:10AFD800A069002818BFB0F5007F7DD1606B40F0F4
:10AFE8000800082807D04CF64620C0F600004FF4A9
:10AFF800A671F8F7ABF9E0694FEAF000082807D323
:10B008004CF64620C0F6000040F24D11F8F79EF9C4
:10B01800206A40F08000802807D04CF64620C0F611
:10B0280000004FF4A771F8F791F9606A40F010003A
:10B03800102807D04CF64620C0F6000040F24F1109
:10B04800F8F784F9606A80B1E0694FEAF0000828EF
:10B0580007D34CF64620C0F6000040F26111F8F71D
:10B0680075F90020C4E9040045E0206940F00200B9
:10B07800022807D04CF64620C0F600004FF4A9710C
:10B08800F8F764F96069022807D34CF64620C0F641
:10B09800000040F25311F8F759F96068B0F5827F63
:10B0A80027D1E0694FEAF000082824D34CF646205F
:10B0B800C0F6000040F25711F8F748F91BE0B0F568
:10B0C800004F3FF476AF4CF64620C0F6000040F241
:10B0D8004911F8F73BF96CE7B0F5802F3FF47EAFE4
:10B0E8004CF64620C0F6000040F24B11F8F72EF956
:10B0F80074E70020E0610025A56294F85D0020B99E
:10B10800204684F85C50FBF787FF022084F85D0036
:10B118002068D4F80CE00268BEF5E06F22F0400227
:10B1280002604EF4006298BF0125B2F5706F1CBF33
:10B138000023A3624FEA053CD4E90135D4E9042190
:10B1480003F4827305F404452B4402F002021A4406
:10B15800A36901F00101E569114403F40072114487
:10B1680005F03802256A114405F08002A56A1144E9
:10B1780005F40052114301600421626A0EF47065FF
:10B1880001EA1341636B45EA0C0502F010022943FA
:10B1980003F00803114319434160C16921F40061B8
:0EB1A800C16100200121206684F85D10B0BD59
:02B1B600FEE7B2
:10B1B80070B515460E464FF4C05132462B4604462C
:10B1C800F9F796FE68B9204631462A46F9F704FF92
:10B1D80038B920464FF4C06132462B46F9F788FE4D
:10B1E80028B1206E40F020002066032070BD0020AA
:02B1F80070BD28
:02B1FA00FEE76E
:10B1FC0010B5002853D00446006844F6FF71C4F221
:10B20C000001884212DC44F20041C4F20001884281
:10B21C002BD044F60001C4F20001884225D044F63C
:10B22C000041C4F2000188421FD011E045F2000138
:10B23C00C4F20001884218D048F20001C4F20001A7
:10B24C00884212D043F60001C4F2010188420CD0AE
:10B25C00A0694FF49F7100284EF2FD70C0F60000FB
:10B26C0008BF40F24311F8F76FF8D4F8880028B9FA
:10B27C00002084F884002046FBF734FF2420C4F817
:10B28C0088002068A16A026822F00102026011B1F4
:10B29C00204600F019F82046F9F7F6FE08B1012017
:10B2AC0010BD2168486820F490404860886820F000
:10B2BC002A008860086840F0010220460A60BDE858
:06B2CC00104000F01FB964
:02B2D200FEE795
:10B2D40010B50446806AB0F5807F07D34EF2FD7046
:10B2E400C0F6000040F6AE41F8F732F894F82800B2
:10B2F400000714D5A06B40F40040B0F5004F07D010
:10B304004EF2FD70C0F6000040F6B341F8F720F8A5
:10B314002068A16B426822F400421143416094F812
:10B324002800C00714D0E06A40F40030B0F5003FB4
:10B3340007D04EF2FD70C0F6000040F6BA41F8F7AF
:10B3440007F82068E16A426822F400321143416040
:10B3540094F82800800714D5206B40F48030B0F5B1
:10B36400803F07D04EF2FD70C0F6000040F6C141A8
:10B37400F7F7EEFF2068216B426822F48032114314
:10B38400416094F82800400714D5606B40F4802095
:10B39400B0F5802F07D04EF2FD70C0F6000040F6E5
:10B3A400C841F7F7D5FF2068616B426822F4802218
:10B3B4001143416094F82800C00614D5E06B40F4B2
:10B3C4008050B0F5805F07D04EF2FD70C0F60000EB
:10B3D40040F6CF41F7F7BCFF2068E16B826822F4A6
:10B3E40080521143816094F82800800614D5206CA3
:10B3F40040F40050B0F5005F07D04EF2FD70C0F687
:10B40400000040F6D641F7F7A3FF2068216C82685C
:10B4140022F400521143816094F8280040065AD562
:10B42400206844F6FF31C4F20001884212DD44F67C
:10B434000041C4F20001884220D045F20001C4F268
:10B44400000188421AD043F60001C4F20101884287
:10B4540014D00BE044F20041C4F2000188420DD044
:10B4640044F60001C4F20001884207D04EF2FD7098
:10B47400C0F6000040F6DD41F7F76AFF606C40F467
:10B484008010B0F5801F07D04EF2FD70C0F60000AA
:10B4940040F6DE41F7F75CFF2068616C4268B1F565
:10B4A400801F22F4801242EA0102426013D1A06C90
:10B4B4004FEA7050042807D34EF2FD70C0F6000026
:10B4C40040F6E341F7F744FF2068A16C426822F498
:10B4D400C0021143416094F82800000614D5E06CC2
:10B4E40040F40020B0F5002F07D04EF2FD70C0F6F6
:10B4F400000040F6EB41F7F72BFF2068E16C42684F
:0AB5040022F400221143416010BD43
:02B50E00FEE756
:10B51000B0B582B004460020C4F89000F8F7A2F855
:10B5200021680546096809071AD56FF07E4C204648
:10B530004FF4001100222B46CDF800C0F9F794FF1C
:10B5400070B100BF206850E8000F216820F0800033
:10B5500041E80002002AF5D103202021882232E0B0
:10B5600020680068400725D56FF07E4C20464FF4D8
:10B57000800100222B46CDF800C0F9F775FFC8B155
:10B58000206850E8000F216820F4907041E8000224
:10B59000002AF5D12068083050E8000F216820F01B
:10B5A0000100083141E80002002AF3D103202021E4
:10B5B0008C2208E02020C4F88800C4F88C00002108
:10B5C00070220020E166A150002184F8841002B0AE
:02B5D000B0BD0C
:02B5D200FEE792
:10B5D400D0F88830202B09D1944600294FF001027D
:10B5E40018BFBCF1000F04D1104670470222104668
:10B5F4007047B0B5002221230165A0F854C0A0F81B
:10B6040056C0C0F89020C0F88830C36F13B34BF213
:10B61400DD65C0F600054BF285644BF2C96E5D63CF
:10B624000568C0F60004C0F6000EC3E90B4E9A6329
:10B6340005F12802044618466346FDF7D1FC01468D
:10B64400204639B11021C0F890102021C0F888108C
:10B65400012210E0016840220A6200BF016808313B
:10B6640051E8001F026841F08001083242E80013EB
:0EB67400002BF3D10022BDE8B0401046704715
:02B68200FEE7E1
:10B684000168806A0968890619D40021A0F8561057
:10B694000168083151E8001F026821F08001083276
:10B6A40042E80013002BF3D1016851E8001F02683F
:10B6B40041F0400142E80013002BF5D17047FAF73E
:02B6C40013BDB4
:02B6C60043003F
:06B6C800806A00F069BA7F
:0EB6CE0041F27471C1F20001096800F029B860
:10B6DC00B0B5846A2168D4F88800D4F88C50896895
:10B6EC00090607D5212805D10020A4F856002046CC
:10B6FC00F9F78CFF20688068400607D5222D05D10C
:10B70C000020A4F85E00204600F01CF8D4F890004D
:10B71C0040F010012046C4F89010BDE8B040FAF794
:02B72C007DBCE2
:10B72E0080B50B468DF803000DF1030001210122B7
:10B73E0000F000FA9DF80310002808BF411E0846CD
:02B74E0008BD34
:10B75000016851E8001F026821F4907142E800136B
:10B76000002BF5D14FF6FE7CCEF6FF7C0268083246
:10B7700052E8002F036802EA0C02083343E8002174
:10B780000029F3D1C16E01290AD100BF016851E837
:10B79000001F026821F0100142E80013002BF5D1D0
:0EB7A0002021C0F88C100021C166416770475F
:10B7AE0038B541F27471C1F2000104460D6802F021
:10B7BE00F8FE02462846214600F0C2FA013004D0B7
:0EB7CE000A20BDE83840FFF77BBFC04338BDFE
:10B7DC0070B5046840F62F03E2692168A66813402F
:10B7EC00202B05D101F0200306F080555B1936D1D2
:10B7FC0040F60F0313400CD00123C1F2000306EAFC
:10B80C00030C40F22013C0F200430B4013EB0C036B
:10B81C002BD1C36ED50616D5012B14D111F0100304
:10B82C0011D010212162A168490600F1AA80B0F85C
:10B83C005C10B0F85E20B0F85E30002B18BF91425F
:10B84C0040F0358170BDD30278D516F4800375D0E5
:10B85C004FF480112162BDE8704000F08DBA416F49
:10B86C000029EFD0BDE870400847D30718BF11F48A
:10B87C00807307D001232362D0F8903043F001038A
:10B88C00C0F89030930706F0010E0AD5BEF1000FF8
:10B89C0007D002232362D0F8903043F00403C0F8A1
:10B8AC00903053070AD5BEF1000F07D00423236252
:10B8BC00D0F8903043F00203C0F8903013070CD549
:10B8CC0001F0200353EA0C0307D008232362D0F8BD
:10B8DC00903043F00803C0F8903013050BD511F0ED
:10B8EC00806308D04FF400632362D0F8903043F0AB
:10B8FC002003C0F89030D0F89030002BA2D09206E4
:10B90C000AD501F0200106F08052891804D0416F4D
:10B91C0011B10446884720460168D0F89020896808
:10B92C0002F0280201F040010446891840F08A8098
:10B93C00FAF774FB0020C4F8900070BD130606D50E
:10B94C0001F0800306F400069B1940F0E2805306D8
:10B95C0040F1A48011F0400300F0A080016851E890
:10B96C00001F026821F0400142E80013002BF5D1C2
:10B97C002021C0F8881000218167BDE87040FAF7DB
:10B98C00AFBBD0F880100A6851688BB2002B4ED038
:10B99C00B0F85C60B3424AD2A0F85E101168890618
:10B9AC0039D400BF016851E8001F026821F480718E
:10B9BC0042E80013002BF5D10168083151E8001F53
:10B9CC00026821F00101083242E80013002BF3D188
:10B9DC000168083151E8001F026821F0400108326B
:10B9EC0042E80013002BF3D12021C0F88C10002169
:10B9FC00C16600BF016851E8001F026821F0100108
:10BA0C0042E80013002BF5D1D0F88010044608460C
:10BA1C00FDF73EFB204602210167B0F85C10B0F840
:10BA2C005E20891A89B2BDE8704000F09BB8B0F86E
:10BA3C005C1099427FF406AF126892067FF502AF54
:10BA4C00022261E0FFF77EFE2168204689684906E4
:10BA5C0020D500BF0168083151E8001F026821F0B1
:10BA6C004001083242E80013002BF3D1D0F88010CB
:10BA7C0081B145F24D60C0F6000088630846FDF7C1
:10BA8C003FFB00283FF4DEAED4F88000816BBDE8AC
:10BA9C0070400847BDE87040FAF7C0BA13023FD5B2
:10BAAC0011F080433CD0BDE8704000F0ADB9891A6C
:10BABC00026852E8002F036822F4907243E80026D3
:10BACC00002EF5D14FF6FE72CEF6FF7203680833E6
:10BADC0053E8003F06681340083646E80035002D51
:10BAEC00F4D12022C0F88C200022C266426700BF2D
:10BAFC00026852E8002F036822F0100243E8002687
:10BB0C00002EF5D1022289B20267BDE8704000F028
:10BB1C0029B8816F00293FF495AEBDE87040084705
:10BB2C00D2017FF58FAEB1F1FF3F3FF78BAEBDE891
:06BB3C00704000F04DB95D
:10BB4200F8B51D4617460C460646184602F091FC0B
:10BB5200002803D407FB04F2A24201D20020F8BD60
:0EBB62002846314600F0F2F8B0FBF4F0F8BDD2
:02BB700070471C
:10BB720052EC10CBC2F30A5340F2FF718B4218BF52
:10BB8200002B02D100210160704740F2FE3161F3C7
:0EBB92001E52A3F2FE31016042EC10CB704750
:02BBA0007047EC
:10BBA2002DE9F8432DED028B8E1E00EBC6070D46E4
:10BBB20097ED008BD7E9022359EC108B404649469A
:10BBC200FAF73DFC53EC182B01F097FC032D41ECE6
:10BBD200100B12D3741E17ED028B083F53EC102B7F
:10BBE20040464946FAF72BFC53EC182B01F085FC32
:10BBF200012E41EC100B2646ECD853EC102B40469C
:10BC02004946FAF71CFC41EC100BBDEC028BBDE877
:02BC1200F883B5
:02BC1400704777
:10BC16002DE9F8430F46804600EBC10256EC109B17
:10BC26007C1EA2F1080552E9022351EC100B01F02B
:10BC360062FC4A463346FAF700FC022F41EC100B31
:10BC46002A462746ECD8D8E9002301F054FC41ECFB
:06BC5600100BBDE8F883AD
:02BC5C0070472F
:10BC5E0042694AB110B50446036A002B1CBF216924
:0ABC6E0098470020606110BD704788
:10BC7800026848F20003C4F200039A4218D0B0B533
:10BC8800B1F1807F0CD34EF2FD72C0F6000204467B
:10BC980010460D4640F6AF21F7F758FB29462046D7
:10BCA8000068426902F07F4211434161BDE8B0403B
:02BCB8007047D3
:0ABCBA00436A08460121FFF73FBF6F
:10BCC4000168806A0968890634D40021A0F85E10EE
:10BCD400016851E8001F026821F4807142E80013F2
:10BCE400002BF5D10168083151E8001F026821F0EA
:10BCF4000101083242E80013002BF3D10168083136
:10BD040051E8001F026821F04001083242E80013A4
:10BD1400002BF3D12021C0F88C10C16E012909D168
:10BD2400016851E8001F026821F0100142E8001385
:10BD3400002BF5D100210167C16E012903D1B0F8B0
:0ABD44005C10FFF713BFFFF763BFA9
:06BD4E00006800F045B89A
:10BD5400806A01210167C16E012904D1B0F85C1029
:0ABD64004908FFF703BFFFF777BFA0
:10BD6E000146C0680A6982426FEA000010449CBF17
:06BD7E00896808447047CB
:02BD8400704706
:10BD86002DE9F843144688460546C7684FF0000972
:10BD96002869F943B8420844A96898BF0844CE1BED
:10BDA600B04238BF06466868A64228BF26463844D1
:10BDB60041463246FAF775FCA868F1190F1A18BF02
:10BDC6000F46A41BB144B044BFF35F8FEF60DFD1D1
:06BDD6004846BDE8F883B9
:02BDDC007047AE
:10BDDE00F8B540F6E413C1F2000314461B78002BAD
:10BDEE000D46064608BF02F05CFBEFF311874FF0DD
:10BDFE00200181F3118830462946224602F0A5FB28
:06BE0E0087F31188F8BD66
:02BE1400704775
:10BE160084460020002918BF002A0ED0097848B2AF
:10BE260000280BD4BCF1000F18BFCCF8001000217D
:10BE3600C3E90011002818BF012070476FF0010008
:02BE4600704743
:10BE480010B5016844F6FF72C4F20002914212DC98
:10BE580044F20042C4F20002914229D044F60002A2
:10BE6800C4F20002914223D044F60042C4F2000218
:10BE780091421DD011E045F20002C4F20002914245
:10BE880016D048F20002C4F20002914210D043F6E4
:10BE98000002C4F2010291420AD04CF6DA21C0F63F
:10BEA80000010446084640F23621F7F74FFA2046CB
:10BEB80090F88410012901D1022010BD2421C0F876
:10BEC800881001680A680B6822F0005223F0010309
:10BED8000B60002343660A602021C0F8881080F8B0
:06BEE8008430002010BDB3
:0EBEEE007F298EBF6FF00100017001207047A8
:10BEFC0001460120A1F8400000220020A1F84020BA
:0ABF0C00A1F84420A1F8502070476E
:10BF160053797374656D20636F726520636C6F630C
:0ABF26006B3A2025754D487A0A0099
:10BF30002DE9F04182B00DF105060C464FF02208C4
:10BF40004FF47A7731463246032305468DF8058053
:10BF50000097F8F78DFE9DF80700314600F00700C6
:10BF600020438DF8060042208DF805002846324611
:10BF700002230097F8F77CFE284631463246032319
:10BF80008DF805800097F8F773FE9DF807002040B4
:10BF9000A04202D102B0BDE8F0814EF6F200C0F638
:0ABFA0000000FFF704FC00BFFEE7FD
:10BFAA004261636B75705265676973746572446147
:0EBFBA00746120617661696C61626C650D00D6
:10BFC8000246D0F8880100219067B2F8CE00A2F8A6
:10BFD8007C00B2F8CC00A2F87E00D2F8D43040F24F
:0EBFE8000000C1F20000C2F8803000F06DBB16
:10BFF6002E2E2E466C61736820756E6C6F636B65B2
:02C006006400D4
:10C008000246D0F8D4004FF47A73C2F88400D2F80C
:10C018008400D2F88010401A41F2DC21C1F20001FC
:10C028000968594391FBF0F340F20000C1F20000A7
:0AC038000021C2F8883000F047BB79
:10C04200466C617368206F6220756E6C6F636B2043
:06C052006572726F7200BE
:10C0580040F20000C1F20000C16D4FF2F012CFF6BD
:10C06800FF725143CB17C0E95813C16D4942C0F85C
:10C078004011C16D5143CA17C0E97812C16D4942D8
:06C08800C0F8D81170475A
:0EC08E00466C61736820206C6F636B65640004
:10C09C00824202D1002000B2704794469042B8BF51
:10C0AC000246BCEB00009C4648BF404280B5DDF820
:10C0BC0008E09942B8BF0B46BCEB010148BF4942AE
:10C0CC00AEEB0202434301FB023191FBF0F0BDE801
:06C0DC00804000B2704735
:10C0E200443A5C50726F6A656B74655C6563735346
:10C0F2006D61727450726F5C7472756E6B5C667790
:10C102005F673437337263745C4472697665727345
:10C112005C53544D3332473478785F48414C5F4426
:10C1220072697665725C5372635C73746D333267E5
:0AC132003478785F68616C2E6300BA
:10C13C00B0B504464EF67840C0F60000FFF731FB70
:10C14C0040F2F835C1F2000541F2407105F11800DA
:10C15C00C0F60001B822FAF7B0FAA868D021013075
:10C16C00C5E9011001202870002000212A46D023A7
:0EC17C0000F034F82046BDE8B04000F097B85F
:10C18A00443A5C50726F6A656B74655C656373539D
:10C19A006D61727450726F5C7472756E6B5C6677E7
:10C1AA005F673437337263745C447269766572739D
:10C1BA005C53544D3332473478785F48414C5F447E
:10C1CA0072697665725C5372635C73746D3332673D
:0EC1DA003478785F68616C5F6164632E630087
:10C1E8002DE9F04F83B0924606465818012241F2D5
:10C1F800F0181F4602EB901B0025C1F2000800BF93
:10C208008AB212FA87F23C4641EA8610402A28BFD1
:10C21800C1F140041AFA85F1A2B21FFA85F9CDE9F5
:10C22800001282B24046A02102234FF47A7502958B
:10C23800F7F7B0FF052001363F1B19FA84F5F7F729
:10C2480013FABBF1010B4FF00001D9D103B0BDE8DF
:02C25800F08F65
:10C25A00443A5C50726F6A656B74655C65637353CC
:10C26A006D61727450726F5C7472756E6B5C667716
:10C27A005F673437337263745C44726976657273CC
:10C28A005C53544D3332473478785F48414C5F44AD
:10C29A0072697665725C5372635C73746D3332676C
:0EC2AA003478785F68616C5F6372632E6300A6
:10C2B800F0B581B040F2F834C1F200040546002020
:10C2C80000212246D023F9F76FFEA0692861A08BD0
:10C2D800A882E08BE882208C2883608CA883A08CBD
:10C2E800E883E08C2884208D6884608DA5F87C0024
:10C2F800A08DA5F87E00E08DA5F89800208EA5F801
:10C308009A00608EA5F88C00A08EA5F8A000E08E9B
:10C31800A5F8A80004F1380090E80F50D4E9146794
:10C32800C5F88000C5F88410C5F88820C5F8903095
:10C33800C5F89CC0C5F8A4E0C5F8AC60AF6704F1C7
:10C34800580007C8C5F89400C5F8B010C5F8B4205F
:10C35800B4F88800A5F85200B4F88A00A5F850008F
:10C36800D4F88C00E865D4F890002866B4F89400F6
:10C37800A5F85400B4F89600A5F85600B4F898004B
:10C38800A5F85800B4F89A00A5F85A00B4F89C002B
:10C39800A5F86400B4F89E00A5F86800B4F8A000F9
:10C3A800A886B4F8A200E886B4F8A4002887B4F8F0
:10C3B800A6006887B4F8A800A887B4F8AA00E88798
:10C3C800B4F8AC00A5F84000B4F8AE00A5F84200F7
:10C3D800B4F8B000A5F84400B4F8B200A5F84600D7
:10C3E800B4F8B400A5F84800B4F8B600A5F84A00B7
:10C3F800B4F8B800A5F84C00B4F8BA00A5F84E0097
:10C40800B4F8BC00A5F86A00B4F8BE00A5F86C0042
:10C41800B4F8C000A5F86E00B4F8C200A5F8700022
:10C42800B4F8C400A5F87200B4F8C600A5F8B800BE
:10C43800B4F8C800A5F8BA00B4F8CA00A5F8BC005A
:10C44800B4F8CC00A5F8BE00B4F8CE00A5F8C0003A
:10C45800E0686860A088E188227880F0D00089B21E
:10C468000843D1B281F00101084318BF012001B08F
:02C47800F0BD15
:10C47A00443A5C50726F6A656B74655C65637353AA
:10C48A006D61727450726F5C7472756E6B5C6677F4
:10C49A005F673437337263745C44726976657273AA
:10C4AA005C53544D3332473478785F48414C5F448B
:10C4BA0072697665725C5372635C73746D3332674A
:0EC4CA003478785F68616C5F646D612E63008A
:10C4D800F0B581B004464EF6F510C0F60000FFF73F
:10C4E80062F92046FFF7E4FEB4F87C0040F2F83227
:10C4F800C1F200025085B4F87E009085D4F880C05F
:10C50800D4F88410D4F88830B4F88C005086D4F865
:10C518009000D4F878E0D4F89450D4F8B060D4F807
:10C52800B4709565D6651766B4F89850D585B4F893
:10C538009A501586D4F89C50B4F8A0609686D4F822
:10C54800A460B4F8A870D786D4F8AC70C2E91030EB
:10C5580002F14800C2E90EC180E8E0404FF496407D
:10C568004FF48031C2E906010021C2F82610C2F852
:10C57800221040F2DE31A2F8881047F20011C0F212
:10C5880002014FF4FA13C2E923130A21A2F8941006
:10C598006921A2F88A100221C6F66051C2F89610E5
:10C5A80046F2E001A2F89A100121C0F2020145F614
:10C5B800C05347F2A03702F19C0CC6F2A813C6F686
:10C5C80060578CE88A004FF25421CFF6FF7101F5CD
:10C5D8007A7301F5FA71A2F8BA103221A2F8B030D4
:10C5E8004FF63003A2F8BC104FF63001C1F2707359
:10C5F800CFF6FF71C2F8B23041F27C5301F5E16128
:10C608004FF6837641F27075CFF25423A2F8BE102C
:10C6180044F62061C0F27D06C1F27C55C2F8B630FE
:10C62800C0F2070140F28433012702F1C00C012057
:10C63800C2E92A65C0F20103C6F6402764268CE8E1
:10C648008A00D0211084C2F8CC6051601070107438
:10C6580060680021D0600020D023FFF7C1FD20468C
:0AC6680001B0BDE8F040FFF723BE6B
:10C67200443A5C50726F6A656B74655C65637353B0
:10C682006D61727450726F5C7472756E6B5C6677FA
:10C692005F673437337263745C44726976657273B0
:10C6A2005C53544D3332473478785F48414C5F4491
:10C6B20072697665725C5372635C73746D33326750
:0EC6C2003478785F68616C5F6932632E6300C4
:10C6D0002DE9F04104464EF68D40C0F60000884634
:10C6E000FFF765F8206940F2F836C1F20006B06144
:10C6F000A08AB8F1000FB083E08AF083208B3084E9
:10C70000A08B7084E08BB084208CF084608C3085AA
:10C71000B4F87E00B085B4F87C007085B4F8980059
:10C72000F085B4F89A003086B4F88C007086B4F8BE
:10C73000A000B086B4F8A800F086D4F88000D4F841
:10C740008410D4F88820D4F89030D4F89C50D4F8D1
:10C75000A470D4F8ACC0D4F878E0B063F16332646C
:10C760007364B564F764C6F850C0C6F854E0D4F8F2
:10C77000940006F15803D4F8B010D4F8B42007C3DD
:10C78000B4F85200A6F88800B4F85000A6F88A0061
:10C79000E06DC6F88C00206EC6F89000B4F8540026
:10C7A000A6F89400B4F85600A6F89600B4F858001D
:10C7B000A6F89800B4F85A00A6F89A00B4F86400F5
:10C7C000A6F89C00B4F86800A6F89E00A08EA6F813
:10C7D000A000E08EA6F8A200208FA6F8A400608F2B
:10C7E000A6F8A600A08FA6F8A800E08FA6F8AA00D9
:10C7F000B4F84000A6F8AC00B4F84200A6F8AE00C9
:10C80000B4F84400A6F8B000B4F84600A6F8B200A8
:10C81000B4F84800A6F8B400B4F84A00A6F8B60088
:10C82000B4F84C00A6F8B800B4F84E00A6F8BA0068
:10C83000B4F86A00A6F8BC00B4F86C00A6F8BE0014
:10C84000B4F86E00A6F8C000B4F87000A6F8C200F4
:10C85000B4F87200A6F8C400B4F8B800A6F8C60090
:10C86000B4F8BA00A6F8C800B4F8BC00A6F8CA002C
:10C87000B4F8BE00A6F8CC00B4F8C000B168A6F8C1
:10C88000CE0001F101004FF0D001C6E901104FF0D8
:10C890000100307007D04EF6C070C0F60000FEF701
:10C8A00086FF6068F06040F2F832C1F200020020BA
:10C8B0000021D023FFF798FC2046BDE8F041FFF7A8
:02C8C000FBBCBF
:10C8C200443A5C50726F6A656B74655C656373535E
:10C8D2006D61727450726F5C7472756E6B5C6677A8
:10C8E2005F673437337263745C447269766572735E
:10C8F2005C53544D3332473478785F48414C5F443F
:10C9020072697665725C5372635C73746D333267FD
:0EC912003478785F68616C5F7063642E630038
:10C9200040F20001A0F50040C1F20001C1F8B000E2
:02C9300070474E
:10C93200443A5C50726F6A656B74655C65637353ED
:10C942006D61727450726F5C7472756E6B5C667737
:10C952005F673437337263745C44726976657273ED
:10C962005C53544D3332473478785F48414C5F44CE
:10C9720072697665725C5372635C73746D3332678D
:0EC982003478785F68616C5F7263632E6300C7
:10C9900010B582B09C460446ACF10300134610F17A
:10C9A000020F4FF009000A46049938BF4FF0010CFE
:10C9B000022B38BF0A2000EB0C0E2046CDE900CE3A
:10C9C000F5F79EF90020A08484F82600E061C4F801
:06C9D0001F0002B010BDC3
:10C9D600443A5C50726F6A656B74655C6563735349
:10C9E6006D61727450726F5C7472756E6B5C667793
:10C9F6005F673437337263745C4472697665727349
:10CA06005C53544D3332473478785F48414C5F4429
:10CA160072697665725C5372635C73746D333267E8
:0ECA26003478785F68616C5F7274632E630011
:10CA3400B0B50C460546F9F76BFB0146A01C29531B
:02CA4400B0BD83
:10CA4600443A5C50726F6A656B74655C65637353D8
:10CA56006D61727450726F5C7472756E6B5C667722
:10CA66005F673437337263745C44726976657273D8
:10CA76005C53544D3332473478785F48414C5F44B9
:10CA860072697665725C5372635C73746D33326778
:0ECA96003478785F68616C5F7370692E63009E
:10CAA400B0B5044610F8275FD0F8011205290DD35C
:10CAB400F9F74CFB013009D035B140F20000C1F266
:10CAC4000000008BA84201D10220B0BD0020C4F8B0
:06CAD40028022075B0BD30
:10CADA00443A5C50726F6A656B74655C6563735344
:10CAEA006D61727450726F5C7472756E6B5C66778E
:10CAFA005F673437337263745C4472697665727344
:10CB0A005C53544D3332473478785F48414C5F4424
:10CB1A0072697665725C5372635C73746D333267E3
:10CB2A003478785F68616C5F756172745F65782EBE
:02CB3A00630096
:10CB3C0070B5014611F8273F002600F22715044670
:10CB4C00C0F82C6280F827312846012200F016F834
:10CB5C0001462846FFF768FFC4F82C022046F9F777
:0ACB6C00C7FAC4F82862267570BDF0
:10CB76002D2D2D204761696E202043414C202D2DFF
:02CB86002D0080
:10CB880091F801C0BCF1100F09D0BCF1060F04D018
:10CB9800BCF1030F05D100F011B8F9F7E5BAF9F7C0
:10CBA80013BB8CF08001831881540121901C5970AB
:02CBB8007047C4
:0ACBBA0054736869703D25660A0097
:10CBC4002DE9F04140F2000CC1F2000C002BBCF83E
:10CBD400187018BF9F420CD10B794E7946EA032393
:10CBE400A3F17E0717F17E0F07D883218154032117
:10CBF40014E0862181540B2110E091F80280CD7855
:10CC040045EA082103EB010EAEF2FD1717F5FE7F8E
:10CC140000EB020707D283213970022110444170CE
:10CC2400901CBDE8F08103243C7074007C708BB1CF
:10CC34004FEA482343EA45036344013313F8027B74
:10CC44008618B77013F8037C0131714502F10202B2
:0ACC5400F770F3D3901CBDE8F081E7
:10CC5E002D2D2D204761696E202043414C20454EDD
:06CC6E0044452D2D2D00B0
:10CC740040F20000C1F200004FF0FF31A0F80611AD
:06CC8400A0F80411704746
:0ECC8A0064656C746120543D256620430A00E9
:10CC980070B540F20004C1F20004B4F8740041F227
:10CCA8003035C1F2000598B1B4F8740001281ABFF4
:10CCB800B4F874000022012240F20040C4F60000DB
:10CCC8004FF40061F7F782F9B4F87400288070BD5A
:10CCD800288800284FF6FF7018BFA4F80601B4F89A
:10CCE800061119B1B4F80611814249D1D4F8D80017
:10CCF800A18E884205DA4EF6F6400126C0F60000FD
:10CD080031E0D4F8E400B4F93C104FF47A7251439E
:10CD1800884205DA4EF6FC700226C0F6000022E0D2
:10CD2800B4F9CE00B4F94810884205DD4DF28620EA
:10CD38000326C0F6000016E0B4F9CC00B4F9481098
:10CD4800884205DD04264EF6D540C0F600000AE00C
:10CD5800B4F9CE00B4F94C10884254DA4EF63B20B0
:10CD68000526C0F60000FEF71EFD40F20040C4F69E
:10CD780000004FF400610022A4F80661F7F726F9D5
:10CD8800B4F8060100289FD0D4F8D800E18E884274
:10CD98009ADDD4F8E400B4F93C104FF47A725143A8
:10CDA800884291DDB4F9CE00B4F94A108842BFF642
:10CDB8008BAFB4F9CC00B4F94A108842BFF684AFFF
:10CDC800B4F9CE00B4F94E1088427FF77DAFB4F9BC
:10CDD800CC00B4F94E1088427FF776AFB4F806015C
:10CDE80002283FF471AFB4F8060107283FF46CAF8E
:10CDF8004DF2DE20C0F60000FEF7D5FC0020A4F8B6
:10CE08000601012258E7B4F9CC00B4F94C10884265
:06CE1800B6DA062697E7DA
:0ACE1E0052656620493D25660A00B2
:10CE280070B540F20004C1F20004B4F8760041F293
:10CE38002E35C1F2000598B1B4F8760001281ABF62
:10CE4800B4F876000022012240F20040C4F6000047
:10CE58004FF48051F7F7BAF8B4F87600288070BD1F
:10CE6800288800284FF6FF7018BFA4F80401B4F80A
:10CE7800041119B1B4F80411814255D1D4F8D8007D
:10CE8800218F884205DD4FF22C000126C0F60000F4
:10CE98003DE0D4F8E400B4F93E104FF47A725143FF
:10CEA800884205DD4FF214000226C0F600002EE08D
:10CEB800B4F9CE00B4F94010884205DD4DF2923045
:10CEC8000326C0F6000022E0B4F9CC00B4F9401003
:10CED800884205DD4EF638500426C0F6000016E0FC
:10CEE800B4F9CE00B4F94410884205DA4EF65E2053
:10CEF8000526C0F600000AE0B4F9CC00B4F94410E5
:10CF0800884211DA4EF617500626C0F60000FEF7E2
:10CF18004AFC40F20040C4F600004FF48051002261
:10CF2800A4F80461F7F752F8B4F80401002893D084
:10CF3800D4F8D800618F8842BFF68EAFD4F8E400E9
:10CF4800B4F93E104FF47A7251438842BFF684AF69
:10CF5800B4F9CE00B4F942108842BFF67DAFB4F9F7
:10CF6800CC00B4F942108842BFF676AFB4F9CE00CF
:10CF7800B4F9461088427FF76FAFB4F9CC00B4F922
:10CF8800461088427FF768AFB4F8040102283FF4DE
:10CF980063AFB4F8040107283FF45EAF4DF2D23016
:10CFA800C0F60000FEF7FFFB0020A4F804010122F0
:02CFB8004AE746
:10CFBA004552524F52204144535F313236305F4915
:0ECFCA006E7075744D757853656C65637400F8
:10CFD80070B540F20004C1F20004B4F8BC0041F29C
:10CFE8002035A0F10A06B4F8BC00D4F8D4100A30F1
:10CFF8008142C1F200051CD9B4F8500141F26F71A9
:10D00800884216D82878A0B94EF68120C0F60000CC
:10D01800FEF7C9FB01202870B4F8C0004FF4005196
:10D02800B0FA80F0420940F60000C4F60000F6F7B6
:10D03800CDFFD4F8D400B04203D22878012808D014
:10D048001EE0B4F8500141F27171884218D3287873
:10D05800B0B14FF24C00C0F60000FEF7A4FB002070
:10D068002870B4F8C02040F60000002A18BF01223A
:10D07800C4F600004FF40051BDE87040F6F7A6BFB3
:02D0880070BD79
:10D08A00466972737420737461727420646574657E
:06D09A00637465642100CF
:10D0A000F0B581B040F20005C1F20005D5F80001ED
:10D0B000B5F8BC104FF47A7740F60004794341F29A
:10D0C0001C36C4F600048842C1F2000613DD307835
:10D0D00088B94EF68C20C0F60000FEF768FB0120F0
:10D0E0003070B5F8C0004FF40051B0FA80F042093A
:10D0F0002046F6F76FFFD5F80001B5F8BE1079436A
:10D10000884216DA3078A0B14FF25800C0F600001D
:10D11000FEF74DFB00203070B5F8C0202046002AF5
:10D1200018BF01224FF4005101B0BDE8F040F6F7FE
:06D1300051BF01B0F0BD8B
:0ED1360075617274206572726F72200A0D00AE
:10D14400B0B540F2000441F22A30C1F20004C1F249
:10D154000000B4F9CE10B0F90000A0F5FA708842CE
:10D164005CDBB4F9CC10884258DB41F22830C1F2C0
:10D174000000B4F9CE10B0F9000000F5FA7088424E
:10D184004CDCB4F9CC10884248DC41F22630C1F2C0
:10D194000000B4F9CE10B0F90000A0F5FA7088428E
:10D1A4003CDBB4F9CC10884238DB41F22230C1F2C6
:10D1B4000000B4F9CE10B0F9000000F5FA7088420E
:10D1C4002CDCB4F9CC10884228DC41F22C30C1F2BA
:10D1D4000000D4F8E410B0F900204DF6F0054FF04B
:10D1E400FF33CFF6FF754FF47A70C2FB00536A1A0F
:10D1F40073EBE17112DB41F21E33C1F20003D4F888
:10D20400E410B3F90030002542F21072C3FB00258C
:10D214004FEAE17C881A7CEB05001DDA41F22435E3
:10D22400C1F20005287800B1B0BD4EF65950C0F6E1
:10D234000000FEF7BAFA01202870B4F8C000B0FA72
:10D2440080F0420940F60000C4F600004FF400519B
:10D25400BDE8B040F6F7BCBE41F22435C1F200058A
:10D2640028780028E0D14DF20640C0F60000FEF711
:10D274009CFA00202870B4F8C020002A18BF0122AC
:02D28400E0E7E1
:10D286004F5554505554535F4C56505F5348554E66
:10D29600545F4F56455254454D5045524154555290
:02D2A600450041
:10D2A80040F20000C1F20000B0F8BA00032803D829
:10D2B800DFE800F0020F0B0D40F60000C4F6000096
:10D2C8004FF400510022F6F781BEFFF7E5BEFFF7E5
:06D2D80035BFFFF77DBE2B
:0ED2DE004F5554505554204C5650204F4B0085
:10D2EC0040F20000C1F2000040F20A21018000214E
:10D2FC004FF0FF324FF0010C4FF00043C0F82411F7
:10D30C00C0F82011A0F81421C0F80C21C0F810218D
:10D31C00A0F81C21A0F81E21A0F81821A0F81A21B1
:10D32C00A0F808C041818181C0F8E8306FF000435B
:10D33C00C0F8EC304FF4004348F20002A0F8D030B3
:10D34C0047F6FF73CFF6FF72A0F8D230C0F8DC209E
:10D35C00C0F8E030A0F882110321A0F826C00185A6
:10D36C0005214185612180F8A011622180F8A1116D
:10D37C00792180F8B6117A2180F8B7114FF47A71BF
:06D38C00A0F8D611704765
:10D392004F5554505554535F4F56505F5348554E56
:10D3A200545F4F56455254454D5045524154555283
:02D3B200450034
:10D3B40040F20000C1F20000D0F84811D0F8482132
:0ED3C400002948BF5242C0F81021F8F75DBFA3
:0ED3D2004F5554505554204F5650204F4B008D
:10D3E00040F20000C1F20000016E4FF46162A1FB47
:10D3F0000212C0E95C120021C0E95A11C0F84811BC
:06D40000C0F82011704786
:10D40600415558206F66662028416C61726D204D2B
:06D416006F6465290D00A2
:10D41C004EF68850CEF20000016841F470010160B4
:02D42C00704747
:10D42E0053756E646179004D6F6E64617900547549
:10D43E006573646179005765646E65736461790024
:10D44E00546875727364617900467269646179001B
:0AD45E005361747572646179000077
:10D4680041F20C0CC4F2020C5CF8041C42F20042BB
:10D47800C1F3810341F28071C0F2F402C1F20001EC
:10D48800DFE803F02928020743F20062C0F26E12B7
:10D4980020E0DCF80000DCF8003000F0030002288F
:10D4A80043F20060C3F30313C0F26E1003F10103EB
:10D4B80008BF1046DCF80020B0FBF3F0DCF80030C1
:10D4C800C2F306225043C3F34162022303EB420234
:10D4D800B0FBF2F20A605CF8040C4FF26C02C0F385
:10D4E8000310C0F60002105C0A6822FA00F0086017
:02D4F80070477B
:02D4FA002E0002
:10D4FC0030B591EA030F00F18280841A71EB030CB2
:10D50C0005D2121953EB0C03001B71EB0C0140F20A
:10D51C00000CCFF6E07C1CEA430F52D0BCEB410F61
:10D52C005FD90C0DA4EB135E5FF0010C6CF31F5173
:10D53C006CF31F53DEF1200C2AD303FA0CF54019BF
:10D54C0041F1000122FA0EF5401923FA0EF569415A
:10D55C0012FA0CF2CD0208D349085FEA30005FEAF8
:10D56C00320228BF42F00102641C641E5FEA500CB8
:10D57C0072F1004250F1000051EB04514FF40013D2
:10D58C0013EB410F38BF30BD6FF31301002030BDDA
:10D59C00BEF1200EBEF1200F1ED223FA0EF540195B
:10D5AC0041F10001CEF1200C124218BF012203FA06
:10D5BC000CF52A43CEE711EA5C0F04BF00200021D2
:10D5CC0030BD1CEA410F04BF01F00041002030BD0A
:10D5DC0001F00041002030BD21F4801101EB045119
:10D5EC0030BD004218BF41F00101BCEB410F08BF38
:10D5FC0030BD4FF0FE4141F47801002030BD83F086
:10D60C000043841A71EB030E07D28EF0004E001B00
:10D61C0071EB0E01121953EB0E0340F2000CCFF616
:10D62C00E07C1CEA430FC6D0BCEB410F72D90C0D49
:10D63C00A4EB135EC90241EA5051C00241F0004113
:10D64C00DB0243EA5253D20243F00043DEF1200CDA
:10D65C0041D312FA0CF522FA0EF203FA0CF542EA57
:10D66C00050218BF42F0010223FA0EF3801A994109
:10D67C00E30AC4F30A0411F0404F03D418D0641E1B
:10D68C0040004941641E23D44205C00A40EA41507F
:10D69C00C90A51EAC3715FEA500C72F1004250F1B1
:10D6AC00000051EB045130BD01002FD00020203C74
:10D6BC000029F9D0B1FA81FCDCF1200E11FA0CF141
:10D6CC0030FA0EF510FA0CF02943A4EB0C04D9E750
:10D6DC000020D90730BDAEF1200EBEF1200F0DD2C7
:10D6EC00CEF1200C03FA0CF533FA0EF32A4318BFD3
:10D6FC0043F00103C01A61F10001B9E721F00041C8
:10D70C00C00A40EA4150C90A01EB045130BD002067
:10D71C00002130BD004218BF41F00101BCEB410FAC
:0ED72C007FF467AFBCEB430F3FF463AF30BD3B
:01D73A0000EE
:10D73C002DE9F04391EA030E0EF0004E40F2000783
:10D74C00CFF6E07717EA41051EBFBD4217EA430545
:10D75C00BD4200F09F807F0D17EA135623EA475312
:10D76C0043F4801317EA115521EA475141F4801113
:10D77C00AD1B05F2FD354FEAD31C1CF1010C4FF02B
:10D78C000047B7FBFCF77F01A2FB079C0024E3FBDF
:10D79C0007C4D9F100096CEB4C0CA0FB076200200C
:10D7AC00E1FB072000275FEAC628E0FB0987760D1E
:10D7BC0046EAC226520DF61900277A41E0FB0C62AC
:10D7CC005FEAC823E2FB09375FEA585848EAC628E3
:10D7DC00760D18EB070800214E41E2FB0C8602EB9C
:10D7EC00C020DA02E6FB09215B0D43EAC8235FEA9D
:10D7FC0058585B18002758EB0708E6FB0C38D10289
:10D80C00E8FB0917520D42EAC3225B0DD21900271F
:10D81C007B41E8FB0C2308EBC6265FEAC128E3FB3F
:10D82C000987490D41EAC221520DC91942F1000282
:10D83C00E3FB0C12470019EB08095CEB010C72EBD3
:10D84C00040453EBC62047EB56530026B3F5000FE8
:10D85C007641AD19B61CD6F1200910FA09F4F04046
:10D86C0013FA09F21043F340E40F001943F10003DB
:10D87C00B3F5001F24BF5B086D1C40F2FE77BD4260
:10D88C0004D24EEA05511944BDE8F0832D4224D54B
:10D89C00714626E0004218BF41F00101124218BF48
:10D8AC0043F00103B7EB410F2CBFB7EB430F1BE069
:10D8BC00B7EB410F04BFB7EB430F15E017EA410F6D
:10D8CC0004BF17EA430F0FE017EA410FE0D017EA45
:10D8DC00430F02D0B7EB430FDAD04EF0FE4141F4C8
:10D8EC0070010020BDE8F08340F20001C7F6F8712A
:02D8FC00F7E74C
:10D8FE0057726F6E6720706172616D6574657273B9
:10D90E002076616C75653A2066696C6520257320FA
:0DD91E006F6E206C696E652025640D0A0097
:0DD92B004144533132363020496E6974009A
:10D93800C1F30A5340F21E42D21A0EDD202A0AD839
:10D94800CB0243EA505040F00040D04090EAE170EA
:10D95800B0EBE1707047002070474B00004218BFE1
:10D9680043F0010313F5001F88BF21F0004111F0B7
:0AD97800004058BF6FF000407047F8
:10D9820053484F52545F434952435549545F505292
:09D992004F54454354494F4E0027
:10D99B004A756D7020686173206661696C656421DE
:01D9AB00007B
:10D9AC0010F0004160B148BF40420A0D02F21D4226
:10D9BC00B0FA80F3D21A9840C30A400503EB025127
:02D9CC007047A2
:10D9CE002E2E2E466C617368206F6220756E6C6F02
:05D9DE00636B656400AD
:10D9E3002E2E2E44697361626C65206C6F636B200D
:10D9F30070726F636573732066696E6973686564BB
:01DA03000022
:10DA040070B5CC1760406140001BA141DD176A402E
:10DA14006B40521BAB4100F029F862406340121B7B
:0EDA2400A3416C4060406140001BA14170BDF9
:10DA3200466C617368204F7074696F6E62797465A9
:10DA42002070726F6772616D6D206661696C6564CA
:01DA520000D3
:10DA53002E2E2E466C617368206C6F636B20616C95
:0DDA63007265616479206163746976650005
:10DA7000002B35D129B9B0FBF2FC0CFB1202604639
:10DA80007047914215D22DE9F041B2FA82F39A40E3
:10DA90009940D3F1200C30FA0CFC51EA0C0198406B
:10DAA00000F04EF8280036FA03F200210023BDE80A
:10DAB000F081F0B5B1FBF2FC0CFB1211B2FA82F36B
:10DAC0009A409940D3F1200630FA06F63143984047
:10DAD00000F036F8614628003200DA400023F0BD3D
:10DAE000F3B5B3FA83FC49085FEA300013FA0CF38C
:10DAF000DCF1200432FA04F423430CB41A0000F0E1
:10DB00001FF80CBC33FA0CF3DCF11F0C35FA0CF5E2
:10DB100018BF6D1E03BCA5FB026705FB0377801BC6
:10DB2000B941904271EB030C05D3821A71EB0303E8
:10DB3000681C0021F0BD02000B0028000021F0BD90
:10DB4000940D4FF6C2752D02B5FBF4F4D60A761C7F
:10DB500004FB04F5A5FB0656F64306EB0416550830
:10DB600032BF002777086D1C05FB1677A6FB074719
:10DB70007F0807EBC63714001500E7FB02457F1B43
:10DB80004D1C0400E7FB014505FB1206A64284BFBD
:0EDB90006D1EB618964224BF6D1CB61A704763
:10DB9E002E2E2E456E61626C65206C6F636B206558
:05DBAE0072726F7200AD
:10DBB300443A5C50726F6A656B74655C656373535A
:10DBC3006D61727450726F5C7472756E6B5C6677A4
:10DBD3005F673437337263745C447269766572735A
:10DBE3005C53544D3332473478785F48414C5F443B
:10DBF30072697665725C5372635C73746D333267FA
:10DC03003478785F68616C5F6164635F65782E6305
:01DC13000010
:10DC14002DE9F04F89B01546894682460020CAF89E
:10DC240000000DF10E0819F8011B252906D0002962
:10DC340000F04F82504600F067FBF4E72C460027C3
:10DC44004A4619F8010BA0F12003102B0DD88021AE
:10DC5400DFE803F0091B1B191B1B1B151B1B3018CA
:10DC64001B101B1B120040210DE05E280DD14FF448
:10DC7400805108E0102106E04FF4007103E04FF4F6
:10DC8400004100E020210F43DAE7A0F13001C9B2DE
:10DC940009294FF000010BD801EB810100EB410190
:10DCA40019F8010BA0F13002D2B230390A2AF3D3A9
:10DCB40025460CE0254655F8040B010048BF4142B7
:10DCC400102303EAD060074302F1020950782E289A
:10DCD4000BD14A4612F8010B2A2809D155F804BB86
:10DCE40099F8010009F1020218E04FF0000B1EE060
:10DCF400A0F13003DBB2092B4FF0000B14D80BEB6F
:10DD04008B0300EB430312F8010BA0F130095FFA17
:10DD140089F9B9F10A0FA3F1300BF0D3BBF1000F6D
:10DD240004D447F4807701E047F480779146A0F16A
:10DD34006802D3B2D20142EA5302D2B2092A22D8EB
:10DD4400DFE802F0050E122121210F21210F4A469E
:10DD540012F8010B682812D199F8010008370BE07A
:10DD6400023719F8010B0EE04A4612F8010B6C2831
:10DD740007D199F80100023709F1020903E00437D9
:10DD840000E001379146622821EAE17620DDA0F126
:10DD9400630115293FF647AFDFE811F0380017009B
:10DDA40016001600160016001700160016001600BE
:10DDB40016009A00440006011600160029001600F9
:10DDC4004E001600160022002DE747F4804737E086
:10DDD400252800F08A80582840F08C8147F40057A9
:10DDE40043F2580278281ED143F278021BE00195D1
:10DDF4002D68002D04BF4EF69F25C0F60005F805DA
:10DE0400284600F1458100F0D1FB44E12C78013E25
:10DE140050463946324600F0C9FA5046214600F0D1
:10DE240073FA4AE13022390602EAE1710291F905F6
:10DE340008D527F4007705E0F90548BF27F40077F3
:10DE44000021029179044FEA8771009604D40029D5
:10DE540009D4291D00240CE0002913D4294651F8C3
:10DE6400045BEC1714E0E91D21F0070505F1080136
:10DE74006C687A072D6814D417F0080F13D00024A7
:10DE8400EDB210E0E91D21F007014C6851F8085B80
:10DE94000191790709D439070AD545F3C0146DB245
:10DEA40006E0ADB20024019126E045F3C0342DB262
:10DEB400002C07DBB9061DD47906029A48BF20223C
:10DEC400029219E000216D4261EB04042D2112E05D
:10DED40055F8040B3907DAF8001000F1F880BA0796
:10DEE40052BF0160002206C09DE65046252100F085
:10DEF4000BFA98E62B210291F90548BF27F4007725
:10DF0400F90558BF4FF0010B00266E2821DD6F384C
:10DF1400092800F27980DFE800F0055677777777F3
:10DF24002277775655EA04006ED0E80840EA447038
:10DF3400062262F3DF0508F80650013650EAD401E0
:10DF44004FEAD4044FEAD001054641EA4470F0D1C7
:10DF54005AE0582837D0642818BF692854D155EAA4
:10DF6400040051D0380407D506F00300032802BF8B
:10DF74002C2008F806000136284621460A220023F0
:10DF8400FFF774FD00EB8002A5EB4202D5F1090313
:10DF94000023A34142F0300208F8062006F10106EE
:10DFA40005460C46DED32FE02846009650F8045B65
:10DFB40001903806232101EAE070029047F480774B
:10DFC40000244FF0080B002655EA04001CD04FF241
:10DFD4008400C0F60000B9045CBF4FF29400C0F6A0
:10DFE4000000290941EA047105F00F020D46825C24
:10DFF40008F80620013651EA14114FEA14144FEAC6
:10E00400151141EA0471EFD1ABEB060020EAE07B85
:10E0140006EB0B000099029D0C1A4FF0FF30FF2D08
:10E0240088BF0138002D18BF0444B80505D45046F4
:10E034003946224600F0BAF90024FF2D04D9290AF2
:10E04400504600F061F900E01DB15046294600F049
:10E054005BF950463946224600F0A8F95046302173
:10E064005A4600F093F9012E08DB751E504618F845
:10E07400051000F049F9012E2E46F6D8F806019D48
:10E084007FF5D1AD50462021224600F07FF9CAE544
:10E09400594600F0A1FA044627F40077361A504690
:10E0A4003946324600F082F934B115F8011B504666
:10E0B40000F02AF9013CF8D1019D0435F8067FF5FA
:10E0C400B2AD50462021324600F060F9ABE5017054
:10E0D400A9E5DAF80C0028B1DAE9001291423CBF54
:10E0E400002242545046FDF7B8FDDAF8000009B0AA
:10E0F400BDE8F08F00287FF496AD5046FDF7ADFDE6
:06E104004FF0FF30F3E7CD
:10E10A00443A5C50726F6A656B74655C65637353FD
:10E11A006D61727450726F5C7472756E6B5C667747
:10E12A005F673437337263745C44726976657273FD
:10E13A005C53544D3332473478785F48414C5F44DE
:10E14A0072697665725C5372635C73746D3332679D
:10E15A003478785F68616C5F636F727465782E6378
:01E16A0000B4
:10E16B00443A5C50726F6A656B74655C656373539C
:10E17B006D61727450726F5C7472756E6B5C6677E6
:10E18B005F673437337263745C447269766572739C
:10E19B005C53544D3332473478785F48414C5F447D
:10E1AB0072697665725C5372635C73746D3332673C
:10E1BB003478785F68616C5F6372635F65782E6338
:01E1CB000053
:10E1CC004AB1884207D007D28018891852428B5C1A
:10E1DC008354521CFBD17047521E8B5C8354FBD171
:02E1EC0070477A
:10E1EE00443A5C50726F6A656B74655C6563735319
:10E1FE006D61727450726F5C7472756E6B5C667763
:10E20E005F673437337263745C4472697665727318
:10E21E005C53544D3332473478785F48414C5F44F9
:10E22E0072697665725C5372635C73746D333267B8
:10E23E003478785F68616C5F6932635F65782E63EE
:01E24E0000CF
:10E24F00443A5C50726F6A656B74655C65637353B7
:10E25F006D61727450726F5C7472756E6B5C667701
:10E26F005F673437337263745C44726976657273B7
:10E27F005C53544D3332473478785F48414C5F4498
:10E28F0072697665725C5372635C73746D33326757
:10E29F003478785F68616C5F7077725F65782E6332
:01E2AF00006E
:10E2B000010002000400060008000A000C00100023
:08E2C000200040008000000175
:10E2C80051EC102BC1F30A53002B1CBF40F2FF7C0A
:10E2D800634514D01844604506DB0020C7F6F0708B
:10E2E80060F31E01002208E00028C7BF6FF31E512B
:10E2F80041EA005101F00041002241EC102B704727
:04E30800F4F71EB94F
:10E30C0010B582B0044600698DF8071078B1D4E9D5
:10E31C0000239A4231D26269531C63618154D4E95F
:10E32C000501884229D12046FDF793FC25E0E068E1
:10E33C0050B1D4E9002C62451FD2531CB3EB0C0333
:10E34C0018BF0B46835418E0A06858B1D4E9002CD0
:10E35C00624512D2531CB3EB0C0318BFCBB240F87E
:10E36C0022300AE0236A43B1D4E90001884204D286
:10E37C000DF10701204601229847206801302060EA
:04E38C0002B010BD0E
:10E39000012A0CDBF8B514460D460646671E3046CA
:10E3A0002946FFF7B3FF012C3C46F7D8F8BD70476C
:10E3B000CB0606D43023890558BF20231946FFF722
:04E3C000E7BF7047FC
:10E3C40070B514460D460646F8F7CEF901463046B8
:0CE3D4002A462346BDE8704000F000B867
:10E3E0002DE9F04F03AF8DB047F83C3C91460C4609
:10E3F000064600F05BF80546EB46073020F00700C4
:10E40000ADEB0008C546A7F1380A5046002124228A
:10E41000F8F77CF947E908546FF0004047F8340CEE
:10E420004BF6BB40C0F6000047F8288C47E90606CB
:10E430005046494657F83C2CFFF7ECFBDD46A7F168
:08E440000C04A546BDE8F08FB5
:10E4480083B000B582B0CDE9031241F2747CC1F209
:10E45800000C059303AA01920146DCF80000FFF7BF
:0CE46800ADFF02B05DF804EB03B070479C
:10E4740041F27871C1F2000141F27472C1F20002FA
:10E484000968126841F27C73C1F20003411A1B68E7
:10E4940018BF0121821A18BF01221140C01A18BFE7
:08E4A4000120084040427047CE
:04E4AC004020704755
:10E4B00040F6E410C1F2000003214EF67F52C0F690
:10E4C00000020161416141F23631C1F20001826115
:10E4D000C1614FF480610162002181624162C162C9
:10E4E00041F23673C1F2000302664366102282666F
:10E4F0000167C1664EF66E52C0F600024167BFF377
:10E500005F8F531ADB7B435401311029F9D1BFF3DC
:04E510005F8F704762
:10E514002DE9F04104468068E66815466268871B69
:10E524009019BD4206D22A46F8F7BCF8BFF35F8FB4
:10E5340035440CE088463A46F8F7B4F8ED1B08EB8E
:10E54400070160682A46F8F7ADF8BFF35F8FE5600E
:04E55400BDE8F081AD
:10E5580070B500EB400040F6E413C1F2000303EB92
:10E56800C00303F11806D86A022818D00D461446CD
:10E57800012807D020B93046FDF7F5FBA04207D2A5
:10E5880000240AE03046FDF7EEFBA04238BF0446FF
:10E59800304629462246FFF7B9FF204670BD30466F
:08E5A800BDE87040FDF7EBBB7C
:10E5B000017889B14FF0013C0346194653F8042B0A
:10E5C000CCFA52F2002AF8D092FAA2F2B2FA82F20F
:0CE5D00001EBD201081A704700207047D0
:10E5DC0000291CBF0278002A01D10020704700B529
:10E5EC000429D0F800E0024609D34FF0013CCCFAE4
:10E5FC005EF323B90439032952F804EFF7D84FF02E
:10E60C000133C3FA5EF393FAA3F3B3FA83F3101A4C
:0CE61C00B1EBD30F88BFD908084400BD43
:10E628007F280BD84FF2A402C0F600024EF6E8533A
:10E63800C0F60003105C595C084070470020704722
:0CE64800A0F161011A2938BF203870478A
:0CE65400A0F141011A2938BF20307047A6
:10E660007F280BD84FF2A402C0F600024EF6E85302
:10E67000C0F60003105C595C0840704700207047EA
:0CE68000A0F161011A2938BF2038704752
:0CE68C00A0F141011A2938BF203070476E
:0FE698005465737420646562756720696F0D00A7
:10E6A700666163746F727920726573746F72652E19
:03E6B7002E2E0004
:0FE6BA006572726F722068616E646C65720D001C
:10E6C900466C61736820756E6C6F636B206572723E
:03E6D9006F72005D
:10E6DC00443A5C50726F6A656B74655C6563735326
:10E6EC006D61727450726F5C7472756E6B5C667770
:10E6FC005F673437337263745C4472697665727326
:10E70C005C53544D3332473478785F48414C5F4406
:10E71C0072697665725C5372635C73746D333267C5
:10E72C003478785F68616C5F666C6173685F65787C
:03E73C002E630049
:10E73F00443A5C50726F6A656B74655C65637353C2
:10E74F006D61727450726F5C7472756E6B5C66770C
:10E75F005F673437337263745C44726976657273C2
:10E76F005C53544D3332473478785F48414C5F44A3
:10E77F0072697665725C5372635C73746D33326762
:0FE78F003478785F68616C5F6770696F2E630024
:10E79E00443A5C50726F6A656B74655C6563735363
:10E7AE006D61727450726F5C7472756E6B5C6677AD
:10E7BE005F673437337263745C4472697665727363
:10E7CE005C53544D3332473478785F48414C5F4444
:10E7DE0072697665725C5372635C73746D33326703
:0FE7EE003478785F68616C5F697764672E6300C9
:10E7FD00443A5C50726F6A656B74655C6563735304
:10E80D006D61727450726F5C7472756E6B5C66774D
:10E81D005F673437337263745C4472697665727303
:10E82D005C53544D3332473478785F48414C5F44E4
:10E83D0072697665725C5372635C73746D333267A3
:0FE84D003478785F68616C5F756172742E630058
:0FE85C0049205265666572656E7A3D25660A0031
:0BE86B00547368756E743D25660A004A
:10E876002D2D2D204761696E2044726966742043F0
:07E88600414C202D2D2D0057
:0FE88D0041637475616C20543D256620430A0079
:10E89C0041637574616C20493D2566204128776978
:10E8AC0074686F7574206761696E2074656D702073
:10E8BC00647269667420636F7272656374696F6EDB
:03E8CC00290A0016
:10E8CF004B6F7272656B74757266616B746F723DAC
:10E8DF002566205B2031202F2043656C736975738B
:03E8EF005D0A00BF
:10E8F2004552524F52204144535F313236305F53BA
:0BE9020065744461746152617465002B
:10E90D004552524F52204144535F313236305F539E
:0BE91D00657443686F704D6F64650007
:10E9280054696D652025643A20456D7074792065B9
:10E9380076656E742831292C20636E3D25642C2061
:10E9480063613D25642C2074446973636861726750
:10E95800653D25642C20753D25642C20693D256482
:03E968000D0A0095
:10E96B0054696D652025643A20456D707479206576
:10E97B0076656E742832292C20636E3D25642C201D
:10E98B0063613D25642C207444697363686172670D
:10E99B00653D25642C20753D25642C20693D25643F
:03E9AB000D0A0052
:10E9AE00454550524F4D20776173206368616E6705
:10E9BE00656421205765206E65656420746F207034
:10E9CE00726573657276652063616C6962726174DB
:10E9DE00696F6E20616E642073657474696E6773FF
:07E9EE002064617461210047
:10E9F500454550524F4D20464143544F52592052A0
:0FEA05004553544F52452F55504441544521001D
:10EA140055617274204572726F7220626569206E4E
:10EA240065757374617274206E61636820466568ED
:07EA34006C6572200A0D0061
:10EA3B004F5554505554535F4C56505F5348554E99
:10EA4B00545F554E44455254454D504552415455D3
:03EA5B0052450021
:10EA5E004F5554505554535F4F56505F5348554E73
:10EA6E00545F554E44455254454D504552415455B0
:03EA7E00524500FE
:0BEA8100486561746572206F6E0D0027
:10EA8C00415558206F6E2028534F43204D6F6465BD
:03EA9C00290D0041
:07EA9F00286E756C6C290064
:10EAA6004A616E7561727900466562727561727946
:10EAB600004D6172636800417072696C004D617946
:10EAC600004A756E65004A756C7900417567757305
:10EAD600740053657074656D626572004F63746F80
:10EAE600626572004E6F76656D626572004465639D
:07EAF600656D62657200000E
:07EAFD00414D00504D0000E7
:0FEB0400256120256220256520255420255900F4
:10EB1300443A5C50726F6A656B74655C65637353EA
:10EB23006D61727450726F5C7472756E6B5C667734
:10EB33005F673437337263745C44726976657273EA
:10EB43005C53544D3332473478785F48414C5F44CB
:10EB530072697665725C5372635C73746D3332678A
:10EB63003478785F68616C5F7263635F65782E6386
:01EB730000A1
:10EB7400443A5C50726F6A656B74655C6563735389
:10EB84006D61727450726F5C7472756E6B5C6677D3
:10EB94005F673437337263745C4472697665727389
:10EBA4005C53544D3332473478785F48414C5F446A
:10EBB40072697665725C5372635C73746D33326729
:10EBC4003478785F68616C5F7274635F65782E6314
:01EBD4000040
:10EBD500492028776974686F757420636F6D706557
:0DEBE5006E736174696F6E293D25660A002C
:10EBF2004144535F313236305F42617474657279D9
:10EC020043757272656E744761696E43616C6962C5
:10EC1200726174696F6E53746172743A2045525214
:10EC22004F5220494E2043414C4942524154494F90
:10EC32004E2C204E4F205245464552454E434520CC
:09EC420043555252454E54210085
:10EC4B004E6F726D616C207374617274207769748E
:10EC5B00686F757420454550524F4D206368616E47
:0DEC6B0067657320646574656374656400FB
:10EC7800454550524F4D2046554C4C205245535413
:05EC88004F5245210080
:10EC8D00454550524F4D2053544F524520434F4E02
:05EC9D0046494721007B
:10ECA2004D4220444D41204572726F7221200A0D5F
:01ECB2000061
:10ECB3004D42204F5245204572726F7221200A0D3A
:01ECC3000050
:10ECC4004552524F52205561727420494E49540D99
:01ECD400003F
:10ECD5004F5554505554535F4C56505F4348495017
:10ECE5005F4F56455254454D504552415455524536
:01ECF500001E
:10ECF6004F5554505554535F4C56505F42415454EF
:10ED06004552595F554E444552564F4C544147451E
:01ED160000FC
:10ED17004F5554505554535F4F56505F43484950D1
:10ED27005F554E444554454D504552415455524503
:01ED370000DB
:10ED38004F5554505554535F4F56505F43484950B0
:10ED48005F4F56455254454D5045524154555245D2
:01ED580000BA
:10ED5900415558206F6E2028416C61726D204D6FAE
:05ED69006465290D00A6
:10ED6E0000000000000054545220524547474553BE
:01ED7E000094
:09ED7F005465726D696E616C004F
:09ED8800256D2F25642F2579006B
:09ED910025483A254D3A255300AE
:10ED9A0053756E004D6F6E005475650057656400BB
:0DEDAA0054687500467269005361740000E2
:10EDB7004A616E00466562004D61720041707200E3
:10EDC7004D6179004A756E004A756C0041756700A0
:10EDD700536570004F6374004E6F7600446563009F
:01EDE700002B
:0DEDE80000070320041702010857104080A7
:10EDF8008C6700088C6700088C6700088C6700081F
:04EE08008C6700080B
:04EE0C0069D40008BD
:10EE1000554E4B4E4F574E20434F4D4D414E4400A3
:10EE2000466C617368204F7074696F6E62797465A7
:0CEE30002070726F6772616D6D65640088
:10EE3C00537461727420656E61626C6520726561D9
:10EE4C00646F75742070726F74656374696F6E0093
:10EE5C002E2E2E466C61736820756E6C6F636B0082
:10EE6C00466C617368204F7074696F6E627974655B
:08EE7C00206C6F636B656400FC
:10EE84002E2E2E456E61626C65206C6F636B207054
:10EE9400726F636573732066696E69736865640075
:10EEA400443A5C50726F6A656B74655C6563735356
:10EEB4006D61727450726F5C7472756E6B5C6677A0
:10EEC4005F673437337263745C4472697665727356
:10EED4005C53544D3332473478785F48414C5F4437
:10EEE40072697665725C5372635C73746D333267F6
:10EEF4003478785F68616C5F666463616E2E63006A
:08EF04000101010307010000F7
:08EF0C000804020408010101E0
:10EF14004B6F7272656B74757266616B746F723D60
:04EF240025660A0054
:10EF28002D2D2D204761696E204472696674204337
:0CEF3800414C20454E4445202D2D2D005D
:10EF44004552524F52204144535F313236305F5361
:10EF54006574496E7465726E616C5265666572653E
:04EF64006E63650073
:10EF680054696D652025643A20426174746572693C
:10EF7800652046756C6C206576656E74206D4168F9
:10EF88004361726765643D25642C2074436861722F
:10EF980067653D25642C2063656641683D25642CC2
:10EFA8002063656657683D25642C20753D25642CD3
:08EFB80020693D25640D0A00EB
:0CEFC00057726974696E6720534E21007F
:10EFCC004D42204645204572726F7221200A0D0079
:10EFDC004D42205045204572726F7221200A0D005F
:10EFEC004D42204E45204572726F7221200A0D0051
:10EFFC004F5554505554535F4C56505F4F564552D5
:08F00C0043555252454E5400D9
:10F014004F5554505554535F4F56505F4F564552B9
:08F0240043555252454E5400C1
:10F02C004F5554505554535F4F56505F42415454B2
:10F03C004552595F4F564552564F4C544147450027
:0CF04C00486561746572206F66660D00F7
:10F05800415558206F66662028534F43204D6F64F2
:04F0680065290D0009
:10F06C00000000000000000001020304060708096C
:08F07C00000000000102030482
:10F0840030313233343536373839414243444546DA
:10F09400303132333435363738396162636465660A
:10F0A40020202020202020202068282828282020F4
:10F0B400202020202020202020202020202020204C
:10F0C4004810101010101010101010101010101004
:10F0D40084848484848484848484101010101010A4
:10F0E40010818181818181010101010101010101FD
:10F0F40001010101010101010101011010101010B1
:10F1040010828282828282020202020202020202CD
:10F114000202020202020202020202101010102075
:10F1240000B506480649884205D00268043003B495
:10F13400904703BCF7E708BC184700000CEE000832
:04F1440010EE0008C1
:10F14800E5F10008000000101D130000E5F10008BB
:10F158001E13001003000000E5F100082213001040
:10F1680003000000E5F10008261300102004000049
:10F17800E5F100088417001004000000E5F100081C
:10F18800000000205C030000F7F100088817001059
:10F19800B8F10008140000000BF200084C1700102A
:10F1A800CCF100083800000025F1000807640008C9
:10F1B8008C6700088C6700088C6700088C6700085B
:10F1C8008C670008FFFFFE01FFEE100144C4121017
:0CF1D800C8121094CC121024F4000000A7
:10F1E400206861680834002200E04254491EFCD5BE
:02F1F400704762
:10F1F60020686168A2680C3401E08B5C8354521E5F
:04F20600FBD570477D
:10F20A0020686168A2680C340B78491C082600251E
:10F21A005B0801D20D78491C0570401C521E02D0B1
:08F22A00761EF4D1F0E77047F5
:04000005080064117A
:00000001FF
